:020000040800F2
:10000000F0FF0120E1AC04089D1D0408F97002080E
:1000100059AD040859AD040859AD040800000000AA
:10002000000000000000000000000000A31D040804
:10003000A11D0408000000009F1D04081D380208CF
:1000400059AD040859AD040859AD040859AD040868
:1000500059AD040859AD04086D7E0208997F020865
:100060005D7F0208217F0208E57E02089DC8000826
:100070008DC800087DC800086DC8000859C8000870
:1000800045C8000831C8000859AD04080000000048
:10009000000000000000000000000000A97E02082F
:1000A0005D1E02084922020859AD0408092302080E
:1000B00089210208C9200208FD1F0208A9EA0008D8
:1000C000B1EA000899EA0008A1EA000859AD04085D
:1000D00059AD0408F93802085D3802080000000034
:1000E000317E020859AD0408715404080000000074
:1000F0000000000000000000000000001DC8000813
:100100000000000059AD04082D1F020859AD040875
:1001100000000000000000000000000000000000DF
:1001200009C80008F5C70008E1C70008CDC70008E6
:10013000B9C7000800000000000000000000000037
:10014000000000000000000000000000A92C0408CE
:10015000A5C7000891C700087DC7000859AD04086D
:1001600089EA000891EA0008000000000000000091
:10017000000000000000000000000000000000007F
:100180000000000059AD040800000000000000005D
:0801900059AD040859AD040843
:0801980078A80400010000003A
:1001A00010020100842C0020802C002000000000A0
:1001B000DC0600080902010030460020F04600205D
:1001C00000000000DE0600080C109C008C4200209D
:1001D000F4460020000000002D93020801020500F3
:1001E00010420020904700200000000085F4000825
:1001F000000205000842002098470020000000008F
:10020000000000001B020800E4410020A04700207D
:1002100000000000B18300081E000500C43F00205C
:10022000A847002000000000E00600081B00F400C2
:10023000142D0020B047002000000000B10001088C
:100240000E0202009C440020A44800200000000090
:10025000E606000823001000A8460020A848002059
:1002600000000000296B01082F0011007C460020CF
:10027000B848002000000000E8060008051006004D
:10028000C4460020CC48002000000000FA06000808
:100290003710220098450020D448002000000000BC
:1002A00000070008F5418400882C0020F848002051
:1002B000000000006525010826000E008C49002082
:1002C0007C4900200000000061EB00082C001000B9
:1002D0006063002050630020000000004786010892
:1002E0002B002400946300207063002000000000B5
:1002F000198601082920780058620020B863002080
:1003000000000000000000001C021000306100200E
:100310003064002000000000BD83000814000300CA
:1003200078600020406400200000000022070008E0
:1003300010100200F45E0020446400200000000061
:100340002607000828101000E45E00204864002002
:1003500000000000116B010819000500DC5E0020A0
:10036000586400200000000028070008F82106005B
:10037000D45E002060640020000000002E0700080A
:100380000A6028008C4B00206864002000000000F8
:10039000C56A01080E604A01404A002090640020AE
:1003A000000000002918030801010400B0490020E2
:1003B000DC650020000000000000000000010400D7
:1003C000A8490020E0650020000000003407000874
:1003D00002010300A4490020E465002000000000A1
:1003E000AD9302081A023C00E4660020EC6A00208B
:1003F000000000003991000827000400E06600209A
:10040000286B0020000000003807000807020200E7
:1004100080760020A4760020000000003C07000841
:1004200002000C0058760020A87600200000000092
:100430000000000006020C004C760020B47600207C
:1004400000000000C991000808120900D4750020BE
:10045000C076002000000000E5830008F7010600D8
:10046000CC750020CC760020000000003E0700087C
:100470000A020A00EC700020D47600200000000080
:10048000FD97020803000100EC6B0020E0760020DD
:1004900000000000000000001A000E00807F002015
:1004A0009883002000000000440700080120080095
:1004B000507F0020A88300200000000052070008A1
:1004C000031233004A780020608200200000000000
:1004D0005A07000825102C01E07800203481002004
:1004E0000000000000000000F6210C004480002005
:1004F000288100200000000090070008150070000F
:10050000E8760020B8800020000000000000000015
:100510002A00600080780020588000200000000041
:1005200001180308161006001485002024850020F9
:10053000000000009C0700080B201000788F0020AE
:10054000D893002000000000A40700081F302400FA
:10055000FC860020E893002000000000B40700089B
:10056000050204007C9100200C9400200000000093
:10057000D807000803010A00288F002010940020EB
:1005800000000000DC070008130204007085002052
:100590001C94002000000000E60700080400800012
:1005A00058C3002064CD00200000000000000000BF
:1005B0000D002C00CCC10020E4CD00200000000084
:1005C00061BE0308F9010400ACB8002010CE002081
:1005D00000000000490E020813000400A8B8002023
:1005E00014CE002000000000EC070008FD012400EC
:1005F00084B8002018CE002000000000D10D0208B1
:1006000018202C0054B800203CCE00200000000030
:10061000E191000806101800A0AB002068CE002071
:1006200000000000B1180308FB010100D8AA002057
:1006300080CE0020000000004D920008FC0109005F
:10064000A4A9002084CE0020000000005D920008D4
:1006500034001000D0A8002090CE00200000000040
:100660008518030811020800A8A80020A0CE0020C9
:1006700000000000F007000812120400A0A80020EB
:10068000A8CE002000000000F8070008122010008B
:1006900090A80020ACCE002000000000FC0700085D
:1006A0000202030070940020BCCE00200000000075
:1006B000000000000C0204002C940020C0CE00209A
:1006C0000000000005840008FE011000D096002004
:0C06D000C4CE0020000000001D840008C3
:1006DC00000000000000010000000000000000000D
:1006EC0000000000000000000000000000002000DE
:1006FC000301000020003200C800D007960014004F
:10070C0032002800B00440060005500014000F0011
:10071C00080064000100030000000005000028012F
:10072C0000000401F40114009001000020030000FB
:10073C00013C2201000000007E05EA05B4053200F0
:10074C00E803D0070000E8036400040A000100007D
:10075C00000000000000000000000000000000008D
:10076C00000000000000000000000000000000007D
:10077C00000000000000000000000000000000006D
:10078C000100000000000000010000000202000057
:10079C00C4090000190000002B21231E6401010074
:1007AC00000001000A012900000000000001000007
:1007BC000005000001020300000000000000000022
:1007CC000000000000000000008007000000000096
:1007DC00040101006C16000000000000013F000045
:1007EC00480404300000000001010101FFFFFFFF7D
:1007FC00000000010000054653443431000008009D
:10080C0001000000000000000000000001020304D1
:10081C00060708090100000000000100E0010101C9
:10082C000100000031F800080000000098010020D1
:10083C001C0D050800000000000000000000000076
:10084C0000000000752E05080000000000000000EC
:10085C00EC05002004000000C80C05080D00000089
:10086C0055890108D405002000000000701B050804
:10087C000D0000002D890108C805002000000000B3
:10088C003C0D05080800000000000000BC0500201D
:10089C00040000002C0D05080D000000E1640108A7
:1008AC00B0050020000000008C17050803000000B4
:1008BC005D8C0108A405002000000000340D050823
:1008CC00030000005D8C010898050020000000006A
:1008DC00DC0B050801000000000000000000000017
:1008EC0000000000000000000E00000000000000EE
:1008FC0000000000000000001C0D050800000000B6
:10090C00000000000000000000000000752E05082B
:10091C000000000000000000EC05002004000000B6
:10092C00600C0508030000002DFA00088C0500205F
:10093C00080000002C0D05080D000000E164010802
:10094C00B0050020000000008C1705080300000013
:10095C005D8C0108A405002000000000340D050882
:10096C00030000005D8C01089805002000000000C9
:10097C00DC0B050801000000000000000000000076
:10098C0000000000000000000E000000000000004D
:10099C000000000000000000440D050800000000ED
:1009AC00000000000000000000000000752E05088B
:1009BC000000000000000000EC0500200400000016
:1009CC00680C0508030000005D8C0108E0050020A0
:1009DC0000000000DC0B0508010000000000000016
:1009EC000000000000000000000000000E000000ED
:1009FC000000000000000000000000000108FFFFE4
:100A0C00010000000000803F0000803FFFFFFFFF5F
:100A1C00563F002088136F1701000000583F00203C
:100A2C0088136F1700000000B40B050800000000CD
:100A3C00000000000000000000000000C40B0508CE
:100A4C0008000000000000001C0200200400000050
:100A5C00D00B050808000000000000001002002068
:100A6C00000000008C170508040000001D1D010883
:100A7C000000000000000000DC0B05080100000075
:100A8C00000000000000000000000000000000005A
:100A9C000E0000000000000000000000000000003C
:100AAC00543F002088136F1701000000689100204C
:100ABC0088136F170000000099F800080000000070
:100ACC00280200202843002001000000BCCC0408B0
:100ADC006A91002001000000C8CC0408609100203D
:100AEC0002000000D0CC040852C40020000000001A
:100AFC000000000050C400200000000000000000B6
:100B0C004EC4002000000000000000004CC4002077
:100B1C0000000000000000004AC40020000000009B
:100B2C000000000048C4002000000000000000008D
:100B3C005C2000200000000000000000533F00205B
:100B4C0002000000DCCC0408180C050800000000B2
:100B5C00000000000000000000000000C40B0508AD
:100B6C000800000000000000AC020020040000009F
:100B7C00D00B05080800000000000000A0020020B7
:100B8C00000000008C1705080400000069F800083C
:100B9C000000000000000000DC0B05080100000054
:100BAC000000000000000000000000000000000039
:100BBC000E0000000000000000000000000000001B
:100BCC00280C0508000000000000000000000000D8
:100BDC0000000000380C05080D000000D588010845
:100BEC00DC02002004000000440C05080D0000008D
:100BFC007D880108D002002004000000500C05087C
:100C0C000D000000A1880108C402002000000000B3
:100C1C005C0C0508030000004DFA0008B802002027
:100C2C0008000000680C0508030000005D8C01083A
:100C3C00E005002000000000DC0B050801000000AE
:100C4C000000000000000000000000000000000098
:100C5C000E0000000000000000000000000000007A
:100C6C00700C0508000000000000000000000000EF
:100C7C0000000000780C050804000000351D010878
:100C8C000000000000000000DC0B05080100000063
:100C9C000000000000000000000000000000000048
:100CAC000E0000000000000000000000000000002A
:100CBC00D00C05080000000000000000000000003F
:100CCC0000000000B83605080D0000000000000010
:100CDC003C03002004000000E00C050808000000A4
:100CEC00000000003003002004000000EC0C05089C
:100CFC000800000000000000240300200400000095
:100D0C00F40C050808000000000000001803002087
:100D1C0004000000FC0C05080800000000000000A6
:100D2C000C03002004000000040D0508080000005E
:100D3C000000000000030020040000000C0D05085A
:100D4C000800000000000000F40200200400000075
:100D5C00140D05080800000000000000E802002047
:100D6C0004000000DC0B050801000000000000007E
:100D7C000000000000000000000000000E00000059
:100D8C0000000000000000000000000081F80008D6
:100D9C0000000000480300200000000000000000DC
:100DAC00C0030020000000000000000060040020D0
:100DBC006691002004000000E8CC04086491002037
:100DCC00E0150C17000000006391002008000000E3
:100DDC00FCFD04086291002005000000FCCC040816
:100DEC000000000000000000B00400202D202D2D7C
:100DFC00202D2D2D2D202D2D2D000000000000006C
:100E0C000000000000000000000000002070002026
:100E1C00702D7200FFFFFFFFD601010000010101E0
:100E2C00000000000000000000000000A81C0020D2
:100E3C0001000000FA0000000100000001000000A9
:100E4C0001010100CF4B002000C80100CE4B002057
:100E5C0000500100CD4B0020005A0100CB4B00206C
:100E6C000200000090CE040818170508201705088A
:100E7C00700C0508000000000000000000000000DD
:100E8C0000000000DC10050804000000911C0108A3
:100E9C000000000000000000DC0B05080100000051
:100EAC000000000000000000000000000000000036
:100EBC000E00000000000000000000000000000018
:100ECC006C17050800000000000000000C06002054
:100EDC0000000000D05F05080D00000000000000BD
:100EEC005C060020000000008417050805000000C7
:100EFC0000000000CC4B00200000000090170508FB
:100F0C000700000000000000540600200000000054
:100F1C00A417050807000000000000004C06002084
:100F2C0000000000B01705080700000000000000DA
:100F3C004406002000000000DC0B05080100000046
:100F4C000000000000000000000000000000000095
:100F5C000E00000000000000000000000000000077
:100F6C00FAC300200100C40900000000F8C30020EF
:100F7C000100C40900000000F6C300200100C409F0
:100F8C0000000000F4C300200100C40900000000B0
:100F9C00F0C300200100C40900000000F2C30020CF
:100FAC000100C40900000000EEC300200100C409C8
:100FBC0000000000ECC300200100C4090000000088
:100FCC00C44900200100C80001000000C2490020F3
:100FDC003200307532000000C1490020055A05006E
:100FEC00BE49002000FF0100C049002001000000A4
:100FFC0068060020BC490020020000008CCC0408CC
:10100C00BD49002000FF0100BF4900200100000085
:10101C0068060020BB490020020000008CCC0408AC
:10102C00B649002080C1803E05000000B449002074
:10103C0080C1803E05000000AE49002080C1803E8A
:10104C0005000000AC49002080C1803E0500000076
:10105C00A749002000FF0100A24900200A3201002C
:10106C00A1490020040000009CCE0408A0490020E7
:10107C0002000000B0CE04080000000000000000D8
:10108C00700600202C9100209CFF2C010000000019
:10109C001E0000200A000000BCCE0408503F0020B7
:1010AC00E0150C17000000002000002008000000D4
:1010BC00FCFD04081F00002005000000FCCC040807
:1010CC00523F002002000000D4CE0408064C002041
:1010DC000100FF7F01000000054C00200200000011
:1010EC00E0CE0408314A002003000000F0CE0408D2
:1010FC00304A002003000000F0CE0408BE4B002054
:10110C000000F40101000000BC4B00200000F401C1
:10111C0001000000BA4B00200000F40101000000A7
:10112C00B84B00200000F40101000000B64B002079
:10113C000000803E01000000B44B00200000803E07
:10114C0001000000E34B002019640100E24B002079
:10115C000200000000CF0408E04B0020E803D00799
:10116C000A000000DE4B0020006401000A000000B1
:10117C00D34B002000640100D24B0020006401001E
:10118C00DA4B0020006401000A000000D94B00205B
:10119C00006401000A000000D84B0020006401002C
:1011AC000A000000DD4B0020006401000A00000072
:1011BC00DC4B0020006401000A000000DB4B002027
:1011CC00006401000A000000D74B002001FF010061
:1011DC000A000000D64B002001FF01000A000000AD
:1011EC00D54B002001FF01000A0000003A4A002004
:1011FC000000F40101000000384A00200000F40156
:10120C0001000000364A00200000F401010000003B
:10121C00344A00200000F40101000000324A002092
:10122C000000F40101000000C5680108896801088C
:10123C00C0060020CA4B002000640100C84B0020EF
:10124C001400E80301000000C64B0020E8033075D1
:10125C000A000000C44B002000C80100C34B002052
:10126C0000C80100C24B002000C80100C14B002087
:10127C00006401000A000000FA4B00200000D007B7
:10128C0001000000F54B002000C80100F44B0020C9
:10129C0000C80100F34B002000C80100F84B0020EF
:1012AC000000D00701000000F24B002000C8010034
:1012BC00F14B002000C80100F04B002000C80100D9
:1012CC00F64B00200000D00701000000EF4B00207F
:1012DC0000C80100EE4B002000C80100ED4B0020BF
:1012EC0000C80100BC170508000000000000000049
:1012FC000000000000000000CC17050809000000E9
:10130C0000000000B407002004000000D4170508FA
:10131C000900000000000000A807002004000000E5
:10132C00B41F050809000000000000009C07002005
:10133C0004000000600F0508090000000000000018
:10134C009007002004000000DC17050809000000CD
:10135C00000000008407002004000000E4170508CA
:10136C0009000000000000007807002004000000C5
:10137C00EC17050809000000000000006C070020B5
:10138C0004000000F417050809000000000000002C
:10139C006007002004000000DC0B050801000000C1
:1013AC000000000000000000000000000000000031
:1013BC000E00000000000000000000000000000013
:1013CC005C1A05080000000000000000000000008E
:1013DC0000000000FC54050807000000000000009D
:1013EC00D8070020000000006C1A05080800000057
:1013FC0000000000CC07002000000000781A05084F
:10140C000800000000000000C007002000000000E1
:10141C00DC0B0508010000000000000000000000CB
:10142C0000000000000000000E00000000000000A2
:10143C000000000000000000801A050800000000F9
:10144C00000000000000000000000000901A0508D9
:10145C000D00000000000000140800200000000037
:10146C00981A05080D000000000000000808002074
:10147C0000000000A01A0508070000000000000092
:10148C000008002000000000A81A05080D0000004C
:10149C0000000000F407002000000000B01A05084E
:1014AC000D00000000000000E80700200000000014
:1014BC00B81A05080700000000000000E007002033
:1014CC0000000000DC0B050801000000000000001B
:1014DC000000000000000000000000000E000000F2
:1014EC00000000000000000000000000C01A050809
:1014FC0000000000000000000000000000000000E0
:10150C00FC5405080C00000000000000C649002037
:10151C0004000000D41A05080C00000000000000B4
:10152C00C849002004000000E41A05080C00000063
:10153C0000000000FE49002004000000F41A050819
:10154C000C00000000000000F24900200400000024
:10155C00081B05080C00000000000000CA49002010
:10156C0004000000141B05080C0000000000000023
:10157C00CC490020040000001C1B05080C000000D6
:10158C0000000000CE49002004000000301B0508BC
:10159C000C00000000000000D049002004000000F6
:1015AC00381B05080C00000000000000D249002088
:1015BC0004000000401B05080C00000000000000A7
:1015CC00104A002004000000581B05080C00000005
:1015DC0000000000D449002004000000641B050832
:1015EC000C00000000000000D649002004000000A0
:1015FC00981705080C00000000000000D8490020D6
:10160C00040000006C1B05080C000000000000002A
:10161C00DA49002004000000781B05080C000000CB
:10162C0000000000DC49002004000000841B0508B9
:10163C000C00000000000000DE4900200400000047
:10164C00901B05080C00000000000000E049002081
:10165C00040000009C1B05080C00000000000000AA
:10166C00E249002004000000A81B05080C00000043
:10167C0000000000F649002004000000B01B050823
:10168C000C00000000000000F449002004000000E1
:10169C00B81B05080C00000000000000024A0020E6
:1016AC0004000000C41B05080C0000000000000032
:1016BC00044A002004000000D01B05080C000000A8
:1016CC0000000000244A002004000000DC1B050878
:1016DC000C000000000000000A4A0020040000007A
:1016EC00A41805080C00000000000000E4490020CC
:1016FC00040000002C0D05080C0000000000000088
:10170C00EC49002004000000E81B05080C00000058
:10171C0000000000E649002004000000F41B05084E
:10172C000C00000000000000E8490020040000004C
:10173C00001C05080C00000000000000EA49002015
:10174C0004000000081C05080C000000000000004C
:10175C00EE490020040000008C0D05080C00000070
:10176C0000000000F849002004000000141C0508CB
:10177C000C00000000000000F049002004000000F4
:10178C00201C05080C00000000000000004A00208E
:10179C00040000002C1C05080C00000000000000D8
:1017AC00FA49002004000000341C05080C0000005D
:1017BC0000000000FC490020040000003C1C05084F
:1017CC000C00000000000000064A0020040000008D
:1017DC00441C05080C00000000000000084A002012
:1017EC00040000004C1C05080C0000000000000068
:1017FC001A4A002004000000541C05080C000000CC
:10180C0000000000204A002004000000DC0B05084A
:10181C0001000000000000000000000000000000BB
:10182C00000000000E00000000000000000000009E
:10183C0000000000601C0508000000000000000013
:10184C0000000000000000006C1C05080D000000EA
:10185C00000000006C08002000000000741C05084B
:10186C000D000000000000006008002000000000D7
:10187C007C1C050807000000000000005808002030
:10188C0000000000881C0508070000000000000094
:10189C005008002000000000941C050809000000FE
:1018AC00000000004408002000000000A01C0508F7
:1018BC0009000000000000003808002000000000B3
:1018CC00AC1C050809000000000000002C080020DA
:1018DC0000000000BC1C050809000000000000000E
:1018EC002008002000000000DC0B050801000000AF
:1018FC0000000000000000000000000000000000DC
:10190C000E000000000000000000000000000000BD
:10191C00D01C0508000000000000000000000000C2
:10192C0000000000E01C050805000000000000009D
:10193C002F4A002000000000DC0B0508010000000D
:10194C00000000000000000000000000000000008B
:10195C000E0000000000000000000000000000006D
:10196C00E81C05080000000000000000000000005A
:10197C0000000000980B05080000000000000000AB
:10198C002020002004000000F41C05080D000000BD
:10199C00F51C0108C008002000000000C80C050858
:1019AC000D00000015F80008B4080020000000002D
:1019BC00701B05080D000000F9F70008A8080020AE
:1019CC00000000003C0D05080800000000000000AD
:1019DC009C080020040000002C0D05080D000000E0
:1019EC0041F700089008002000000000F81C0508D2
:1019FC000900000000000000840800200400000022
:101A0C008C170508030000005D8C01087808002085
:101A1C0000000000DC0B05080100000000000000C5
:101A2C000000000000000000000000000E0000009C
:101A3C00000000000000000000000000001D050870
:101A4C00000000000000000000000000000000008A
:101A5C00101D05080D00000000000000D808002033
:101A6C0000000000181D05080A000000000000001E
:101A7C002550002000000000241D05080A0000006D
:101A8C00000000002D500020000000002C1D050857
:101A9C000A0000000000000035500020000000008B
:101AAC00341D05080800000000000000CC080020D0
:101ABC0000000000DC0B0508010000000000000025
:101ACC000000000000000000000000000E000000FC
:101ADC000000000000000000000000003C1D050894
:101AEC0000000000000000000000000000000000EA
:101AFC00501D05080D00000000000000F00800203B
:101B0C0000000000601D050804000000258A010883
:101B1C000000000000000000681D05080D0000001A
:101B2C0000000000E4080020000000007C1D0508F7
:101B3C0004000000018A0108000000000000000001
:101B4C00DC0B050801000000000000000000000094
:101B5C0000000000000000000E000000000000006B
:101B6C000000000000000000841D050800000000BB
:101B7C00000000000000000000000000981D050897
:101B8C0008000000000000003809002000000000E0
:101B9C00A41D050808000000000000002C0900200E
:101BAC0000000000B01D0508080000000000000047
:101BBC002009002000000000BC1D050808000000E2
:101BCC00000000001409002000000000C81D0508DA
:101BDC0008000000000000000809002000000000C0
:101BEC00D41D05080800000000000000FC080020BF
:101BFC0000000000DC0B05080100000000000000E4
:101C0C000000000000000000000000000E000000BA
:101C1C00000000000000000000000000E01D0508AE
:101C2C0000000000000000000F0600200000000073
:101C3C00EC1D05080B00000000000000E00900206E
:101C4C0000000000F81D05080B000000000000005B
:101C5C00D409002000000000041E05080B00000041
:101C6C0000000000C809002000000000101E05083C
:101C7C000B00000000000000BC0900200000000068
:101C8C001C1E05080B00000000000000B00900201D
:101C9C0000000000281E05080B00000000000000DA
:101CAC00A409002000000000341E05080B000000F1
:101CBC00000000009809002000000000401E0508EC
:101CCC000B000000000000008C0900200000000048
:101CDC004C1E05080B0000000000000080090020CD
:101CEC0000000000581E050807000000000000005E
:101CFC007809002000000000601E050807000000A5
:101D0C000000000070090020000000006C1E050897
:101D1C000B0000000000000064090020000000001F
:101D2C00781E05080800000000000000580900207B
:101D3C0000000000841E05080D00000000000000DB
:101D4C004C09002000000000941E0508070000004C
:101D5C00000000004409002000000000DC0B050816
:101D6C000100000000000000000000000000000066
:101D7C00000000000E000000000000000000000049
:101D8C0000000000A01E050800000000000000007C
:101D9C000000000000000000B41E05080800000050
:101DAC00000000001C0A002000000000C01E0508F6
:101DBC000800000000000000100A002000000000D5
:101DCC00CC1E05080800000000000000040A0020DA
:101DDC0000000000D81E05080800000000000000EC
:101DEC00F809002000000000E41E050808000000AF
:101DFC0000000000EC09002000000000DC0B0508CE
:101E0C0001000000000000000000000000000000C5
:101E1C00000000000E0000000000000000000000A8
:101E2C0000000000EC1E050800000000000000008F
:101E3C000C06002000000000FC1E05080B00000032
:101E4C00000000006C0A002000000000081F0508BC
:101E5C000700000000000000640A002000000000E1
:101E6C00141F050807000000000000005C0A002099
:101E7C0000000000201F0508070000000000000003
:101E8C00540A0020000000002C1F05080800000068
:101E9C0000000000480A002000000000341F050864
:101EAC0008000000000000003C0A002000000000B8
:101EBC003C1F05080700000000000000340A002049
:101ECC0000000000481F0508030000005D8C01089D
:101EDC00280A002000000000DC0B050801000000AF
:101EEC0000000000000000000000000000000000E6
:101EFC000E000000000000000000000000000000C8
:101F0C00581F050800000000000000000C0600200F
:101F1C0000000000641F050807000000000000001E
:101F2C00DC0A0020000000006C1F05080700000000
:101F3C0000000000D40A002000000000741F0508F7
:101F4C000700000000000000CC0A00200000000088
:101F5C007C1F05080800000000000000C00A0020DB
:101F6C0000000000280F050807000000000000001A
:101F7C00B80A002000000000300F05080700000020
:101F8C0000000000B00A002000000000380F050817
:101F9C000700000000000000A80A0020000000005C
:101FAC00E40F050808000000000000009C0A002057
:101FBC0000000000841F050807000000000000005E
:101FCC00940A0020000000008C1F05080700000088
:101FDC00000000008C0A002000000000941F05087F
:101FEC000700000000000000840A00200000000030
:101FFC009C1F05080800000000000000780A002063
:10200C0000000000DC0B05080100000000000000CF
:10201C000000000000000000000000000E000000A6
:10202C0000000000000000000000000000000000A4
:10203C00F5660108E40A00202D4A00202E0000005D
:10204C000CCF04082C4A002000C801002A4A0020AA
:10205C00E803D0070100000046554C4C5350454551
:10206C004446343131000000BA490020000301001D
:10207C00B949002000030100416601081D660108F2
:10208C00C00B0020E16501089D650108380C00209B
:10209C007D66010865660108EC0C002035650108B9
:1020AC0005650108341000200B670108D18901086F
:1020BC001011002081F700080000000060110020C2
:1020CC007D890108196A01083C120020316701085A
:1020DC0000000000DC120020F1670108B567010860
:1020EC006813002001690108496901081C140020CB
:1020FC00D04B0020010601007967010845670108F3
:10210C00841500202D680108498A01082416002036
:10211C007D690108A58A010800170020C04B00202A
:10212C0001030100A41F05080000000000000000CE
:10213C000000000000000000B01F050808000000AF
:10214C00000000004C18002000000000B81F05081B
:10215C0007000000000000004418002000000000F0
:10216C00C81F05080D0000000000000038180020F2
:10217C0000000000D41F0508030000005D8C01085E
:10218C002C18002000000000DC0B050801000000EA
:10219C000000000000000000000000000000000033
:1021AC000E00000000000000000000000000000015
:1021BC00DC1F05080000000000000000000000000B
:1021CC0000000000EC1F05080A00000000000000E1
:1021DC00F41F050800000000FC1F05080A000000A1
:1021EC000000000014110508000000000420050880
:1021FC000A00000000000000FC4B00200000000062
:10220C000C2005080A0000000000000058180020EF
:10221C0000000000DC0B05080100000000000000BD
:10222C000000000000000000000000000E00000094
:10223C000000000000000000000000001420050851
:10224C000000000000000000000000000000000082
:10225C0020200508030000005D8C01089018002068
:10226C00000000002C200508030000005D8C010814
:10227C008418002000000000342005080300000032
:10228C005D8C010878180020000000003C20050837
:10229C000500000000000000B8490020000000000C
:1022AC004420050807000000000000007018002002
:1022BC00000000005020050807000000000000008E
:1022CC006818002000000000DC0B0508010000006D
:1022DC0000000000000000000000000000000000F2
:1022EC000E000000000000000000000000000000D4
:1022FC005C20050800000000000000000000000049
:10230C000000000070200508030000005D8C01082F
:10231C00C0180020000000007C200508030000000D
:10232C005D8C0108240000200000000084200508BA
:10233C00030000005D8C0108B418002000000000B0
:10234C008C200508030000005D8C0108A8180020F3
:10235C00000000002C0D0508030000005D8C010836
:10236C009C18002000000000DC0B05080100000098
:10237C000000000000000000000000000000000051
:10238C000E00000000000000000000000000000033
:10239C00982005080000000000000000000000006C
:1023AC0000000000A820050807000000018B0108B0
:1023BC001C19002000000000041C0508030000008C
:1023CC005D8C01081019002000000000B4200508E5
:1023DC00030000005D8C01080419002000000000BF
:1023EC00BC200508030000005D8C0108F8180020D3
:1023FC0000000000C420050807000000E58A010861
:10240C00F018002000000000A00F050803000000D9
:10241C005D8C0108E418002000000000D0200508A5
:10242C00030000005D8C0108D8180020000000009B
:10243C00DC200508030000005D8C0108CC1800208E
:10244C0000000000DC0B050801000000000000008B
:10245C000000000000000000000000000E00000062
:10246C00000000000000000000000000C56601082C
:10247C009566010824190020F96901080000000084
:10248C00B019002081650108656501083C1A00201F
:10249C000000000000000000F01A0020D1690108C3
:1024AC001D8B0108901B0020E8200508000000008F
:1024BC0000000000000000000000000000100508F3
:1024CC00030000005D8C01089C1C00200000000033
:1024DC00F4200508030000005D8C0108901C00200E
:1024EC000000000078100508030000005D8C010856
:1024FC00841C0020000000000021050803000000DF
:10250C005D8C0108781C0020000000000C210508DF
:10251C00030000005D8C01086C1C00200000000012
:10252C001421050802000000FD080208000000004C
:10253C00000000001C21050802000000FD08020834
:10254C000100000000000000282105080200000026
:10255C00FD0802080200000000000000000000005E
:10256C000E00000000000000000000000000000051
:10257C00685E0C0001000000A00F0000B80B00000A
:10258C000102FFFF01000000010000000000803F7D
:10259C00000000000000000000000000FF00000030
:1025AC005CD604080508040000000000FCCC0408FC
:1025BC00FCFD0408E8CC040800000000000000004A
:1025CC0088D6040805080A0000000000FCCC0408AA
:1025DC00FCFD0408BCCE0408000000000000000054
:1025EC00FFFF00000000803F000000000000000022
:1025FC00000000000000803F000000000000000010
:10260C0000000000000000000000000000000000BE
:10261C0000000000000000000000000001000000AD
:10262C000000803F000000000000000000000000DF
:10263C00FFFFFFFFFFFFFFFFFFFFFFFF0000803FDB
:10264C00000000003C850020080000000000000095
:10265C002C85002008000000A10B0408D3090408F5
:10266C005923040800000000FD0604083920040862
:10267C00110B0408BD1F040800000000000000003E
:10268C00BD060408130B040895090408A1220408CC
:10269C0000000000D5060408BF1F0408E50A040862
:1026AC002B1F04080000000000000000C9060408ED
:1026BC000403090412010002EF02014083045632A4
:1026CC00000201020301000012010002020200409C
:1026DC008304405700020102030100000902640058
:1026EC00030100C0320904000001030000000921AD
:1026FC00110100012226000705830308000A080BBC
:10270C00010202020100090401000102020100059C
:10271C0024001001052401000204240202052406F1
:10272C000102070582030800FF09040200020A00E7
:10273C00000007050102400000070581024000006F
:10274C0009024300020100C0320904000001020228
:10275C0001000524001001052401000104240202DB
:10276C000524060001070582030800FF0904010087
:10277C00020A000000070501024000000705810263
:10278C0040000000FF00000000FFFF000000000000
:10279C00AA5505010000010005010905A101A100D0
:1027AC000501093009310932093309350934094069
:1027BC0009381581257F750895088102C0C0000075
:1027CC0009022200010100E03209040000010301AA
:1027DC0002000921110100012226000705830308CC
:1027EC00000A0000000000000102030401020304BF
:1027FC0006070809472104084B2004087B2304081A
:10280C00330704084B0A0408430704085F0704084D
:10281C000D070408FF06040800000000000000007B
:10282C002D202D2D202D2D2D2D202D2D2D2D00004D
:10283C00000000000000000000000000000000AAE2
:10284C00550B010000AA5507010000AA550902000A
:10285C000000AA5503009F0001000000C0120000F8
:10286C00FF1FFF1FAC93002000000000D09300203E
:10287C000000000008000000850604088306040818
:10288C00810604087B060408790604087F06040800
:10289C007D06040895060408870604082913040815
:1028AC003D1304081513040801130408EB12040863
:1028BC0001000000006002401060024000000000B7
:1028CC0000000000000B00000000000000000000F1
:1028DC00000000000060024028600240010000007F
:1028EC0000000000060C00000000000000000000CA
:1028FC000000000000600240406002400200000046
:10290C0000000000100D000000000000000000009E
:10291C00000000000060024058600240030000000C
:10292C0000000000160E0000000000000000000077
:10293C0000000000006002407060024004000000D3
:10294C0000000000200F000000000000000000004C
:10295C00000000000060024088600240050000009A
:10296C000000000026100000000000000000000025
:10297C000000000000600240A06002400600000061
:10298C0000000000301100000000000000000000FA
:10299C000000000000600240B86002400700000028
:1029AC0000000000362F00000000000000000000B6
:1029BC0000000000006402401064024000000000AF
:1029CC0000000000003800000000000000000000C3
:1029DC000000000000640240286402400100000076
:1029EC00000000000639000000000000000000009C
:1029FC00000000000064024040640240020000003D
:102A0C0000000000103A0000000000000000000070
:102A1C000000000000640240586402400300000003
:102A2C0000000000163B0000000000000000000049
:102A3C0000000000006402407064024004000000CA
:102A4C0000000000203C000000000000000000001E
:102A5C000000000000640240886402400500000091
:102A6C0000000000264400000000000000000000F0
:102A7C000000000000640240A06402400600000058
:102A8C0000000000304500000000000000000000C5
:102A9C000000000000640240B8640240070000001F
:102AAC00000000003646000000000000000000009E
:102ABC0000000000405505086010050800000000EB
:102ACC0029BC0308A08601000400000000000000DF
:102ADC0000000000000000000000000000000000EA
:102AEC000000000000000000405505084461050886
:102AFC00000000006D0C0208E80300000400000058
:102B0C0000000000000000000000000000000000B9
:102B1C00000000000000000000000000041C05087C
:102B2C000033050800000000919E02087D000000A3
:102B3C000600000000000000000000000000000083
:102B4C000000000000000000000000000000000079
:102B5C00B05405080000000000000000592E0208C7
:102B6C00E80300000300000000000000000000006B
:102B7C000000000000000000000000000000000049
:102B8C00000000004C61050800000000000000007F
:102B9C00951C030810270000030000000000000033
:102BAC000000000000000000000000000000000019
:102BBC000000000000000000780D05080000000077
:102BCC0005830108397102085F76000005000000DA
:102BDC0000000000000000000000000000000000E9
:102BEC00000000000000000000000000FC5605087A
:102BFC000000000000000000918102081027000076
:102C0C0001000000000000000000000000000000B7
:102C1C0000000000000000000000000000000000A8
:102C2C00586105080000000000000000710C02084B
:102C3C00E803000005000000000000000000000098
:102C4C000000000000000000000000000000000078
:102C5C000000000064610508000000000000000096
:102C6C0041C20308204E00000300000000000000D9
:102C7C000000000000000000000000000000000048
:102C8C000000000000000000746105080000000056
:102C9C000000000065BC0308204E0000030000008B
:102CAC000000000000000000000000000000000018
:102CBC000000000000000000000000008461050816
:102CCC00000000000000000001120208400D03008B
:102CDC0003000000000000000000000000000000E5
:102CEC0000000000000000000000000000000000D8
:102CFC00005605080000000000000000F5CD030898
:102D0C00102700000100000000000000000000007F
:102D1C0000000000000000000000000000000000A7
:102D2C0000000000740D0508000000000000000009
:102D3C00053101081027000003000000000000000E
:102D4C000000000000000000000000000000000077
:102D5C000000000000000000B45405080000000052
:102D6C00000000002D11020850C3000001000000FB
:102D7C000000000000000000000000000000000047
:102D8C00000000000000000000000000A41805086E
:102D9C000000000000000000590E0208A8610000AD
:102DAC000100000000000000000000000000000016
:102DBC000000000000000000000000000000000007
:102DCC00946105080000000000000000594901084A
:102DDC00A0860100010000000000000000000000BF
:102DEC0000000000000000000000000000000000D7
:102DFC00000000000457050800000000000000005F
:102E0C00493A0208A00F0000010000000000000079
:102E1C0000000000000000000000000000000000A6
:102E2C000000000000000000A06105080000000088
:102E3C00000000009DFC00081027000001000000AD
:102E4C000000000000000000000000000000000076
:102E5C0000000000000000000000000078100508D1
:102E6C000000000000000000755A01081A41000023
:102E7C000100000000000000000000000000000045
:102E8C000000000000000000000000000000000036
:102E9C006418050800000000000000004D0E040836
:102EAC0010270000010000000000000000000000DE
:102EBC000000000000000000000000000000000006
:102ECC000000000074100508000000000000000065
:102EDC00F99901081A4100000100000000000000EF
:102EEC0000000000000000000000000000000000D6
:102EFC000000000000000000AC61050800000000AC
:102F0C0000000000893D0408400D03000000000093
:102F1C0000000000000000000000000000000000A5
:102F2C00000000000000000000000000B461050873
:102F3C000000000000000000290C0208400D0300F6
:102F4C000000000000000000000000000000000075
:102F5C000000000000000000000000000000000065
:102F6C00BC61050800000000000000002D3B0108BA
:102F7C0050C300000300000000000000000000002F
:102F8C000000000000000000000000000000000035
:102F9C0000000000C86105080000000000000000EF
:102FAC000DC2030840420F000000000000000000AA
:102FBC000000000000000000000000000000000005
:102FCC000000000000000000D461050800000000B3
:102FDC000000000031BF030850C3000000000000D7
:102FEC0000000000000000000000000000000000D5
:102FFC000000000000000000000000000000803F06
:1080000003685A1C02601970704700BF2DE9F047E1
:10801000089C2578002B804689460CBF4FF0200A2B
:108020004FF0300A661C25B3002A26DD334601E0F6
:10803000024698B113F8011B501E0029F8D1971E73
:1080400060B13D46013D51464046C8476B1C002B80
:10805000F8DC257827EAE770013045B1041B294692
:108060004046C847301916F8015B002DF7D1BDE82E
:10807000F087002A03DC2846F9E70020EEE7571EC8
:10808000DFE700BF2DE9F04714461D4606464FF4D2
:108090007A7200232046294642F056FC4D4BDFF809
:1080A00048814D4A4D4F034488FB03101844D917AB
:1080B00082FB032CC1EB601088FB002887FB0327A1
:1080C0009C44474AC1EBEC2CC0EB001E82FB0C2900
:1080D000A3EB8E0E1F44434A86F806E0C1EB274708
:1080E0004FEAEC7E08EB000ACEEBA90E82FB07827A
:1080F0004FEAE0780EEB4E0EC8EB6A18ACEBCE0CF4
:10810000C8EB0818DFF8E4E086F804C0A0EB8800AC
:1081100070718EFB0303F817C0EBE21240F2B5500A
:1081200000FB1272C1EBE353B2F5896F4FEA83078C
:108130003CDA40F2DA239A4242DCB2F5B77FB4BFB0
:108140004FF0000E4FF0010E4FEA4E09DFF8A0800D
:1081500009EB0E0308EBC3031FFA8EFCD88A09EB68
:108160000E0108EBC10116310B2301E031F8020DBD
:10817000904218DD013BF9D1CE44012338F83E008E
:10818000B37007F5FA670132121ABC44F270A6F810
:1081900000C0204629464FF47A72002342F0D4FBF7
:1081A0003281BDE8F0870133DBB2E9E74FF0030C21
:1081B000E64640F29650DFF838804FF00609CEE7E9
:1081C0004FF0020CDFF82880E64640F229404FF0DD
:1081D0000409C4E780BC92C7C5B3A29107452EC26B
:1081E000ABAAAA2A73B06D1689888888792D0311E5
:1081F00078C404080028F0B403DA2D230B70404241
:108200000131092804464FF0010307DD03EB830326
:108210005B00B0FBF3F2092AF8D883B10F48A0FB4A
:108220000326B4FBF3F2092A02F1570C02F13007DE
:1082300009DD03FB1244F30801F801CBEFD1002361
:108240000B70F0BC704703FB1244F30801F8017B8C
:10825000E5D100230B70F0BC704700BFCDCCCCCC77
:10826000884270B44FF0010442D301FB04F4B0FB28
:10827000F4F58D42F9D2ECB142BB092D04FB150097
:1082800005F1570605F130020EDDB4FBF1F403F8F9
:10829000016B7CB1B0FBF4F5092D04FB150005F171
:1082A000570605F13002F0DCB4FBF1F403F8012BC2
:1082B000002CEFD100221A7070BC704703F8016BDC
:1082C000B4FBF1F4002CF5D0B0FBF4F5092D04FB60
:1082D000150005F1370605F13002EFDCB4FBF1F4CF
:1082E00003F8012B002CEFD100221A7070BC7047EC
:1082F0000546002AEAD1C0E790ED057A90ED004AE4
:10830000D0ED066AD0ED014AD0ED047A90ED035A23
:10831000D0ED025AA4EE007AB0EE406AB0EE470A01
:10832000B0EE667AA4EE867A67EEC07AA5EE407A61
:10833000E5EE867A80ED057AC0ED067A704700BFDB
:10834000D0ED057A90ED013AD0ED003AD0ED064A35
:1083500090ED024A90ED077A90ED035A90ED086A8D
:10836000D0ED045AC0ED067AF0EE406A27EE830A9B
:10837000C0ED056AA3EEA60A80ED087AA4EE240AF1
:10838000A5EE470AA5EEC60A80ED070A704700BFB2
:10839000D0ED007A90ED017A30EE670AE7EE007AD0
:1083A000B0EE670AC0ED007A704700BF704700BFAB
:1083B00006224FF47A7302704360704730B4002293
:1083C0000123142511240221C57084710270C27228
:1083D0008273C273417041728370C371037283727E
:1083E00030BC704730B41523162517242D212E22BA
:1083F00003702F2345708470C1700271437130BCCB
:10840000704700BF10B42C21012402220023047005
:1084100041708270C3705DF8044B704701220023E5
:1084200010B4212120244470417102720270027143
:1084300043818381C3815DF8044B70476D4B2DE907
:10844000F04F1C686C4BB3F80AE0B3F804809A89CB
:108450004FEA0E2AB4EB0A044FEA1E6B4FF00005F8
:1084600087B065EB0B05CDE900450746009C1889F0
:10847000019EA0FB044500FB0655E00940EA45606B
:108480004FEA08448C46E9114FEA184510EB0408FE
:10849000D888009C41EB0509CDE90489A0FB04457F
:1084A000B3F8028000FB0655200A40EA05604FEA57
:1084B000C83429124FEA584510EB040841EB05096E
:1084C0000099A2FB010102FB06114FEAD05A4AEAC9
:1084D000412A1AF5FA634FEAE15B4BF10004B3F568
:1084E000FA6FCDE9023474F10003424E64DA0524D8
:1084F000AAFB040104FB0B1100FB0BF40AFB014473
:10850000DDE90423A0FB0A0121444D104FEA3004A9
:10851000121B4FEA900463EB050344EA8174B8EB45
:108520000408CDE90423DDE9023434484FEAA1050B
:1085300069EB05094FF0FF31834274EB010326DA42
:1085400040F6AC501AEB00024FF000014BEB010378
:1085500002FB03F1A2FB022303EB4103D400DD0085
:10856000101B45EA527563EB0501DDE9044524184B
:108570004D41CDE904450B24A2FB040104FB03118A
:1085800049104FEA3000B8EB000869EB0109DDE95A
:1085900000325343009ADDE90201A2FB02AB0BEB70
:1085A000430B4FEADA7242EA4B02801A4FEAEB734E
:1085B00061EB0301CDE9020197B17168A1FB0823CA
:1085C00001FB0933540D5D1544EAC324DDE904239E
:1085D000A21A65EB03031D46D30B43EA45433B60F8
:1085E000BCF1000F02D0029BCCF8003007B0BDE810
:1085F000F08F00BF002800206861002024FAFFFFF0
:108600002DE9F04FDFF8DCC1754CDCF8085022880A
:10861000B4F90AA0C2EB25135200C2EBE502B4F98B
:1086200002505B436A43B4F904501B135D43AD131E
:1086300005EBE225B5F5FA324FEAE57B85B04BF163
:10864000FF33CDE90023DDE900325343009AA561F1
:10865000A2FB0289CDE90201B4F908200199009832
:1086600009EB43095143D31700FB0311A2FB00237D
:108670000B444FEAEA7B0AFB09F11F0308FB0B13CB
:10868000AAFB080119444FEA102A4AEA016A1603B4
:108690004FEA212B47EA12571AEB0602E6884BEB0A
:1086A000070312F1000A43F5004BAAFB060106FB83
:1086B0000B114A10CB1752EA030100F08E80B4F977
:1086C0001060009806FB09F1F71708FB0711A6FBDD
:1086D00008673944B4F90E808B4601994FEAE8796E
:1086E00008FB01F100FB0911A8FB00898944DCF8B3
:1086F0000C104FEA4947C1F5801C47EAD837B2460B
:108700004FEA4846B4F90C801AEB060A66464BEB72
:10871000070BF7174FEAC806019600260096F907DF
:10872000DDE900674FEACC7016EB0A0647EB0B0752
:1087300041EA5C01801B61EB070140F6354C89463C
:10874000A0FB0C010CFB091142F0FEF8B4F9162055
:10875000B4F914A04E13470B47EAC14702FB06FCCD
:10876000D31707FB03CCA2FB07236344564307FB45
:108770000366A2FB07233344560E46EAC31632189B
:108780004FEA636747EB010380460AFB01F14FEABA
:10879000EA7B08FB0B17AAFB08013944C60C46EA22
:1087A000413612EB06084FEAE147B4F9122043EBD9
:1087B00007094FEA182141EA096113010B44029AA3
:1087C0000AB11B0A1360039B23B105EB85058035B5
:1087D0002D121D6005B0BDE8F08F0023EFE700BF4C
:1087E0007C61002000280020704770472DE9F0418F
:1087F000334B344E1A8A7489B6F91450B6F9048092
:10880000B6F90E70B6F920C05B69121B3489544367
:10881000E213B6F912401544E40294FBF5F4B6F9FC
:1088200002501444A4F57A6E0EFB0EF20EFB05F511
:108830000EFB08FEB6F90C80F4611213574302FBDD
:1088400008F2121402EB6E32ED1205EBE72702324A
:10885000B6F90050B6F806E0921002F5004207EBB8
:1088600085070EFB02F207FA0CF74FEAD23E0237F9
:108870004CF25032A3EBA70742FA0CF37B4355BFEF
:108880005B00B3FBFEF3B3FBFEF35B0078B11A129F
:1088900002FB02F540F6DE326A430B4D12145D43D3
:1088A00002EB254202F6CF6203EB2213036021B1F3
:1088B0000A235C43083424110C60BDE8F08100BF3A
:1088C000002800204461002043E3FFFF4FF40063D1
:1088D000038370474FF4006303837047012380F8DC
:1088E000503070474FF4006303837047F0B4037C4B
:1088F000456902681F2B37D9203B202154689940D5
:108900000C4223D010249C40D160D4605168D940DF
:10891000CE074ED4EFF31183502282F31288EA6B14
:108920001168C90709D45468002C52D1D5E90961EE
:108930008E4243D1012285F86020DBB283F3118897
:10894000037C02681F2B194614D9203B082150686C
:108950009940084200D0D1600421506801FA03F325
:10896000184223D1F0BC7047202416689C40264250
:108970000FD11946082310688B40184200D093602D
:108980000423106803FA01F10842EBD09160F0BCB7
:10899000704710219940946091601168D940CC07CC
:1089A000B8D5012101FA03F39360B3E7D360F0BCBB
:1089B0007047012101FA03F3D360ABE7AF690F44BD
:1089C000D7600ED82E69711A5160AC62002185F80B
:1089D0006010116841F00101DBB2116083F311886E
:1089E000AEE7711A5160AE62F0E700BF70B4037C6D
:1089F00001681F2B26D9A3F1200520224C68AA402C
:108A0000224214BF01220022D2B142691B481C4CF1
:108A100002EB420200EB4212257854682068CDB97F
:108A2000E56856892C6824F001042C6082891F2B8C
:108A300022EA060282811AD8202202FA03F38B600E
:108A400070BC704720220C689A40224214BF012259
:108A50000022D9E7A469226822F0010222608289FB
:108A600022F480721204120C1F2B8281E4D9A3F12C
:108A7000200220239340CB6070BC7047CCAB002019
:108A8000C8AB002070B59D4C2368002B40F00581D9
:108A90009B4B1A78002A68D09A4B19789A4B002978
:108AA00064D11868B3F82C5141628489012A44EAE0
:108AB00005048481A3F82C1157D0D3F83001B3F802
:108AC0005C5241628489022A44EA05048481A3F845
:108AD0005C124AD0D3F86002B3F88C5341628489A7
:108AE000032A44EA05048481A3F88C133DD0D3F80B
:108AF0009003B3F8BC5441628489042A44EA050413
:108B00008481A3F8BC1430D0D3F8C004B3F8EC557A
:108B100041628489052A44EA05048481A3F8EC159E
:108B200023D0D3F8F005B3F81C5741628489062A94
:108B300044EA05048481A3F81C1716D0D3F8200753
:108B4000B3F84C5841628489072A44EA05048481B9
:108B5000A3F84C1809D0D3F85028B3F87C495162D7
:108B6000908920439081A3F87C1970BD5C681989B5
:108B700061602568186845F0010540F20D312560F7
:108B8000A0F848108489012A44F480748481ECD0D0
:108B9000D3F83441B3F83851D3F830016560256813
:108BA00045F001052560A0F848108489022A44F4A4
:108BB00080748481D9D0D3F86442B3F86852D3F872
:108BC00060026560256845F001052560A0F8481041
:108BD0008489032A44F480748481C6D0D3F89443F2
:108BE000B3F89853D3F890036560256845F0010504
:108BF0002560A0F848108489042A44F48074848194
:108C0000B3D0D3F8C444B3F8C854D3F8C0046560F3
:108C1000256845F001052560A0F848108489052ADB
:108C200044F480748481A0D0D3F8F445B3F8F855A7
:108C3000D3F8F0056560256845F001052560A0F8CA
:108C400048108489062A44F4807484818DD0D3F836
:108C50002447B3F82857D3F820076560256845F006
:108C600001052560A0F848108489072A44F480741F
:108C700084813FF47AAFD3F85428B3F85808D3F876
:108C800050385060106840F001001060A3F84810A0
:108C90009A8942F480729A8170BD05461AF06AFC86
:108CA000217AA9B16DB1194A002316890133002E2A
:108CB00018BF0021AB4202F16002F6D100293FF457
:108CC000E7AE00F51C501030002320602372DFE671
:108CD0002368C31A002BFFF648AF637A3BB1013B10
:108CE000DBB263722BB100F57A702060D0E62360AE
:108CF000CEE6636803442360CAE600BF306B002001
:108D0000CCAE0020C8AB0020D0AE0020CCAB002001
:108D100010B5027C01681F2A4FF020030ED94C6861
:108D2000203A93401C4208D00B4A4068002414703B
:108D3000026822F001020260CB6010BD0C68934013
:108D40001C42FAD0044A406800241470026822F0E1
:108D5000010202608B60F0E78C3200202DE9F041C7
:108D6000C40023189B00B749CA585268958AADB20F
:108D7000EFB2FE070B4461D4BE0737D5BFF35F8F58
:108D80001D7EEDB2012D00F0BB80AF4E138BBFF303
:108D90005F8F231801EB83031D7E022D00F0CE8030
:108DA000231801EB83031D7E032D05D19B7E1BB190
:108DB000737E002B40F01A81938896F918C043F413
:108DC00080639380231801EB83031B7E013363458B
:108DD0000AD1B37E00257576002B40F08A802044AE
:108DE00001EB800000234375BDE8F081964E17F03B
:108DF000040F96F918C04DD117F0400700F0B2806B
:108E0000178A1D6AFFB205F80C705FFA8CF56F1CAB
:108E100093F818E07BB2DF1CBE4533769C4600F029
:108E20000981271801EB87073F7EBB42CAD105F1B4
:108E3000020C4FFA8CFC86F818C0C3E71588824EE6
:108E400025F400652D042D0C1580158845F48065EA
:108E500015809D7E00273776002D3DD0757E002D34
:108E600037D0231801EB830301251B7E7576022B77
:108E700003D1138843F400631380231801EB8303A9
:108E80009B7D43F001031382204401EB8000037EAD
:108E9000BDE8F0819F7E757E4FF0010E86F81AE0E6
:108EA000002F5CD0002D78D1231801EB83035B7E6B
:108EB000002B00F0A48013880CF1010C4FFA8CFCFD
:108EC00043F4007386F818C013801388DF05FCD4C0
:108ED00078E7DB7DFF2BC4D0231801EB83039D7D56
:108EE00005F0FE051582DB7DFF2BCDD0FF23337609
:108EF000CAE7938823F440731B041B0C93806EE72E
:108F00009B7E514E002B3FF441AF737E002B3FF40C
:108F10003DAF138823F480631B041B0C1380BFF345
:108F20005F8F138B1388B57643F400731380938897
:108F300096F918C043F48063938043E79B7E002B2F
:108F40003FF42EAF737E002B3FF42AAF138896F9BF
:108F500018C023F480631B041B0C138016E0002D43
:108F6000A2D0A8E72D067FF52DAFBCF1FF3F6DD055
:108F7000DD6915F80C5015820CF1010C1D7E4FFABD
:108F80008CF39D429C4633767FF41CAF938823F488
:108F900080631B041B0C938014E71F7ED3F8208092
:108FA0005FFA8CF5AE44022F4FFA8EFE17882DD94A
:108FB00027F480673F043F0C1780178AFFB208F838
:108FC0000C701788D3F820C047F400731380138AFD
:108FD000DBB20CF80E30938805F1020C4FFA8CFCD2
:108FE00043F4806386F818C093806EE7938896F9FF
:108FF00018C023F480631B041B0C9380E2E61388E3
:10900000012543F48073138075765EE747F400779B
:109010001780178AFFB208F80C70178AD3F82080DF
:1090200005F1030C4FFA8CFCFBB286F818C008F867
:109030000E304AE7978827F480673F043F0C9780FB
:10904000EFE600BFE075002000280020DD7D1582DE
:109050009D7E37761DB91B7E002B7FF415AF93885C
:1090600023F480631B041B0C93800DE7F0B5876924
:1090700083B0064617B13B68BA885A837069DFF837
:10908000A8E08389C3244FF47A734FF0060C6D4631
:109090004FF6FF710EF1010E03E0013B9BB28B42D4
:1090A00020D002899207F8D5A3B283814FF47A7356
:1090B00002E0A3B28B4215D00289D20703F1FF343C
:1090C000F7D5828992B20DB12A700135BCF1000F3B
:1090D0000BD00CF1FF3CFF24BEF1000FE1D09EF855
:1090E0000040D7E71EF0F2FFB76917B13B68BA88B6
:1090F0001A839DF805009DF801509DF802109DF817
:1091000003409DF804209DF8063041EA052143EA1A
:10911000002342EA04220120A6F85010A6F85220AB
:10912000A6F8543003B0F0BDD8C40408014B186849
:109130001AF086BC9C6A002038B51D4B1B7804468B
:1091400000F1250593B104221A49203041F018FF9F
:1091500028461422184941F013FF012384F83A30BD
:10916000164B1B7873B984F83B3038BD284614225F
:10917000134941F005FF012384F83A300F4B1B7867
:10918000002BF0D00F4B186859689A68DD68E560CD
:1091900020606160A260DD69186959699A69A261FD
:1091A0000123E5612061616184F83B3038BD00BF77
:1091B0002E7800202F780020357800200C780020B1
:1091C0008C0605080D78002010B4292128240122DE
:1091D0000023047041708270C3705DF8044B7047C7
:1091E00038B52C22002141F08DFE034640F2DC51BF
:1091F000642040F21A4240F202241874598213206B
:1092000020219A8240F2753240F26C751C83987668
:109210000E240A201977DA8302210122DD8283F8E5
:109220002B0040F64305197283F82A1083F8224078
:109230009A7383F8252083F829201D841946024853
:10924000BDE8384016F0ACBB9C06050810B50021FF
:109250000446012019F054FA207010BD38B50024DE
:109260000472451EE1B2022019F04AFA0134082CBA
:1092700005F8010FF6D138BD2DE9F04F87B0AB4BA3
:1092800002904068984200F04581A94A90420CBF84
:10929000302238220388029923F040031B041B0C60
:1092A0008968038003889BB223F038031A43028045
:1092B000038843F04003038011B10B688A885A8306
:1092C00040F2E93302E0002B00F090810289013B7B
:1092D00012F0020F9BB2F6D06B23838140F2E93388
:1092E00002E0002B00F082810289013B12F0010FA5
:1092F0009BB2F6D0838940F2E93302E0002B00F004
:1093000072810289013B12F0020F9BB2F6D08023DA
:10931000838140F2E93302E0002B00F0648102898E
:10932000013B12F0010F9BB2F6D08389029B9B6830
:1093300013B11A689B88138306237E4CDFF80082E2
:10934000DFF800A27C4D7D4E04939623DFF8F8C130
:1093500001934FF0100EDAF80430C3F30803002B2A
:1093600040F0B180EFF31183002B40F0AC80206817
:10937000AA6823689842FAD133689A42F7D8D8F895
:1093800000704FF47A7101FB07F39B1AB3FBF7F3FC
:1093900001FB00304FF47A774FF00109DAF804301E
:1093A000C3F30803002B6FD1EFF31183002B6BD1B4
:1093B0002368A96822689342FAD132689142F7D8AB
:1093C000D8F8002007FB02FBABEB0101B1FBF2F187
:1093D00007FB03131B1AB3F57A7FDFD3019B013B15
:1093E0000193B8D1029B9B6813B11A689B88538381
:1093F000029B586840F2E93302E0002B00F08580C0
:109400000289013B12F0020F9BB2F6D0F523838153
:1094100040F2E93301E0002B77D00289013B12F0E2
:10942000010F9BB2F7D08389838940F2E93301E0D1
:10943000002B67D00289013B12F0020F9BB2F7D0DC
:10944000FF23838140F2E93301E0002B5AD00289E7
:10945000013B12F0010F9BB2F7D08389DBB203937B
:10946000029B9A6812B1136891881983039B682B39
:1094700052D0049B013B13F0FF0304937FF465AFCC
:10948000184607B0BDE8F08FEFF311818EF3128814
:10949000D5F808B02B68DB0344BFCCF80090D5F8B2
:1094A00008B02368DCF80020C9B281F31188D8F82D
:1094B0000010134407FB01F2A2EB0B02B2FBF1F226
:1094C00007FB032386E7EFF311838EF31288AF685F
:1094D0002A68D20303D50122CCF80020AF682068A7
:1094E000DCF80090DBB283F31188D8F800104FF459
:1094F0007A72484402FB01F3DB1BB3FBF1F302FB7E
:10950000003047E71EF0E2FDAAE71EF0DFFD029BF8
:10951000586889E73022BDE612B1136892885A83F1
:10952000029B586840F2E93312E000BF0038004067
:10953000003C00407C96002010E000E08496002073
:109540008096002000ED00E078960020002B45D0AA
:109550000289013B12F0020F9BB2F7D08C2383816A
:1095600040F2E93301E0002B38D00289013B12F0D0
:10957000010F9BB2F7D08389838940F2E9330289D6
:10958000013B12F0020F9BB215D1002BF7D11EF058
:109590009DFD029B9B6813B11A689B881383059BF2
:1095A000142B04D3182B17D9543B062B14D90020A5
:1095B00007B0BDE8F08FFF23838140F2E93301E07B
:1095C000002BE4D00289013B12F0010F9BB2F7D0CF
:1095D0008389DBB20593DCE7032052E71EF076FDBA
:1095E000029B5868C8E71EF071FD9FE61EF06EFDF5
:1095F000029B58687FE600BF38B505463B4B406884
:10960000984262D03A4A904214BF0822002203884E
:10961000A96823F040031B041B0C038003889BB242
:1096200023F0380313430380038843F0400303808F
:1096300011B10B688A885A8340F2E93301E0002BAC
:1096400045D00289013B12F0020F9BB2F7D0F523FF
:10965000838140F2E93301E0002B38D00289013BDD
:1096600012F0010F9BB2F7D08389838940F2E9336E
:1096700000E00BB30289013B12F0020F9BB2F8D05D
:10968000FF23838140F2E93300E0ABB10289013B63
:1096900012F0010F9BB2F8D08489E4B2AB6813B129
:1096A0001A689B881383712C1BD008D9AC2C16D058
:1096B000AF2C10D1092038BD1EF008FDEEE7122CAA
:1096C00011D0702C09D1052038BD00229FE71EF073
:1096D000FDFC6868C9E7732C03D0002038BD072063
:1096E00038BD062038BD082038BD00BF0038004016
:1096F000003C004008B5012039F052F9174A936840
:1097000003F00C03042B1ED0082B18D151685368AA
:10971000490203F03F0319D452681148B0FBF3F03B
:10972000C2F3881300FB03F00C4B0E4A5B68C3F3D3
:10973000014301335B00B0FBF3F0106008BD094B3F
:10974000074A1A6008BD074B186008BDB0FBF3F06C
:109750005368C3F3881300FB03F0E5E700380240C9
:109760000024F4009CAB0020427A4AB110B50446B4
:1097700004F10A01D0E9003098470023637210BD5C
:10978000704700BF437A5A1C0344D2B242729972A6
:10979000037A93420AD84AB110B5044604F10A018B
:1097A000D0E9003098470023637210BD704700BFB6
:1097B00028B1302801D0312802D129B300207047C8
:1097C0003228FAD03328F8D03428F6D03528F4D00F
:1097D0002028F2D02128F0D01028EED01128ECD08B
:1097E0001228EAD01328E8D01428E6D01528E4D0AF
:1097F000162803D1B1FA81F0400970471728DDD14E
:10980000B1FA81F04009704701207047302829D013
:10981000312829D0322829D0332829D0342829D0FA
:10982000352829D020282BD021282BD0102825D02E
:10983000112829D0122829D0132829D0142829D05A
:10984000152829D0162805D0172808BF0F2302D0C5
:10985000002070470E23114A03EB4303134493F88F
:109860006A0070470023F6E70123F4E70223F2E7DA
:109870000323F0E70423EEE70523ECE70823EAE7F8
:109880000623E8E70723E6E70923E4E70A23E2E7FC
:109890000B23E0E70C23DEE70D23DCE778C40408A4
:1098A000024A136823EA000010607047A8B800203D
:1098B000DFED2E7AB4EEE70AF1EE10FA4ADDDFEDC5
:1098C0002C6A9FED2C7A01E0B0EE670AB4EEC70A6D
:1098D000F1EE10FA70EE667AF6DC9FED277AF4EE80
:1098E000C77AF1EE10FA3ED5DFED216A9FED237ABB
:1098F00001E0F0EE407AF4EEC77AF1EE10FA37EEBE
:10990000A60AF6D4DFED1E7AB4EEE70AF1EE10FAFD
:1099100014DDDFED167A37EEC00A60EE006A9FEDC7
:10992000196A9FED197ADFED197AA6EE867A20EE94
:10993000266AE6EE877AA6EE270A7047DFED147AEC
:10994000B4EEE70AF1EE10FA44BFDFED0B7A37EE22
:10995000C00AE2E79FED087AF0EE407AF4EEC77AAB
:10996000F1EE10FAC0D4B0EE670ACBE7DB0F494046
:10997000DB0FC940E4CB1641DB0F49C0E4CB16C175
:10998000DB0FC93F92E741B99730083C15A82ABEC2
:10999000DB0FC9BFF0EEC07AB0EEE07AB4EEE77A42
:1099A000F1EE10FAB4BFB0EE676AB0EE476AB5EEFA
:1099B000406AF1EE10FA46D0B4EEE77AF1EE10FA12
:1099C0008CBFF0EE675AF0EE475AC5EE866A9FEDFF
:1099D0001F3A9FED1F6A9FED1F4A9FED1F5ADFED53
:1099E0001F3ADFED1F4ADFED1F5AA6EEC36AE6EE0F
:1099F000A34AA6EE864AB7EE006AA6EE845AA6EE01
:109A0000A46AE6EE855AC5EE866AB4EEE77AF1EE10
:109A100010FA48BFDFED147AF5EEC00A48BF77EEC2
:109A2000E66AF1EE10FA48BFDFED107AB5EEC00A33
:109A300048BF77EEE66AF1EE10FA48BFF1EE666ACB
:109A4000B0EE660A7047DFED076ADEE739094E3D82
:109A5000E3B59E3E88FA163E45FE7F3F99FB243FC4
:109A600069A2163EA7DFA834DB0FC93FDB0F4940D0
:109A7000DFED317A30EE277AFDEEC76A16EE903AC6
:109A80002033402B02D99FED2D0A7047B4EEE70A30
:109A9000F1EE10FA4DDD9FED2A6ADFED2A6A01E052
:109AA000B0EE677AB4EEE67AF1EE10FA77EE467A27
:109AB000F6DC9FED257AF4EEC77AF1EE10FA35D593
:109AC000DFED1F6A9FED217A01E0F0EE407AF4EEBF
:109AD000C77AF1EE10FA37EEA60AF6D4DFED167A61
:109AE000B4EEE70AF1EE10FA1BDCDFED197AB4EE02
:109AF000E70AF1EE10FA44BFDFED137A37EEC00A41
:109B000060EE006A9FED136A9FED137ADFED137A22
:109B1000A6EE867A20EE266AE6EE877AA6EE270A79
:109B20007047DFED0F7A37EEC00AE9E7B0EE670A5B
:109B3000D4E7F0EE477ABCE7DB0FC93F0000000036
:109B4000DB0FC940E4CB1641DB0F49C0E4CB16C1A3
:109B5000DB0FC9BF92E741B99730083C15A82ABE70
:109B6000DB0F494010B44C09012250F8243001F0B9
:109B70001F0102FA01F10B4340F824305DF8044B59
:109B8000704700BF4B0901F01F0150F8232001234B
:109B900003FA01F1114214BF18460020704700BFBC
:109BA0002DE9F043002489B006460D461F46A04625
:109BB00005E025290CD030460134A847039A531CF0
:109BC000039311780029F4D1204609B0BDE8F08351
:109BD000931CCDE903385078302842D0A0F13003EF
:109BE000DBB2092B4FF0000945D96C282AD0642834
:109BF00073D019D9732858D063D9752840F0828062
:109C000007F1040C386805AB00220A216746FEF70D
:109C100027FB05AB049A009329464B463046FEF7D6
:109C2000F5F9039A0444CAE725283CD051D95828AD
:109C30006BD06328C2D139783046A8470437013445
:109C4000039ABCE7039B5A1C03921B78642B52D0E7
:109C500016D8252B27D064D9582B18D0632BEAD0DF
:109C6000ADE7D31C03939078A0F13003DBB2092B4E
:109C70004FF00109B9D804AA03A93DF0D9FCB4E713
:109C8000732B12D051D9752B2DD0782B97D1A3F1EE
:109C90005802B2FA82F23868520905AB1021043733
:109CA000FEF7DEFAB5E7252185E73B68049A0093C5
:109CB000294600233046FEF7A9F904370444039AE5
:109CC0007DE76E287FF47AAF039A3B6804371C6007
:109CD00075E700283FF478AF70E7386805A9FEF70C
:109CE00089FA043795E7386805AB00220A21FEF7A8
:109CF000B7FA04378DE73B1D386805A91F46FEF704
:109D000079FA86E778287FF459AFA0F15802B2FAC1
:109D100082F23868520905AB1021FEF7A1FA043728
:109D200077E7002B3FF450AF49E76E2BCDD046E7E5
:109D30000EB400B584B005AB019053F8042B06496E
:109D4000039301A8FFF72CFF019B00221A7004B0B7
:109D50005DF804EB03B070470180000870B406683A
:109D60008E4217D90139751E002311F8014F0822C0
:109D7000634013F0800F4FEA430318BF83F0D5030D
:109D8000013ADBB2F5D18D42EFD1721C0260337023
:109D900070BC7047721C00230260337070BC704747
:109DA0000A44914215D010B40139541E11F8012F04
:109DB0000823504010F0800F4FEA400018BF80F099
:109DC000D500013BC0B2F5D1A142EFD15DF8044B03
:109DD000704770474840082310F0800F4FEA40005A
:109DE00018BF80F0D500013BC0B2F5D1704700BF6D
:109DF0000A44914215D030B40139551E41F2210276
:109E000011F8014F082380EA042004044CBF82EAC1
:109E100040004000013B80B2F7D18D42F0D130BC10
:109E20007047704770B502221349144C144E4FF618
:109E3000FF70FFF7DDFF22884AB1A518B54218D29E
:109E4000052A16D92146FFF7D3FF2C46F3E7214612
:109E50000222FFF7CDFF0222A118FFF7C9FF094B2D
:109E6000E41A094B1C8041F60F53C31A584258415B
:109E700070BD0020FCE700BF004000080240000861
:109E800000800008FA3F0008F87700200F4B2DE90A
:109E90003048D3E9004554EA05020AD1034640F2AE
:109EA000011200201880988098715A801881BDE8AE
:109EB0003088074B1A6814EB020B45F1000C5A4628
:109EC0006346FEF7DFF80120BDE8308858400020E7
:109ED0007C96002030B403888278C478154DA3F5B1
:109EE000FA6303F0030101EB4101013A02EB810245
:109EF0009B0835F812500279611E40F2B55404FBFC
:109F000003132B4403EB430302EBC303427984792D
:109F100009490089C3EB031302EB83032144C3EB1C
:109F2000031301EB83034FF47A720021C2FB030198
:109F300030BC704778C4040880436D382DE9F04781
:109F400007468CB01E469246002A5CD11546144640
:109F50000A88B2F5FA6F36D38B78581E0B2832D8A0
:109F600091F803C00CF1FF301E282CD891F804E0C2
:109F7000BEF1170F27D891F80590B9F13B0F22D801
:109F800088793B281FD8B1F80880B8F57A7F1AD2B3
:109F90004FF001085EBB09890491002CB4BF2D214C
:109FA0002B21002CB8BF6442CDE90290CDE9051405
:109FB0000795CDE900CE38462A49FFF7B9FE40465D
:109FC0000CB0BDE8F08700232749ADF828304FF0EA
:109FD000010C18468DF82A30ADF82C3099469E4673
:109FE0001A4698460991634609A9002ED3D0CDE9B7
:109FF0000290CDE900CE38461C49FFF799FE404655
:10A000000CB0BDE8F0871A4C84FB0234A318D417B7
:10A01000C4EB6314C4EB0415A2EB85052DB2002D2F
:10A020000846B8BF6D42FFF755FF4FF47A72002320
:10A030008046894640F088FC3C230AFB030A4FF423
:10A040007A7200234046494640F07EFC4FF47A7114
:10A0500092B20023C1FB0A2309A8FEF713F824B229
:10A0600009A975E7C806050800000101A80605084A
:10A07000898888880378202B024600F10100F9D0F6
:10A08000092BF7D02D2B00F0A4802B2B03BF537886
:10A09000B7EE000A0246B7EE000AA3F13001C8B2DB
:10A0A00009289FED577A10D8F2EE046A07EE901A4D
:10A0B000F8EEE77A12F8013FE7EE267AA3F13001D5
:10A0C000C8B20928B0EE677AF0D92E2B63D003F01E
:10A0D000DF03452B02D020EE070A704710B45178F9
:10A0E0002D294FD02B2979D0A1F13003092B02F172
:10A0F00001027AD80024002303EB830301EB43031E
:10A1000012F8011FA1F130000928A3F13003F3D99F
:10A11000B3F59A7F1A4628BF4FF49A72072B6CD971
:10A12000DFED386A1346F7EE007A083B072B67EE3F
:10A13000A67AFAD802F00702DAB1F2EE046A012A2E
:10A1400067EEA67A15D0022A67EEA67A11D0032A06
:10A1500067EEA67A0DD0042A67EEA67A09D0052A02
:10A1600067EEA67A05D067EEA67A062A18BF67EED4
:10A17000A67A002C3BD087EE277A5DF8044B20EEC0
:10A18000070A70479178A1F13003092B02F102020E
:10A1900030D80124AFE75378A3F13001C8B20928C1
:10A1A00002F1010293D8F2EE046AF0EE665A07EE6D
:10A1B000901AF8EEE77A12F8013F87EEA66AA3F14B
:10A1C0003001C8B2092866EEA56A37EE067AEED9E4
:10A1D0007DE75378BFEE000A02465EE79178A1F171
:10A1E0003003092B02F1020284D9F7EE007A27EE40
:10A1F000277AC2E7F7EE007ABDE7F7EE007A9BE731
:10A200000000000020BCBE4CF8B5064615460846C6
:10A21000B6FBF2F434B905FB14640C4B1B5D00F87B
:10A22000013BF8BDB4FBF2F75FB905FB1747074BDD
:10A2300005FB1464DA5D00F8012B1B5D00F8013B9F
:10A24000F8BD3846FFF7E0FFEFE700BFF806050866
:10A25000B5EEC00ADFED677A674AF1EE10FACCBFBF
:10A2600030EE270A30EE670ADFED647A20EE270A27
:10A270002DE9F047FDEEC07A88B017EE904A84EAE7
:10A28000E4760023A6EBE476CDE902330493A2FB47
:10A2900006325FEAD208054641D105AF5848394633
:10A2A000554BA3FB0623DB0803EB8303A6EB430319
:10A2B000002CC35C0B704FF00002ACBF20232D2399
:10A2C0004A7038468DF808303FF048FE012839467C
:10A2D00039D0022842D0032805BF302302A802A8A3
:10A2E0008DF8093040F016FE02A83FF037FE033823
:10A2F000C4B2224602A9284640F042FE00232B5554
:10A3000028463FF02BFE2E22431C02A92A5421444A
:10A31000E81840F01BFE284608B0BDE8F087394B2E
:10A32000A3FB06235B0922D105AF35483946324AE3
:10A33000A2FB0832D20802EB8202A8EB4202835C45
:10A3400001F8013BACE7302302A88DF809308DF805
:10A350000A308DF80B3040F0DDFDC5E7302302A850
:10A360008DF809308DF80A3040F0D4FDBCE7264A5C
:10A37000A2FB06125FEA92190ED105AF20483946BA
:10A380001D4AA2FB03C2D20802EB8202A3EB4203E6
:10A39000C35C01F8013BCAE71C4AA2FB06125FEA54
:10A3A000523A0ED105AF16483946134AA2FB09C2EC
:10A3B000D20802EB8202A9EB4202825C01F8012B77
:10A3C000DEE71348B6FBF0F058B905AF39460A206E
:10A3D000BAFBF0F200FB12A20948825C01F8012BE3
:10A3E000E3E705AF39460A220193FFF70DFF019B12
:10A3F0000146ECE76F12033ACDCCCCCC00007A4496
:10A40000F80605081F85EB51D34D62105917B7D1D7
:10A41000A086010002B370B48E1803E0121B14D1A1
:10A42000B14215D010F8012BA2F14103192B11F8FC
:10A43000013BA3F1410598BF2032192D03F12004FF
:10A44000ECD9D21A01D1002BEAD1104670BC70476A
:10A450000022104670BC70471046704770B5044625
:10A4600008460D463FF07AFD064602E014F8013F2B
:10A4700043B1324629462046FFF7CCFF0028F5D1EC
:10A48000204670BD1C46204670BD00BF4FF0FF3215
:10A49000FFF7C0BFA0F16103192B98BF20387047A8
:10A4A000A0F14103192B98BF20307047202805D018
:10A4B000093804288CBF0020012070470120704714
:10A4C0002DE9F0411F46064603461C782046FFF75B
:10A4D000EDFF1D4601330028F7D12B2C51D02D2C38
:10A4E00024D0102A804628D04FF0FF33B3FBF2F37C
:10A4F00002FB03FC6FEA0C0C5FFA8CFC01350020B8
:10A500000BE0303CE4B2944225DA98422E461DD846
:10A510001AD002FB004015F8014B392CF1D944F058
:10A520002004602C17D9573CE4B2ECE74FF0010847
:10A53000102A6C7805F10105D6D1302C23D06FF0AC
:10A5400070434FF00F0CD9E76445E2D907EA0808D9
:10A550004FF0FF30DFE701B10E60B8F1000F08D017
:10A5600027B1B0F1004F28BF4FF000404042BDE896
:10A57000F081002FFBD06FF00043984228BF1846AF
:10A58000F5E78046D4E76C782046FFF789FF782806
:10A5900005F1010605D035466FF070434FF00F0C02
:10A5A000ACE7AC786FF0704302354FF00F0CA5E7C5
:10A5B00001230A22002183E7613819288CBF00207B
:10A5C00001207047413819288CBF002001207047B6
:10A5D000303809288CBF002001207047A0F13003DB
:10A5E000092B07D920F02000413819288CBF002002
:10A5F000012070470120704707EE901AF8EE677A45
:10A600009FED807A27EE800A20EE070AFDEEC07AE1
:10A6100017EE903A2033402B7BD8DFED7B7AB4EEF7
:10A62000E70AF1EE10FA40F3E180B0EE407A9FEDD8
:10A63000776ADFED776A01E0B0EE677AB4EEE67A2A
:10A64000F1EE10FA77EE467AF6DC9FED727AF4EED0
:10A65000C77AF1EE10FA40F1CC809FED6C6ADFED25
:10A660006E6A01E0F0EE477AF4EEE67AF1EE10FA67
:10A6700037EE867AF6D4DFED697AB4EEE77AF1EE5A
:10A6800010FA40F3A280DFED607A37EEC77A27EE4A
:10A69000076ADFED635ADFED637ADFED636A9FEDF2
:10A6A000635AE6EE257A67EE065AE6EE276AF7EE7B
:10A6B000007AA5EEA67AF0EE675AE7EE055AE7EEC5
:10A6C000457A87EEA55ADFED557A30EE277AFDEE12
:10A6D000C76A16EE903A2033402B1FD99FED547A6B
:10A6E000F6EE006AB7EE006AF7EE004AC4EEA57A0D
:10A6F00080ED045A67EEA66A27EE866A27EE877A0F
:10A70000C0ED006AC0ED026A80ED016A80ED037A57
:10A710007047B7EE005AF0EE455AD4E7B4EEE70AB8
:10A72000F1EE10FA6BDD9FED396ADFED396A01E079
:10A73000B0EE677AB4EEE67AF1EE10FA77EE467A8A
:10A74000F6DC9FED347AF4EEC77AF1EE10FA53D5C9
:10A750009FED2E6ADFED306A01E0F0EE477AF4EE0D
:10A76000E67AF1EE10FA37EE867AF6D4DFED2B7A40
:10A77000B4EEE77AF1EE10FA33DCDFED2E7AB4EEC8
:10A78000E77AF1EE10FA44BFDFED227A37EEC77AAE
:10A7900027EE076ADFED224ADFED226ADFED227A3B
:10A7A000E6EE246A67EE064AE6EE267AB7EE006A1F
:10A7B000A4EEA77AF6EE006A36EE476AF8EE007A63
:10A7C00027EE277A66EE266A8EE7DFED1A7AB4EE78
:10A7D000E77AF1EE10FA44BFDFED0E7A37EEC77A72
:10A7E00055E7DFED097A37EEC77AD1E7F0EE407A28
:10A7F0002BE7B0EE677A3EE7B0EE677AB6E7F0EEA9
:10A80000477A9EE727D4D236DB0F4940DB0FC94099
:10A81000E4CB1641DB0F49C0E4CB16C1DB0FC93FC7
:10A8200092E741B99730083C15A82ABEF304353F9A
:10A8300000000000DB0FC9BF07EE901AF8EE677A40
:10A840009FED837A27EE800A20EE070AFDEEC07A9C
:10A8500017EE903A2033402B00F28180DFED7D7AB5
:10A86000B4EEE70AF1EE10FA40F3E680B0EE407A7B
:10A870009FED796ADFED796A01E0B0EE677AB4EEB8
:10A88000E67AF1EE10FA77EE467AF6DC9FED747A0E
:10A89000F4EEC77AF1EE10FA40F1D1809FED6E6AC6
:10A8A000DFED706A01E0F0EE477AF4EEE67AF1EE61
:10A8B00010FA37EE867AF6D4DFED6B7AB4EEE77AEB
:10A8C000F1EE10FA40F3A780DFED627A37EEC77A37
:10A8D00027EE076ADFED655ADFED657ADFED656A21
:10A8E0009FED655AE6EE257A67EE065AE6EE276A90
:10A8F000F7EE007AA5EEA67AF0EE675AE7EE055A73
:10A90000E7EE457A87EEA55ADFED577A30EE277AE3
:10A91000FDEEC76A16EE903A2033402B24D99FED06
:10A92000577AF6EE006AB7EE006AF7EE004AC4EE18
:10A93000A57A0023836143610362C36180ED045AF9
:10A9400067EEA66A27EE866A27EE877AC0ED006A70
:10A95000C0ED026A80ED016A80ED037A7047B7EEC0
:10A96000005AF0EE455ACFE7B4EEE70AF1EE10FADE
:10A970006BDD9FED396ADFED396A01E0B0EE677A91
:10A98000B4EEE67AF1EE10FA77EE467AF6DC9FED59
:10A99000347AF4EEC77AF1EE10FA53D59FED2E6AB1
:10A9A000DFED306A01E0F0EE477AF4EEE67AF1EEA0
:10A9B00010FA37EE867AF6D4DFED2B7AB4EEE77A2A
:10A9C000F1EE10FA33DCDFED2E7AB4EEE77AF1EE39
:10A9D00010FA44BFDFED227A37EEC77A27EE076A16
:10A9E000DFED224ADFED226ADFED227AE6EE246A0D
:10A9F00067EE064AE6EE267AB7EE006AA4EEA77A7C
:10AA0000F6EE006A36EE476AF8EE007A27EE277A0D
:10AA100066EE266A89E7DFED1A7AB4EEE77AF1EEA0
:10AA200010FA44BFDFED0E7A37EEC77A50E7DFED5C
:10AA3000097A37EEC77AD1E7F0EE407A26E7B0EE32
:10AA4000677A39E7B0EE677AB6E7F0EE477A9EE7C5
:10AA500027D4D236DB0F4940DB0FC940E4CB164187
:10AA6000DB0F49C0E4CB16C1DB0FC93F92E741B908
:10AA70009730083C15A82ABEF304353F00000000BB
:10AA8000DB0FC9BF10EE103AC3F3160242F07E523C
:10AA900007EE102ADFED167ADFED164A9FED165A03
:10AAA000DFED165A9FED166ADFED163ADFED166AF6
:10AAB0009FED164AE7EE274ADB1507EE903AA4EE23
:10AAC000875AF8EEE77AE5EE075A67EEA37AA5EE25
:10AAD000876AB5EEC00AE6EE077AF1EE10FAD4BF47
:10AAE000B0EE440AB0EE660A37EE800A704700BF47
:10AAF000DACDFE3CB9D593BE5CB8903FAA841DC0A8
:10AB000022E061401872313F07F1B3C2000080FFBC
:10AB1000DFED1D3ADFED1D7A9FED1D7A9FED1D4A99
:10AB2000DFED1D4A9FED1D5ADFED1D5A9FED1D6A99
:10AB3000DFED1D6AE0EE237AF4EEC77AF1EE10FA4B
:10AB400088BFF0EE477AF4EEC47AF1EE10FAB8BF9F
:10AB5000F0EE447AFDEEE77A17EE903AC3F3160270
:10AB600042F07E5207EE102AA7EE245A03F0FF436C
:10AB700000EE103AE5EE075AA5EE876AE6EE076AA0
:10AB800026EE800A704700BF3BAA384B00007E4E7D
:10AB90000000FF4E00000000ED185E3C81900FBBEE
:10ABA000AF9D2A3EB2D19F3EE886023F30B4026894
:10ABB0001146531C036011F8024B0160D31C5178FD
:10ABC00003609378151D05601B0443EA0123D078C8
:10ABD000234343EA006030BC704700BF0368591C40
:10ABE0001A46016012F8021B0260587841EA002000
:10ABF000704700BF03685A1C02601878704700BF96
:10AC000070B5044608460E463FF0A8F931460546A1
:10AC10000246206840F016F920682844206070BD84
:10AC200038B504460068154640F00CF922682A44FD
:10AC3000226038BD036810B40A0E5C1C04601A70F0
:10AC400003680A0C5C1C04601A7003680A0A5C1C26
:10AC500004601A7003685A1C026019705DF8044B96
:10AC6000704700BF036810B40A0A5C1C04601A70C5
:10AC700003685A1C026019705DF8044B704700BFEE
:10AC800003685A1C026010B4197003680A0A5C1C3D
:10AC900004601A7003680A0C5C1C04601A70036874
:10ACA000090E5A1C026019705DF8044B704700BF12
:10ACB00003685A1C026019700368090A5A1C026072
:10ACC0001970704770B544880546C4F30B042246DA
:10ACD00008460E46002140F015F92B69094A9342B7
:10ACE00002D3094A934205D35BB121463046BDE801
:10ACF00070401847224630461946BDE8704040F083
:10AD0000A1B870BDDC0600080C08000838B5064C78
:10AD1000064DAC4206D2616820461434FFF7D2FFDC
:10AD2000AC42F8D338BD00BFA0010008DC06000823
:10AD3000084B09498B4203D309E014338B4206D2F6
:10AD40001A88C2F30B029042F7D1184670470023CD
:10AD500018467047A0010008DC060008164B984210
:10AD600028D003F58063984224D0038823F0400361
:10AD7000B1F5807F4FEA0343A8BF4FF480711B0CED
:10AD8000038002290388B8BF022191FAA1F20029A9
:10AD9000B2FA82F29BB208BF4FF0FF32013A23F0C1
:10ADA000380343EAC2039BB20380038843F04003A5
:10ADB000038070474908D8E70038004030B5204D7F
:10ADC00083B06B6840F2E93200E062B31C89013A5B
:10ADD00014F0020F92B2F8D080B2988140F2E932BA
:10ADE00000E002B31889013A10F0010F92B2F8D0D6
:10ADF0009A8940F2E93200E0E2B11889013A10F094
:10AE0000020F92B2F8D089B2998140F2E93200E0A3
:10AE100082B11989013A11F0010F92B2F8D09889E4
:10AE2000C0B203B030BD184601911DF04FF96B68F8
:10AE30000199DEE718461DF049F9C0B203B030BDF4
:10AE4000209400202DE9F84FDFF8D08298F80030E8
:10AE500003B1FEE7AB4EAC4AAC4B044670681B88AE
:10AE60000125904288F8005000F0718102F580625F
:10AE7000904200F06C810288B56822F04002B3F580
:10AE8000807F4FEA0242A8BF4FF48073120C028009
:10AE9000022B0288B8BF0223002B93FAA3F3B3FA64
:10AEA00083F392B208BF4FF0FF33013B22F0380228
:10AEB00042EAC3039BB20380038843F0400303804C
:10AEC00015B12B68AA885A83914B01221A708B46C0
:10AED00040F2E93302E0002B00F040810289013B9F
:10AEE00012F0020F9BB2F6D00023838140F2E933C7
:10AEF00002E0002B00F032810289013B12F0010FC9
:10AF00009BB2F6D0838940F2E93302E0002B00F0D7
:10AF100022810289013B12F0020F9BB2F6D000237E
:10AF2000838140F2E93302E0002B00F014810289B2
:10AF3000013B12F0010F9BB2F6D08389754F214679
:10AF40000920FFF73BFF0BF1FF3B00254FF00A0AFA
:10AF50004FF00B09706840F2E93302E0002B00F07B
:10AF6000DF800289013B12F0020F9BB2F6D0A0F8FD
:10AF70000CA040F2E93302E0002B00F0D1800289FE
:10AF8000013B12F0010F9BB2F6D0838940F2E93306
:10AF900002E0002B00F0C8800289013B12F0020F92
:10AFA0009BB2F6D0ABB2838140F2E93302E0002BD2
:10AFB00000F0BA800289013B12F0010F9BB2F6D07B
:10AFC00083891BF8014F40F2E93302E0002B00F0C7
:10AFD000AF800289013B12F0020F9BB2F6D0A0F8BD
:10AFE0000C9040F2E93302E0002B00F0A1800289CE
:10AFF000013B12F0010F9BB2F6D0838940F2E93396
:10B0000001E0002B7BD00289013B12F0020F9BB2C2
:10B01000F7D0A4B2848140F2E93301E0002B6ED076
:10B020000289013B12F0010F9BB2F7D083893B6884
:10B0300033B11A689B8851690B4214BF5383138341
:10B040000135362D86D1A0210820FFF7B7FE7368A1
:10B05000A025002440F2E93201E0002A72D01989CB
:10B06000013A11F0020F92B2F7D09D8140F2E9321D
:10B0700001E0002A66D01989013A11F0010F92B25D
:10B08000F7D09A8940F2E93201E0002A54D01989B8
:10B09000013A11F0020F92B2F7D09C8140F2E932EE
:10B0A00001E0002A48D01989013A11F0010F92B24B
:10B0B000F7D09889C0B28206CCD4B26812B11168B8
:10B0C00092880A83104A934243D013498B4214BF9B
:10B0D000082100211A8822F040021204120C1A8062
:10B0E0001A8892B222F03802114319801A8800217E
:10B0F00042F040021A8088F80010BDE8F88F1CF07A
:10B10000E5FF94E7209400200038004074200020E0
:10B110001542002048960020003C00400D420020CF
:10B120001CF0D4FF706831E71CF0D0FF706848E76E
:10B130001CF0CCFF706861E718461CF0C7FF73680D
:10B14000C0B2B8E718461CF0C1FF73689AE75B0805
:10B1500091E60021BEE71CF0B9FFEFE61CF0B6FF58
:10B160007068D0E62DE9F84FDFF8DCA2B04BDAF8D2
:10B170000400B04A9842128800F0578103F58063BA
:10B18000984200F052810388DAF8084023F0400327
:10B19000B2F5807F4FEA0343A8BF4FF480721B0CC7
:10B1A0000380022A0388B8BF022292FAA2F1002A81
:10B1B000B1FA81F19BB208BF4FF0FF31013923F0A2
:10B1C000380343EAC1039BB20380038843F0400382
:10B1D000038014B12368A2885A8340F2E93302E065
:10B1E000002B00F05A810289013B12F0020F9BB242
:10B1F000F6D00523838140F2E93302E0002B00F012
:10B200004C810289013B12F0010F9BB2F6D0838979
:10B2100040F2E93302E0002B00F049810289013B52
:10B2200012F0020F9BB2F6D00023838140F2E93383
:10B2300002E0002B00F03B810289013B12F0010F7C
:10B240009BB2F6D0838940F2E93302E0002B00F094
:10B2500029810289013B12F0020F9BB2F6D006232E
:10B26000838140F2E93302E0002B00F01B81028968
:10B27000013B12F0010F9BB2F6D0838940F2E93313
:10B2800002E0002B00F006810289013B12F0020F60
:10B290009BB2F6D00023838140F2E93302E0002B19
:10B2A00000F0F8800289013B12F0010F9BB2F6D04A
:10B2B0008389614DDFF89481EC7E042044F0010124
:10B2C000FFF77CFDB8F80030002B4CD005F11C09CD
:10B2D0005A4F4E464FF0200B072517F8014FDAF86A
:10B2E0000400FF2C40F2E93303D174E0002B00F09E
:10B2F000C5800189013B11F0020F9BB2F6D0858118
:10B3000040F2E93302E0002B00F0B8800189013BF4
:10B3100011F0010F9BB2F6D0838940F2E93302E0CD
:10B32000002B00F095800189013B11F0020F9BB2C8
:10B33000F6D0A4B2848140F2E93302E0002B00F0A1
:10B3400087800189013B11F0010F9BB2F6D0838900
:10B350003B7806F8013BB8F80010A6EB09039942C8
:10B36000BBDC354BDC7EFF210720FFF727FD2146A4
:10B370000420FFF723FDB8F8003043B1304E00241D
:10B3800016F8015BFF2D66D00134A342F8DCDAF831
:10B39000083013B11A689B881383DAF80430244A02
:10B3A000934275D027498B4214BF082100211A8887
:10B3B00022F040021204120C1A801A8892B222F073
:10B3C00038020A431A801A8842F040021A80BDE807
:10B3D000F88F002B57D00189013B11F0020F9BB26F
:10B3E000F7D0858140F2E93301E0002B4BD0018991
:10B3F000013B11F0010F9BB2F7D0838940F2E93392
:10B4000000E02BB30189013B11F0020F9BB2F8D091
:10B41000A0F80CB040F2E93300E0CBB10189013B68
:10B4200011F0010F9BB2F8D091E75208ABE600BFD4
:10B4300000380040742000200028002077300020D1
:10B4400078300020003C0040209400201C000020A8
:10B450001CF03CFE7CE7C4F307210520FFF7AEFC9F
:10B46000E1B20620FFF7AAFC29460720FFF7A6FC59
:10B47000B8F8003001349C4282DB88E71CF026FEDD
:10B48000DAF8040049E71CF021FEDAF80400B5E719
:10B4900000218CE71CF01AFE0BE71CF017FEDAF80F
:10B4A0000400B5E61CF012FEDAF80400E6E61CF033
:10B4B0000DFEDAF80400C6E62DE9F843B04CB14BB6
:10B4C0006068B14D9842B5F800C000F0408103F5C6
:10B4D0008063984200F03B8163460188A26821F0B6
:10B4E0004001B3F5807F4FEA0141A8BF4FF480735C
:10B4F000090C0180022B0188B8BF0223002B93FAAC
:10B50000A3F3B3FA83F389B208BF4FF0FF33013BD3
:10B5100021F0380141EAC3039BB20380038843F062
:10B520004003038012B1136891885983974B1B78AD
:10B53000012B00F09A81C0F05081022B00F00A81AB
:10B54000934E337813F0400F0CBF4FF4C3714FF498
:10B55000F0718C4B8F4F9842398000F0068103F5D3
:10B560008063984200F00181038823F04003BCF51A
:10B57000807F4FEA0343A8BF4FF4807C1B0C0380FD
:10B58000BCF1020F0388B8BF4FF0020C9CFAACF17B
:10B59000BCF1000FB1FA81F19BB208BF4FF0FF314F
:10B5A000013923F0380343EAC1039BB203800388C7
:10B5B00043F04003038012B1136892885A834FF01E
:10B5C00010084FF0010940F2E93302E0002B00F0CF
:10B5D000CF800289013B12F0020F9BB2F6D01FFA16
:10B5E00088F3838140F2E93302E0002B00F0C08051
:10B5F0000289013B12F0010F9BB2F6D0838940F221
:10B60000E93302E0002B00F0B7800289013B12F021
:10B61000020F9BB2F6D0A0F80C9040F2E93302E0A2
:10B62000002B00F0A9800289013B12F0010F9BB2B0
:10B63000F6D0838908F10108B8F1200FC3D1A168C1
:10B6400011B10B688A881A834E4B984200F0B08083
:10B6500003F58063984200F0AB8003882D8823F0C7
:10B6600040031B041B0C038003889BB223F03803A8
:10B6700043F008030380038843F0400303800388FA
:10B6800023F04003B5F5807F4FEA0343A8BF4FF492
:10B6900080751B0C0380022D0388B8BF022595FA24
:10B6A000A5F2002DB2FA82F29BB208BF4FF0FF3232
:10B6B000013A23F0380343EAC2039BB203800388B4
:10B6C00043F04003038011B10B688A885A833178B4
:10B6D0000020FFF773FB304B02201978FFF76EFB59
:10B6E0002E4B03201978FFF769FB2D4BD97E0420E0
:10B6F0000143FFF763FBA36813B11A689B881383A8
:10B700006368204A934266D0264DAB4214BF082599
:10B71000002519883A88244C244821F04001090466
:10B72000090C1980198889B221F038012943198040
:10B73000198841F04001198000213FF0E3FB237894
:10B740001BB1FFF70FFD00232370BDE8F8834FEA1C
:10B750005C03C2E60E4E082333700A4B0D4F4FF4C4
:10B76000C371984239807FF4FAAE4FEA5C0CFBE675
:10B770001CF0ACFC606842E71CF0A8FC606859E76C
:10B780002094002000380040742000206C94002099
:10B79000FD0100201C000020739400207494002000
:10B7A00000280020003C0040000000201C28002051
:10B7B000038823F040031B041B0C0380038823F041
:10B7C00038031B041B0C0380038843F040030380F1
:10B7D0002D886D0853E700259BE740F2E93301E02F
:10B7E000002B4CD00289013B12F0020F9BB2F7D024
:10B7F000A023838140F2E93301E0002B3FD002898E
:10B80000013B12F0010F9BB2F7D0838940F2E9337C
:10B8100000E083B30289013B12F0020F9BB2F8D023
:10B820000023838140F2E93300E023B30289013B26
:10B8300012F0010F9BB2F8D08389D8B200F0060352
:10B84000022B114E0AD000F00503012B06D148232C
:10B850006068B5F800C0A268337009E0082360682A
:10B86000B5F800C0A268337077E7074E48233370FD
:10B870004FF4F0716DE61CF029FCC0B2DEE71CF05D
:10B8800025FC6068C2E700BFFD0100202DE9F843F8
:10B890009E4C9F4963689F4D8B422A8800F093809D
:10B8A00001F580618B4200F08E801988A06821F03C
:10B8B0004001B2F5807F4FEA0141A8BF4FF480728A
:10B8C000090C1980022A1988B8BF0222002A92FAAC
:10B8D000A2F2B2FA82F289B208BF4FF0FF32013A07
:10B8E00021F0380141EAC20292B21A801A8842F06D
:10B8F00040021A8010B102688188518340F2E93217
:10B9000001E0002A6CD01989013A11F0020F92B2BD
:10B91000F7D080229A8140F2E93201E0002A5FD01C
:10B920001989013A11F0010F92B2F7D09A8940F2C9
:10B93000E93201E0002A4DD01989013A11F0020FD5
:10B9400092B2F7D000229A8140F2E93201E0002A57
:10B9500040D01989013A11F0010F92B2F7D09889BD
:10B96000C0B2A26812B1116892880A83684A9342F1
:10B970002ED069498B4214BF082100211A88674ED6
:10B98000674F22F040021204120C1A801A8892B2F9
:10B9900022F038020A431A801A8842F040021A80C4
:10B9A0003278D7F8008082420FD15E4A127842B9CD
:10B9B000DFF87C91D9F8FC21A8EB0202B2F57A7F7E
:10B9C00013D8BDE8F88352086FE7BDE8F84373E584
:10B9D0000021D3E718461CF079FB6368C0B2C0E7CA
:10B9E00018461CF073FB6368A1E718462988FFF727
:10B9F000B5F9A36813B11A689B885383636840F252
:10BA0000E93201E0002A78D01989013A11F0020FD9
:10BA100092B2F7D0A0229A8140F2E93201E0002AE6
:10BA20006BD01989013A11F0010F92B2F7D09A89BF
:10BA300040F2E93201E0002A59D01989013A11F0A7
:10BA4000020F92B2F7D000229A8140F2E93201E06F
:10BA5000002A4CD01989013A11F0010F92B2F7D0A7
:10BA60009A89D5B2A26812B1116892880A832E4CC5
:10BA700018460421FFF772F92378192B0CD133787B
:10BA80002A4A03F04003002B05F007010CBF0D20EC
:10BA9000102013805180D080690706D50023C9F893
:10BAA0000032C9F8FC81BDE8F88305F00505012DD9
:10BAB00019D0002DF5D133785B06F2D5D9F80022E4
:10BAC0003B68FAB19B1A642BEBD9FFF7F5FC23789E
:10BAD000192BE6D1B9F80432144A01339BB2A9F804
:10BAE00004329380DDE733785A06E7D5D9E7184664
:10BAF0001CF0ECFA6368C5B2B4E718461CF0E6FA2D
:10BB0000636895E7C9F80032CBE700BF20940020B6
:10BB10000038004074200020003C0040FD0100205F
:10BB20007C9600206C940020619400206494002096
:10BB3000002800202DE9F84F664A674E0123137054
:10BB4000FFF7A4FEB6F86034644ADFF8A4E1B2F867
:10BB5000008003F1640C1FFA8CFC00214FF0050BF0
:10BB60004FF0060A4FF0070902E0634500F0AD8090
:10BB7000F4181EF80300227F824203F1010501F14F
:10BB8000050210D0B718721820771C0A82F808B284
:10BB900082F80AA282F80B3282F80C9282F80942EB
:10BBA000063187F80802ABB24345DED30023A6F87E
:10BBB000603421B9474A00231370BDE8F88F484E1E
:10BBC000484A7068484B90421B887AD002F58062E0
:10BBD000904276D00288B76822F04002B3F5807FA9
:10BBE0004FEA0242A8BF4FF48073120C0280022B6E
:10BBF0000288B8BF0223002B93FAA3F3B3FA83F3AE
:10BC000092B208BF4FF0FF33013B22F0380242EA04
:10BC1000C3039BB20380038843F04003038017B142
:10BC20003B68BA885A83DFF8CCC0838901394FF466
:10BC30007A734FF6FF74BCF1000F44D09CF80050AB
:10BC40000CF1010C01E0A34236D00289013B9207BE
:10BC50009BB2F8D5ABB283814FF47A7302E0ABB2FA
:10BC6000A34229D00289D20703F1FF35F7D5013964
:10BC700082894A1CDFD117B13B68BA881A83194BF5
:10BC8000984225D0194A904214BF08220022038806
:10BC900023F040031B041B0C038003889BB223F09A
:10BCA00038031343038003880A4A43F040030380A8
:10BCB00000231370BDE8F88F1CF008FAD6E90107DD
:10BCC000D9E75B0886E7FF25BFE7A6F8603470E791
:10BCD0000022DCE70D420020002800201C0000208C
:10BCE000209400200038004074200020003C0040D8
:10BCF00078300020082A00200E4B10B41C888CB12C
:10BD00000D4B0E4A1878117F88420FD11C441C320B
:10BD1000013305E013F8011B12F8010F884205D129
:10BD2000A342F7D101205DF8044B704700205DF875
:10BD3000044B70471C0000207830002000280020B1
:10BD40001378C3B130B41E240B4D14FB01012944F8
:10BD5000801A84181D2C07DC01F8013B12F8013F02
:10BD6000002BF6D130BC704712F8013F0131002B97
:10BD7000EFD130BC704770477830002070B54E4C22
:10BD80004E4D63684E4AC1F1030141EA8006AB4261
:10BD90001288F6B200F08B804A498B4200F087800F
:10BDA0001988A06821F04001B2F5807F4FEA014177
:10BDB000A8BF4FF48072090C1980022A1988B8BFF5
:10BDC0000222002A92FAA2F2B2FA82F289B208BFE3
:10BDD0004FF0FF32013A21F0380141EAC20292B23B
:10BDE0001A801A8842F040021A8010B102688188D5
:10BDF0005183B6B2102540F2E93201E0002A4CD05E
:10BE00001989013A11F0020F92B2F7D0AAB29A81C1
:10BE100040F2E93201E0002A3FD01989013A11F0DD
:10BE2000010F92B2F7D09A8940F2E93201E0002A7C
:10BE300038D01989013A11F0020F92B2F7D09E81E1
:10BE400040F2E93201E0002A2CD01989013A11F0C0
:10BE5000010F92B2F7D09A890135202DCBD1A2687B
:10BE600012B1116892880A83144A934221D015496D
:10BE70008B4214BF082100211A8822F040021204CC
:10BE8000120C1A801A8892B222F038020A431A80E1
:10BE90001A8842F040021A8070BD18461CF016F94C
:10BEA0006368C1E718461CF011F96368D4E75208CB
:10BEB00076E70021E0E700BF209400200038004032
:10BEC00074200020003C004038B54D4BDD7E00283A
:10BED00040F0888005F0F7054A4C4B4A60684B49B2
:10BEE000DD7690420B887BD002F58062904277D05D
:10BEF0000288A16822F04002B3F5807F4FEA024237
:10BF0000A8BF4FF48073120C0280022B0288B8BFC6
:10BF10000223002B93FAA3F3B3FA83F392B208BF80
:10BF20004FF0FF33013B22F0380242EAC3039BB2D9
:10BF30000380038843F04003038011B10B688A88B3
:10BF40005A8340F2E93301E0002B54D00289013BCF
:10BF500012F0020F9BB2F7D00423838140F2E93341
:10BF600001E0002B47D00289013B12F0010F9BB288
:10BF7000F7D0838940F2E93301E0002B37D0028902
:10BF8000013B12F0020F9BB2F7D0ADB2858140F2B7
:10BF9000E93300E05BB30289013B12F0010F9BB271
:10BFA000F8D08389A36813B11A689B881383164B52
:10BFB00098421AD0164A904214BF082200220388E1
:10BFC00023F040031B041B0C038003889BB223F067
:10BFD000380313430380038843F04003038038BDD4
:10BFE0005B0885E745F0080576E70022E7E71CF0E7
:10BFF0006DF86068D6E71CF069F86068BAE700BFC2
:10C0000000280020209400200038004074200020E8
:10C01000003C0040134B144A196C70B541F080513C
:10C02000124D19640126FF24CA2053212E60546248
:10C03000506251625B6FDB000DD401242046002169
:10C04000013436F0BDFC062CF8D109490020BDE8CA
:10C05000704036F0B5BC002036F0A2FC044B98428C
:10C06000EBD170BD003802400028004020000E4295
:10C0700031666542F0B5012085B036F091FC7E4B0B
:10C080009A6822F003029A609A6812F00C0FFBD1B2
:10C090001A687949B0B942F001021A6041F2883356
:10C0A00002E0013B00F084800A689507F9D5734CE3
:10C0B000002108220223C4F87814C4F86424C4F8C8
:10C0C00068341FE042F480321A6041F2883301E0A4
:10C0D000013B6DD00A689403FAD5684C684A694BF5
:10C0E000B0FBF3F3B0FBF2F0B3EB400F18BF184610
:10C0F0004FF48002B3FBF0F3C4F86404C4F868346E
:10C10000C4F87824022036F04BFC02280FD85E4B8E
:10C11000D4F8681403EBC0008588C2884388C4F84B
:10C120007054B3FBF1F3C4F87424C4F86C34524B6C
:10C1300056491A6C42F080521A640A6842F440422E
:10C140000A609A689A609A689A609A6842F4805283
:10C150009A60D4F86424D4F87864D4F86C54D4F891
:10C160007014D4F87404324342EA8512490842EA52
:10C170000062013942EA01425A601A6842F0807254
:10C180001A601A689201FCD541493B4A40F202709C
:10C190000860996821F003019960996841F00201F3
:10C1A0009960936803F00C03082BFAD1FDF7A2FA0B
:10C1B000384D314B384AEA603849586F384A086080
:10C1C000AA605E6B374C384F384A394826F08006F3
:10C1D0005E635E6F46F080765E67196B0C431C638E
:10C1E000596B5963196C39431964596C04AC0A438F
:10C1F00048F2FF715A6444F8101D012300262146BD
:10C200008DF807304FF6FF778DF804608DF80560E4
:10C210008DF8066036F0F6FB21462648009736F08A
:10C22000F1FB21462448009736F0ECFB21462348D9
:10C2300036F0E8FB2146224836F0E4FB204636F093
:10C24000E5FC204B204C1B68009A20482049A4FBA9
:10C2500003439B09A0FB0202013B920CB3F1807FD8
:10C260000A6007D21B4AF0200721536085F823009B
:10C270009660116005B0F0BD003802400028002033
:10C2800080841E0040420F00E0D40408007000408B
:10C29000003C024000ED00E00005FA0580B80020F7
:10C2A000000000081F906700FFC9FE36335F0700DB
:10C2B000000002400004024000080240000C02405E
:10C2C000001002409CAB0020D34D621083DE1B4364
:10C2D0008096002010E000E010B5032036F060FBEF
:10C2E00000210446032036F06BFB054B9C4206D12F
:10C2F000044B1A6882F308885B689847FEE710BD14
:10C30000EFBEADDE0000FF1F08B50349032036F085
:10C3100057FB72B63EF028FDEFBEADDEF8B50468FF
:10C32000C4F30D0405460E4604B32F6836F058FBDF
:10C33000092840F08980464C236923F44073236127
:10C34000236943F400732361236943F001032361EC
:10C350003E6036F045FB2369092823F00103236181
:10C3600072D12B6804332B60002036E0394B3A4AF7
:10C3700093422CD902F58042934227D902F580429C
:10C3800093422BD902F58042934229D902F580329B
:10C39000934227D902F50032934225D902F50032A3
:10C3A000934223D902F50032934221D902F500329B
:10C3B00093421FD902F5802293421DD9B3F1016F38
:10C3C0001CD3052039F096FEFFF79EFF082436F0B7
:10C3D00007FB092814D04FF0FF30F8BD1024F6E712
:10C3E0001824F4E72024F2E72824F0E73024EEE7CD
:10C3F0003824ECE74024EAE74824E8E75824E6E755
:10C40000134F3B6923F440733B613B6943F4007372
:10C410003B613B6923F0F8033B613B6943F0020356
:10C420001C433C613B6943F480333B6136F0D8FAEE
:10C430003B6923F002033B613B69092823F0F803C1
:10C440003B613FF472AFC6E76FF00100C5E700BF84
:10C45000003C024000400008FF3F0008F8B50446D9
:10C460000D468E180027B542206900D1F8BDE3685B
:10C47000591CE160234415F8012B1A720429F2D1EA
:10C4800018B9A1682046FFF749FFC4E90370EAE73D
:10C49000074A002302E00133102B07D05168814284
:10C4A00002F12002F7D1581CC0B27047002070473B
:10C4B000B42000200138F0B540013C4CDFF820C129
:10C4C00025583B4FDCF83060BD420CBF4FF40015DF
:10C4D0004FF4800527182E437D68CCF83060354E28
:10C4E000F960B54283B07B6151D0334B9D424ED051
:10C4F000A3F57A739D4236D003F580639D4232D016
:10C50000A3F57A739D4246D003F580639D4242D0E5
:10C51000A3F57A739D4240D003F580639D423CD0E1
:10C52000A3F57A739D4234D003F580639D4230D0E9
:10C53000A3F57A739D4232D003F580639D422ED0DD
:10C54000A3F57A739D422CD003F580639D4228D0D9
:10C55000A3F57A739D4226D01849194B8D420CBF22
:10C560001D46002500E0174D04449209667CE561F4
:10C570000021012301A88DF804608DF805208DF8B5
:10C5800006108DF8073039F09FF803B0F0BD0E4D5E
:10C59000EAE70E4DE8E70E4DE6E70E4DE4E70E4DF7
:10C5A000E2E70E4DE0E7064DDEE700BFB4200020D5
:10C5B000006002401060024010640240B864024013
:10C5C00000800028008800102080001020800020BB
:10C5D00000802010008000180088002000802020AB
:10C5E000003802400138F0B444010948094D0359AC
:10C5F000094F2E6B2044BB420CBF4FF400134FF485
:10C60000800333432B6301764276F0BC704700BF52
:10C61000B420002000380240006002402DE9F04FB5
:10C62000534C54F8204083B0002C00F09C80656E81
:10C63000002D00F09A809846174604F16A034D4A8F
:10C64000064628692260636104F1EA028023A26140
:10C65000E3604FF480726B68A1602261E365A246DB
:10C6600068B1FFF715FF721CD2B20C21FFF7BAFFB9
:10C67000E36DA9682A69A26304332164A365E868AD
:10C68000A0B1FFF705FF721C8146D2B20B21FFF764
:10C69000A9FF2346EA7F38494846FFF70BFFD5E953
:10C6A0000212E36D616404336365E26394F8690028
:10C6B0001AF0DCFA814694F868001AF0D7FA83463B
:10C6C000287F00284CD118F0080F36D1BA070DD5B5
:10C6D000B9F1000F0AD00B22731C89F8062089F8E3
:10C6E000073048466A7F22211AF088FBFB0715D4E1
:10C6F000236C7BB995F82020A97F8DF8063001A81E
:10C70000930901228DF805308DF804108DF807206B
:10C7100038F0DAFF504603B0BDE8F08FBBF1000FF0
:10C72000E6D0701C0C238BF807008BF806305846B7
:10C730006A7F22211AF062FBDAE7B9F1000F05D017
:10C74000701C0B2389F8070089F8063018F0100FC9
:10C75000484614BF022112216A7F1AF04FFBC7E737
:10C7600038F036FFAFE7A246D4E7AA46D2E700BFCB
:10C77000B075002010C50408ED8800080348D0F803
:10C78000EC3113B100F5F07018477047B420002069
:10C790000348D0F8CC3113B100F5E070184770476A
:10C7A000B42000200348D0F8AC3113B100F5D070AC
:10C7B00018477047B42000200348D0F88C3113B1DB
:10C7C00000F5C07018477047B42000200348D0F827
:10C7D0006C3113B100F5B07018477047B4200020D9
:10C7E0000348D0F84C3113B100F5A07018477047DA
:10C7F000B42000200348D0F82C3113B100F590701C
:10C8000018477047B42000200348D0F80C3113B10A
:10C8100000F5807018477047B42000200348D0F816
:10C82000EC300BB1E0301847704700BFB420002057
:10C830000348D0F8CC300BB1C0301847704700BF68
:10C84000B42000200348D0F8AC300BB1A03018471A
:10C85000704700BFB42000200348D0F88C300BB1E3
:10C8600080301847704700BFB42000200248C36ED4
:10C870000BB1603018477047B42000200248C36CE9
:10C880000BB1403018477047B42000200248C36AFB
:10C890000BB1203018477047B42000200248C3680D
:10C8A00003B11847704700BFB4200020F8B5040159
:10C8B000634D2B592F19002B6CD00646387A38F06F
:10C8C00087FE3B7A03F01F015B090122032B02FA6A
:10C8D00001F263D0042B6BD0022B64D02B190136EC
:10C8E00018791AF0C3F9F6B2074610B11223C671CF
:10C8F00083712B1958791AF0B9F910B11323C67145
:10C9000083712B1998791AF0B1F910B11423C671FB
:10C9100083712E190A21F27938461AF06FFA70796C
:10C920001AF0A4F9F2790A211AF068FAB0791AF02B
:10C930009DF9F2790A211AF061FA2B59414A934282
:10C940003BD0414A934243D0404A93424BD0404A65
:10C9500093425ED03F4A934266D03F4A93424DD0C5
:10C960002B191B7BBBB9012002222B59198801F41A
:10C97000415141F445710A4302431A809A8B22F4D3
:10C9800000621204120C07219A8319821A8842F05D
:10C9900040021A80F8BD00200246E6E72F4B196AD4
:10C9A0000A431A629AE72D4B596A0A435A6295E77D
:10C9B0002A4B19690A431A6190E702F584324FF451
:10C9C0008050536A43F48053536236F061F8C7E7EE
:10C9D00002F500324FF48040136A43F4804313623F
:10C9E00036F05EF8BCE702F5FE324FF40040136A01
:10C9F00043F40043136236F053F8B1E702F56442A2
:10CA00004FF40010536A43F40013536236F040F8B9
:10CA1000A6E702F582324FF40050536A43F4005304
:10CA2000536236F035F89BE702F568424FF4801008
:10CA3000536A43F48013536236F02AF890E700BF3C
:10CA4000309400200030014000380040003C00409D
:10CA500000340140005001400054014000380240C1
:10CA6000431C00F014812DE9F04F4FEAC00808EB99
:10CA700000039B00DFF8009359F803A087B009EB8F
:10CA80000304BAF1000F00F0FF80143309EB030137
:10CA90000022DAF8047049F80320C1E90122CA60D3
:10CAA000D4E9025B034601330190DBB2002D00F0B4
:10CAB00008811522EB71AA719AF81800BBF1000FDA
:10CAC00000F0E68016228BF806208BF8073038F04D
:10CAD0007FFDBB8823F440731B041B0CBB802846DE
:10CAE0001AF0E2FA58461AF0DFFA112128461AF035
:10CAF00023F8112158461AF01FF80926332405E0BF
:10CB0000013C4FF00A0006D016F086FD28461BF0C7
:10CB100085F90028F4D028461AF0C0FA052016F04E
:10CB20007BFD28461AF0C0FA052016F075FD013E7F
:10CB3000E4D128461AF0B2FA052016F06DFD5846E9
:10CB40001AF0ACFA052016F067FD28461AF0ACFA88
:10CB5000052016F061FD58461AF0A6FA019B08EB75
:10CB6000030409EB84042846E37C227C002B0CBFE1
:10CB7000122132211AF042F9E37C627C002B0CBFB7
:10CB80001221322158461AF039F9714B9F4200F0B8
:10CB9000B180704B9F4200F0C1806F4B9F4200F00C
:10CBA000B380BB886D4A6E4C23F440731B041B0C8E
:10CBB000BB80019B98443B8809EB880943F0010343
:10CBC00099F812103B80BD8802A8002918BF1446AE
:10CBD00036F01CF8049A6348B2FBF4F325F03F05E5
:10CBE000A0FB02122D04900C2D0C0543BD8039884A
:10CBF0005D4C4FF496729BB202FB00F2002BA4FB3B
:10CC0000020221F0010108BF01239209090443F443
:10CC100000430132090C39803A84BB833A88534B74
:10CC200042F001023A803A88134043F480634FF4A3
:10CC300080423B803A813B8823F080031B041B0C1D
:10CC40003B809AF81A308DF80830002402A801259C
:10CC50008DF809408DF80A408DF80B5038F034FDFE
:10CC60009DF80B209AF819308DF808308DF809409E
:10CC70008DF80A40FAB95A09203203F01F033C49E3
:10CC800005FA03F341F8223007B0BDE8F08F704792
:10CC900038F09EFCBB8823F440731B041B0CBB8044
:10CCA00028461AF001FA58461AF0FEF911212846D2
:10CCB00019F042FF21E702A838F006FD07B0BDE8F1
:10CCC000F08F9AF81800BBF1000F31D016228BF8C4
:10CCD00007308BF8062038F07BFCBB8823F44073C8
:10CCE0001B041B0C2846BB801AF0DEF958461AF0CC
:10CCF000DBF9FEE61F4A136A43F4001313624FF494
:10CD0000001035F0CDFE4CE71A4A136A43F40003D5
:10CD100013624FF4000035F0C3FE42E7154A136A70
:10CD200043F4800313624FF4800035F0B9FE38E716
:10CD300038F04EFCBB8823F440731B041B0C584690
:10CD4000BB801AF0B1F958461AF0AEF9D5E600BF2B
:10CD50000054004000580040005C0040009F240048
:10CD6000804F120083DE1B43D34D6210F5FBFFFFA3
:10CD700000E100E000380240E07500202DE9F041BC
:10CD80000678012E82B0054655D0022E59D1806812
:10CD900041F0800110B1046880886083686840F2C7
:10CDA000E93402E0002C00F098800689013C16F07E
:10CDB000020FA4B2F6D089B2818140F2E93102E0DB
:10CDC000002900F08A800489013914F0010F89B22A
:10CDD000F6D0818981894FF0000C4FF47A714FF6BB
:10CDE000FF764FF0FF0E03E0013989B2B1422CD03B
:10CDF0000489A707F8D5A0F80CE04FF47A7102E097
:10CE0000B9B2B14221D00489E40701F1FF37F7D567
:10CE10008489A4B20AB1147001320CF1010C63458B
:10CE2000E6D1AB68002B56D01A689B88138301208B
:10CE300002B0BDE8F08190F90400441C01D0032841
:10CE400006DD002002B0BDE8F0811BF03FF9E8E705
:10CE50004FEAC00EDFF8BCC00EEB00070CEB8707F3
:10CE60007C68002C48D06D793A626D004FF0000864
:10CE7000EDB2BD75F97587F81980BE763B767E7583
:10CE800087F81480A388FA61990512D42388DA05FB
:10CE90000BD44FF4805501E0013D2FD023889B0532
:10CEA000FAD4238843F480732380A38843F4407327
:10CEB000A38086440CEB8E024FF4805401E0013CC9
:10CEC00013D0537D002BFAD10CEB8E0E9EF814007C
:10CED00080F00100B6E70120B4E7CDE900231BF0A4
:10CEE000F5F86868DDE9002374E7094A138801331F
:10CEF0009BB21380FFF7B4FD2046A3E7044A1388D2
:10CF000001339BB21380FFF7ABFD28469AE700BFC1
:10CF1000FE770020E075002007B5032301AA002159
:10CF2000FFF72CFF9DF805309DF804001B0243EA33
:10CF300000439DF80600184303B05DF804FB08B5F4
:10CF4000FFF7EAFF014B586008BD00BF0028002032
:10CF500008B5FFF7E1FF014B186008BD002800206D
:10CF600007B506236A46F721FFF708FF9DF8013051
:10CF70009DF800100B4A1B0143EA01339DF8021093
:10CF800043EA1113D3609DF804309DF803101B0190
:10CF900043EA01339DF8051043EA1113936003B08F
:10CFA0005DF804FB0028002007B5032301AAF62141
:10CFB000FFF7E4FE9DF805309DF804201B0243EACC
:10CFC00002439DF806201343054AB2F92020C2F11E
:10CFD0000802D340034A536103B05DF804FB00BF6D
:10CFE000446100200028002007B5022301AAF62191
:10CFF000FFF7C4FE9DF804209DF8053043EA0223A4
:10D00000024A138203B05DF804FB00BF0028002031
:10D0100070B582B00446062310306A464321FFF7FC
:10D02000ADFEC0B19DF804009DF800609DF80110B0
:10D030009DF802509DF803209DF8053041EA062135
:10D0400043EA002342EA0522A4F85010A4F8522033
:10D05000A4F85430012002B070BD00BF2DE9F04F9C
:10D0600090F8613085B00546002B40F004825C4B9F
:10D07000686993F87C3405F11006002B00F0B68047
:10D08000584B984200F0F581574A90420CBF30222D
:10D090003822038823F040031B041B0C0380038801
:10D0A0009BB223F038031A430280038843F0400305
:10D0B000038095F85B30032B00F2908095F85E407A
:10D0C000012C0AD0022C40F0898095F8633003F0DF
:10D0D000FB03022B0CBF00240724AB6913B11A68B1
:10D0E0009B88538340F2E93304E0013B9BB2002B61
:10D0F00000F0538302899107F7D51A23838140F208
:10D10000E93304E0013B9BB2002B00F04683028927
:10D11000D207F7D5838940F2E93304E0013B9BB2A3
:10D12000002B00F0CC8302899707F7D5848140F269
:10D13000E93304E0013B9BB2002B00F0C08302897D
:10D14000D107F7D58389AB6913B11A689B8813831C
:10D15000012016F061FA6B69224A934200F01B83AA
:10D1600021498B4214BF082100211A8822F0400275
:10D170001204120C1A801A8892B222F0380211435B
:10D1800019801A8842F040021A803046062302AA0B
:10D190004321FFF7F3FD002800F0FA829DF80A60B2
:10D1A0009DF80B309DF808409DF809109DF80C0083
:10D1B0009DF80D2043EA06231BB241EA042142EA0E
:10D1C0000022A5F85230A5F85010A5F854205BB203
:10D1D000013300F02C8205B0BDE8F08F00247CE71D
:10D1E0000028002000380040003C0040CE4B984210
:10D1F00000F06383CD4988420CBF80214FF48071D9
:10D200000388CB4CDFF84CA3DFF82CB3C94F23F0D5
:10D2100040031B041B0C03800388002991FAA1F230
:10D22000B2FA82F29BB208BF4FF0FF32013A23F00C
:10D23000380343EAC2039BB20380038843F04003F0
:10D24000038080226B2130461AF05CFF9623DFF8C2
:10D2500008E3DFF808C30093DBF80430C3F30803E6
:10D26000002B40F09E81EFF31183002B40F0998159
:10D270002068BA6823689842FAD1DCF800309A42F4
:10D28000F6D8DAF800804FF47A7101FB08F39B1AA4
:10D29000B3FBF8F301FB00304FF47A78DBF804308D
:10D2A000C3F30803002B40F05B81EFF31183002BE5
:10D2B00040F056812368B96822689342FAD1DCF8BD
:10D2C00000209142F6D8DAF8009008FB09F2521AD1
:10D2D000B2FBF9F208FB03231B1AB3F57A7FDDD307
:10D2E000009B013B0093B7D10322682130461AF01E
:10D2F00009FF904FDFF860E2DFF860C24FF0960B55
:10D300008D4B5B68C3F30803002B40F06D81EFF396
:10D310001183002B40F068812068BA682368984226
:10D32000FAD1DCF800309A42F6D8DAF800804FF4EF
:10D330007A7101FB08F39B1AB3FBF8F301FB003091
:10D340004FF47A787C4B5B68C3F30803002B40F002
:10D35000CA80EFF31183002B40F0C5802368B968C1
:10D3600022689342FAD1DCF800209142F6D8DAF82C
:10D37000009008FB09F2521AB2FBF9F208FB0323F2
:10D380001B1AB3F57A7FDDD3BBF1010BB8D10322B1
:10D390006B2130461AF0B6FE0F2016F03DF9102230
:10D3A0006A2130461AF0AEFE0F2016F035F95A46C3
:10D3B0006C2130461AF0A6FE0F2016F02DF995F8D4
:10D3C0006020192130461AF09DFE0F2016F024F936
:10D3D00018221B2130461AF095FE0F2016F01CF97A
:10D3E00018221C2130461AF08DFE0F2016F014F979
:10D3F0001022372130461AF085FE0F2016F00CF966
:10D400000122382130461AF07DFE0F2016F004F973
:10D410006A69454B9A4200F04682444882420CBFFA
:10D4200002200420138823F040031B041B0C1380EC
:10D430001388002890FAA0F1B1FA81F19BB208BFDD
:10D440004FF0FF31013923F0380343EAC1039BB2A7
:10D450001380138843F040031380012016F0DCF89A
:10D46000364A6869012382F87C342F4B98427FF456
:10D470000BAE30220DE61F09013F032F03F00F030F
:10D4800000F10C0800F211822D4A32F8170040FA20
:10D4900003F2D40740F10982012606FA03F3013BA7
:10D4A00018403DF0A1FA274B274CDB5D184414EBE4
:10D4B000C00400F0FA812023A3710022234BE27103
:10D4C0004146EB60204638F021F9A388B3FA83F394
:10D4D000C3F11F0316FA03F33FF4C9AD1C490A68F0
:10D4E00013430B60C3E5EFF31181102383F312881C
:10D4F000D7F808903B68DB0304D50123CEF8003051
:10D50000D7F808902368DEF80020C9B281F31188AB
:10D51000DAF80010134408FB01F2A2EB0902B2FB97
:10D52000F1F208FB03232BE700380040003C0040E9
:10D530007C96002010E000E000ED00E000280020D4
:10D54000F0FF0408F8FF040878940020DD88000844
:10D55000003C0140809600207896002084960020B0
:10D56000EFF31181102383F31288D7F808903B68FA
:10D57000DB0304D50123CEF80030D7F808902368E8
:10D58000DEF80020C9B281F31188DAF800101344E4
:10D5900008FB01F2A2EB0902B2FBF1F208FB032344
:10D5A0009AE6EFF31182102383F31288D7F80880EC
:10D5B0003B68D90304D50123CEF80030D7F80880A2
:10D5C0002368DEF80000D2B282F31188DAF8001086
:10D5D0004FF47A72184402FB01F3A3EB0803B3FB88
:10D5E000F1F302FB003057E6EFF31183102282F3D0
:10D5F0001288D7F808803A68D20304D50122CEF801
:10D600000020D7F808802068DEF80090DBB283F3B2
:10D610001188DAF800104FF47A72484402FB01F3E3
:10D62000A3EB0803B3FBF1F302FB003088E695F9A6
:10D63000503001337FF4CFAD0A23A24CDFF898A21B
:10D64000A14FA24DA24E019338F0B4FB4FF4FA73F0
:10D65000DFF888E200934FF010087B68C3F30803FB
:10D66000002B40F0DC80EFF31183002B40F0D780DB
:10D670002068AA6823689842FAD133689A42F7D89A
:10D68000DAF800C04FF47A7101FB0CF39B1AB3FB7C
:10D69000FCF301FB00304FF47A7C4FF001097B680A
:10D6A000C3F30803002B40F09B80EFF31183002BA2
:10D6B00040F096802368A96822689342FAD13268C4
:10D6C0009142F7D8DAF800200CFB02FBABEB01012A
:10D6D000B1FBF2F10CFB03131B1AB3F57A7FDED317
:10D6E000009B013B0093B8D1072038F0B7F94FF405
:10D6F0007A73DFF8E8E100934FF010087B68C3F31A
:10D700000803002B40F0AD80EFF31183002B40F0B5
:10D71000A8802068AA6823689842FAD133689A42A0
:10D72000F7D8DAF800C04FF47A7101FB0CF39B1ABA
:10D73000B3FBFCF301FB00304FF47A7C4FF001099E
:10D740007B68C3F3080363BBEFF311834BBB236810
:10D75000A96822689342FAD132689142F7D8DAF880
:10D7600000200CFB02FBABEB0101B1FBF2F10CFB67
:10D7700003131B1AB3F57A7FE2D3009B013B00939E
:10D78000BCD1019B013B01937FF45EAFFEF7BCFD72
:10D79000B5F952301BE50021E7E41AF097FC6869FF
:10D7A000B9E4EFF3118188F31288D5F808B02B683B
:10D7B000DB0344BFCEF80090D5F808B02368DEF84C
:10D7C0000020C9B281F31188DAF8001013440CFB71
:10D7D00001F2A2EB0B02B2FBF1F20CFB0323C8E750
:10D7E000EFF3118188F31288D5F808B02B68DB03BA
:10D7F00044BFCEF80090D5F808B02368DEF80020CA
:10D80000C9B281F31188DAF8001013440CFB01F25D
:10D81000A2EB0B02B2FBF1F20CFB03235CE7EFF38C
:10D82000118388F31288D5F808C02A68D20304D57A
:10D830000122CEF80020D5F808C02068DEF800905C
:10D84000DBB283F31188DAF800104FF47A7248449F
:10D8500002FB01F3A3EB0C03B3FBF1F302FB00307B
:10D8600019E7EFF3118388F31288D5F808C02A6806
:10D87000D20304D50122CEF80020D5F808C02068D4
:10D88000DEF80090DBB283F31188DAF800104FF471
:10D890007A72484402FB01F3A3EB0C03B3FBF1F3F0
:10D8A00002FB003048E70220BCE50A4BEB60414632
:10D8B000002037F02BFFFFF7DABB8021A0E41AF03D
:10D8C00005FC40E47C96002000ED00E010E000E064
:10D8D00084960020DD88000880960020789600203D
:10D8E00070B582B0044606230C306A463B21FFF730
:10D8F00045FAA8B19DF804009DF800609DF801105C
:10D900009DF802509DF803209DF8053041EA06215C
:10D9100043EA002342EA05226183A283E3830120D4
:10D9200002B070BDF0B5C60033189B00244DEA5814
:10D930005468A28A83B092B20192019A2B4412F4E5
:10D94000706F1CBF01221A75019B13F4E06F07462C
:10D950000CD1A38A3E4423F4706305EB86051B04B7
:10D960001B0C0022A3826A7503B0F0BD238BA38831
:10D9700023F480631B041B0CA380019B9B05E8D44C
:10D9800023889805E5D42388D9050DD52388DA05A1
:10D99000FCD4238843F40073238023889B05FCD4A4
:10D9A0003846FFF75DF8D4E7238843F400732380FB
:10D9B000A38823F440731B041B0CA380C9E700BF9A
:10D9C000E0750020F0B583B0441C8DF8073001D01D
:10D9D000032802DD002003B0F0BDC700274E3B182E
:10D9E00006EB83035C68002CF4D04900C9B299753A
:10D9F00001250021DA755D7699761D765D751975BC
:10DA0000A1880DF107028905C3E9072212D42388F2
:10DA1000DA050BD44FF4805501E0013D25D0238871
:10DA20009B05FAD4238843F480732380A38843F4AE
:10DA30004073A380074406EB87024FF4805401E053
:10DA4000013C09D0537D002BFAD106EB8707387DC6
:10DA500080F0010003B0F0BD094A138801339BB286
:10DA60001380FEF7FDFF2046B5E7054A1388013312
:10DA70009BB21380FEF7F4FF2846ACE7E075002068
:10DA8000FE7700200378012B47D0022B43D1836817
:10DA90002DE9F04101F07F0113B11C689B8863837D
:10DAA00005461746406840F2E93401E0002C3FD0BB
:10DAB0000689013C16F0020FA4B2F7D089B2818129
:10DAC00040F2E93101E0002932D00389013913F035
:10DAD000010F89B2F7D0838940F2E93100E021B328
:10DAE0000489013914F0020F89B2F8D0BFB28781DE
:10DAF00040F2E93300E0C3B10289013B12F0010FAB
:10DB00009BB2F8D08389AB686BB11A689B8813838A
:10DB10000120BDE8F0810020704713460A46417994
:10DB200090F904004EE70120F3E71AF0CFFAEAE794
:10DB30001AF0CCFA6868CFE701224821A2E7012257
:10DB400058219FE73122F4219CE7044B93F82020D1
:10DB50009201343202F0FC02F42193E74461002088
:10DB60002E22F4218EE700BF2DE9F04F87B090F808
:10DB700061300290002B40F03B86029B93F85830B6
:10DB8000072B00F02B861823CDE90433029BC64CEB
:10DB9000C64EDFF82483C64F1033184680226B210F
:10DBA0000393FFF76FFF6423DFF810E3C14801938D
:10DBB0004FF01009DEF80430C3F30803002B40F0E7
:10DBC000BC84EFF31183002B40F0B7842568826892
:10DBD00023689D42FAD13B689A42F7D8D6F800C034
:10DBE0004FF47A7101FB0CF39B1AB3FBFCF301FBBE
:10DBF00005354FF47A7C4FF0010ADEF80430C3F3A8
:10DC00000803002B40F07A84EFF31183002B40F0DF
:10DC100075842368816822689342FAD13A689142F8
:10DC2000F7D832680CFB02FBABEB0101B1FBF2F160
:10DC30000CFB03135B1BB3F57A7FDED3019B013B27
:10DC40000193B7D1072268210398DFF86C82984FBF
:10DC5000FFF718FF6423DFF864E2964801934FF062
:10DC60001009DEF80430C3F30803002B40F0A98448
:10DC7000EFF31183002B40F0A484256882682368A9
:10DC80009D42FAD13B689A42F7D8D6F800C04FF4CB
:10DC90007A7101FB0CF39B1AB3FBFCF301FB053516
:10DCA0004FF47A7C4FF0010ADEF80430C3F3080326
:10DCB000002B40F00484EFF31183002B40F0FF832E
:10DCC0002368816822689342FAD13A689142F7D872
:10DCD00032680CFB02FBABEB0101B1FBF2F10CFB78
:10DCE00003135B1BB3F57A7FDED3019B013B0193EA
:10DCF000B7D11A466B210398DFF8BC816C4FFFF750
:10DD0000C1FE6423DFF8B4E16A4801934FF01009C3
:10DD1000DEF80430C3F30803002B40F03084EFF347
:10DD20001183002B40F02B842568826823689D4274
:10DD3000FAD13B689A42F7D8D6F800C04FF47A710E
:10DD400001FB0CF39B1AB3FBFCF301FB05354FF40D
:10DD50007A7C4FF0010ADEF80430C3F30803002B8D
:10DD600040F08F83EFF31183002B40F08A83236808
:10DD7000816822689342FAD13A689142F7D83268B2
:10DD80000CFB02FBABEB0101B1FBF2F10CFB03134B
:10DD90005B1BB3F57A7FDED3019B013B0193B7D1C7
:10DDA00001226B210398DFF81081414FFFF76AFED3
:10DDB0000F23DFF808E13F4801934FF01009DEF828
:10DDC0000430C3F30803002B40F0E484EFF3118325
:10DDD000002B40F0DF842568826823689D42FAD1D9
:10DDE0003B689A42F7D8D6F800C04FF47A7101FB2D
:10DDF0000CF39B1AB3FBFCF301FB05354FF47A7C63
:10DE00004FF0010ADEF80430C3F30803002B40F0A2
:10DE10001A83EFF31183002B40F015832368816888
:10DE200022689342FAD13A689142F7D832680CFBE3
:10DE300002FBABEB0101B1FBF2F10CFB03135B1B2B
:10DE4000B3F57A7FDED3019B013B0193B7D1029AF0
:10DE500092F85B30032B09D992F85F30012B049BB9
:10DE60000CBF43F0010343F0020304939DF810201C
:10DE70000398DFF844800E4F1B21FFF703FE0F23AA
:10DE8000DFF838E00B4801934FF01009DEF804305A
:10DE9000C3F30803002B40F05B84EFF31183002BE6
:10DEA00040F056840CE000BF7C9600208096002055
:10DEB0008496002010E000E07896002000ED00E05D
:10DEC0002568826823689D42FAD13B689A42F7D858
:10DED000D6F800C04FF47A7101FB0CF39B1AB3FB28
:10DEE000FCF301FB05354FF47A7C4FF0010ADEF8B4
:10DEF0000430C3F30803002B40F08782EFF3118353
:10DF0000002B40F082822368816822689342FAD114
:10DF10003A689142F7D832680CFB02FBABEB010187
:10DF2000B1FBF2F10CFB03135B1BB3F57A7FDED37D
:10DF3000019B013B0193A9D1059A0398DFF8208347
:10DF4000C54F1C21FFF79EFD0F23DFF818E3C348E0
:10DF500001934FF01009DEF80430C3F30803002BDF
:10DF600040F0D583EFF31183002B40F0D083256878
:10DF7000826823689D42FAD13B689A42F7D8D6F866
:10DF800000C04FF47A7101FB0CF39B1AB3FBFCF356
:10DF900001FB05354FF47A7C4FF0010ADEF80430BE
:10DFA000C3F30803002B40F01282EFF31183002B20
:10DFB00040F00D822368816822689342FAD13A6862
:10DFC0009142F7D832680CFB02FBABEB0101B1FBCD
:10DFD000F2F10CFB03135B1BB3F57A7FDED3019BDD
:10DFE000013B0193B7D1029A92F85B30032B00F208
:10DFF000F38392F85E20012A0BD0022A40F0EC83D2
:10E00000029B93F8633003F0FB03022B0CBF00224A
:10E0100007221A210398DFF848828F4FFFF732FD5D
:10E020000F23DFF840E28D4801934FF01009DEF82E
:10E030000430C3F30803002B40F02783EFF3118370
:10E04000002B40F022832568826823689D42FAD124
:10E050003B689A42F7D8D6F800C04FF47A7101FBBA
:10E060000CF39B1AB3FBFCF301FB05354FF47A7CF0
:10E070004FF0010ADEF80430C3F30803002B40F030
:10E080008881EFF31183002B40F08381236881683E
:10E0900022689342FAD13A689142F7D832680CFB71
:10E0A00002FBABEB0101B1FBF2F10CFB03135B1BB9
:10E0B000B3F57A7FDED3019B013B0193B7D1029B7D
:10E0C000039893F86020DFF89881634F1921FFF7D8
:10E0D000D9FC6423DFF88CE1604801934FF010090C
:10E0E000DEF80430C3F30803002B40F0EF82EFF3B7
:10E0F0001183002B40F0EA822568826823689D42E4
:10E10000FAD13B689A42F7D8D6F800C04FF47A713A
:10E1100001FB0CF39B1AB3FBFCF301FB05354FF439
:10E120007A7C4FF0010ADEF80430C3F30803002BB9
:10E1300040F01181EFF31183002B40F00C81236834
:10E14000816822689342FAD13A689142F7D83268DE
:10E150000CFB02FBABEB0101B1FBF2F10CFB031377
:10E160005B1BB3F57A7FDED3019B013B0193B7D1F3
:10E17000102237210398DFF8E880374FFFF782FC41
:10E180000F23DFF8E0E0354801934FF01009DEF887
:10E190000430C3F30803002B40F05682EFF31183E1
:10E1A000002B40F051822568826823689D42FAD195
:10E1B0003B689A42F7D8D6F800C04FF47A7101FB59
:10E1C0000CF39B1AB3FBFCF301FB05354FF47A7C8F
:10E1D0004FF0010ADEF80430C3F30803002B40F0CF
:10E1E0009C80EFF31183002B40F0978023688168B7
:10E1F00022689342FAD13A689142F7D832680CFB10
:10E2000002FBABEB0101B1FBF2F10CFB03135B1B57
:10E21000B3F57A7FDED3019B013B0193B7D103981D
:10E22000DFF83C800C4F01223821FFF72BFC0F2335
:10E23000DFF830E0094801934FF01009DEF80430B0
:10E24000C3F30803002B40F0DE81EFF31183002BB2
:10E2500040F0D98108E000BF8496002010E000E083
:10E260007896002000ED00E02568826823689D42D2
:10E27000FAD13B689A42F7D8D6F800C04FF47A71C9
:10E2800001FB0CF39B1AB3FBFCF301FB05354FF4C8
:10E290007A7C4FF0010ADEF80430C3F30803F3B9C7
:10E2A000EFF31183DBB92368816822689342FAD1C6
:10E2B0003A689142F7D832680CFB02FBABEB0101E4
:10E2C000B1FBF2F10CFB03135B1BB3F57A7FE2D3D6
:10E2D000019B013B0193B1D107B0BDE8F08FEFF393
:10E2E000118189F31288D0F808B00368DB0344BFBA
:10E2F000C8F800A0D0F808B02368D8F80020C9B248
:10E3000081F31188316813440CFB01F2A2EB0B027C
:10E31000B2FBF1F20CFB0323D6E7EFF3118189F393
:10E320001288D0F808B00368DB0344BFC8F800A027
:10E33000D0F808B02368D8F80020C9B281F311885A
:10E34000316813440CFB01F2A2EB0B02B2FBF1F2B9
:10E350000CFB03235BE7EFF3118189F31288D0F8FC
:10E3600008B00368DB0344BFC8F800A0D0F808B0C9
:10E370002368D8F80020C9B281F3118831681344AA
:10E380000CFB01F2A2EB0B02B2FBF1F20CFB03233C
:10E39000E6E6EFF3118189F31288D0F808B003683C
:10E3A000DB0344BFC8F800A0D0F808B02368D8F851
:10E3B0000020C9B281F31188316813440CFB01F2CB
:10E3C000A2EB0B02B2FBF1F20CFB03236FE6EFF3BF
:10E3D000118189F31288D0F808B00368DB0344BFC9
:10E3E000C8F800A0D0F808B02368D8F80020C9B257
:10E3F00081F31188316813440CFB01F2A2EB0B028C
:10E40000B2FBF1F20CFB0323E5E5EFF3118189F395
:10E410001288D0F808B00368DB0344BFC8F800A036
:10E42000D0F808B02368D8F80020C9B281F3118869
:10E43000316813440CFB01F2A2EB0B02B2FBF1F2C8
:10E440000CFB032370E5EFF3118189F31288D0F8F8
:10E4500008B00368DB0344BFC8F800A0D0F808B0D8
:10E460002368D8F80020C9B281F3118831681344B9
:10E470000CFB01F2A2EB0B02B2FBF1F20CFB03234B
:10E48000DDE4EFF3118189F31288D0F808B0036856
:10E49000DB0344BFC8F800A0D0F808B02368D8F860
:10E4A0000020C9B281F31188316813440CFB01F2DA
:10E4B000A2EB0B02B2FBF1F20CFB032368E4EFF3D7
:10E4C000118189F31288D0F808B00368DB0344BFD8
:10E4D000C8F800A0D0F808B02368D8F80020C9B266
:10E4E00081F31188316813440CFB01F2A2EB0B029B
:10E4F000B2FBF1F20CFB0323FFF7F3BBEFF3118147
:10E5000089F31288D0F808B00368DB0344BFC8F869
:10E5100000A0D0F808B02368D8F80020C9B281F371
:10E520001188316813440CFB01F2A2EB0B02B2FB21
:10E53000F1F20CFB0323FFF77DBBEFF3118389F3AB
:10E540001288D0F808C00268D20304D50122C8F8A6
:10E550000020D0F808C02568D8F800A0DBB283F30B
:10E56000118831684FF47A72554402FB01F3A3EB32
:10E570000C03B3FBF1F302FB0535FFF73ABBEFF3F6
:10E58000118389F31288D0F808C00268D20304D539
:10E590000122C8F80020D0F808C02568D8F800A0EB
:10E5A000DBB283F3118831684FF47A72554402FB71
:10E5B00001F3A3EB0C03B3FBF1F302FB0535FFF70B
:10E5C000C6BBEFF3118389F31288D0F808C0026844
:10E5D000D20304D50122C8F80020D0F808C025686D
:10E5E000D8F800A0DBB283F3118831684FF47A7257
:10E5F000554402FB01F3A3EB0C03B3FBF1F302FB65
:10E600000535FFF74DBBEFF3118389F31288D0F87E
:10E6100008C00268D20304D50122C8F80020D0F84F
:10E6200008C02568D8F800A0DBB283F311883168F0
:10E630004FF47A72554402FB01F3A3EB0C03B3FBD6
:10E64000F1F302FB053522E6EFF3118389F312881B
:10E65000D0F808C00268D20304D50122C8F800200F
:10E66000D0F808C02568D8F800A0DBB283F3118881
:10E6700031684FF47A72554402FB01F3A3EB0C03AB
:10E68000B3FBF1F302FB0535A0E5EFF3118389F34A
:10E690001288D0F808C00268D20304D50122C8F855
:10E6A0000020D0F808C02568D8F800A0DBB283F3BA
:10E6B000118831684FF47A72554402FB01F3A3EBE1
:10E6C0000C03B3FBF1F302FB0535CFE4EFF3118349
:10E6D00089F31288D0F808C00268D20304D5012259
:10E6E000C8F80020D0F808C02568D8F800A0DBB230
:10E6F00083F3118831684FF47A72554402FB01F3B9
:10E70000A3EB0C03B3FBF1F302FB053507E5EFF3D5
:10E71000118389F31288D0F808C00268D20304D5A7
:10E720000122C8F80020D0F808C02568D8F800A059
:10E73000DBB283F3118831684FF47A72554402FBDF
:10E7400001F3A3EB0C03B3FBF1F302FB053521E46A
:10E75000EFF3118389F31288D0F808C00268D2035E
:10E7600004D50122C8F80020D0F808C02568D8F8E0
:10E7700000A0DBB283F3118831684FF47A725544FC
:10E7800002FB01F3A3EB0C03B3FBF1F302FB053532
:10E79000FFF7A9BBEFF3118389F31288D0F808C003
:10E7A0000268D20304D50122C8F80020D0F808C0BE
:10E7B0002568D8F800A0DBB283F3118831684FF4E4
:10E7C0007A72554402FB01F3A3EB0C03B3FBF1F3A4
:10E7D00002FB0535FFF712BB019A1AE4029B93F87E
:10E7E0005D30002B3BD11023CDE90433FFF7CEB9C8
:10E7F0001E09013E032E03F00F0300F10C0734D86D
:10E800001E4A32F8160040FA03F2D4072DD501252E
:10E8100005FA03F3013B18403CF0E6F8184B194C9D
:10E820009B5D184414EBC0041FD00022E27120232A
:10E83000029AA371144BD3603946204636F066FF26
:10E84000A388B3FA83F3C3F11F0315FA03F33FF46C
:10E8500094A90E490A6813430B60FFF78EB9182379
:10E860001021CDE90431FFF791B9029A064BD3602C
:10E870003946002036F04AFFFFF77FB9F0FF040861
:10E88000F8FF040878940020DD880008003C01406F
:10E890002DE9F04F744A436983B09342019000F030
:10E8A000D68072498B420CBF282130211A8822F071
:10E8B00040021204120C1A801A8892B222F0380216
:10E8C000114319801A8842F040021A80012014F086
:10E8D000A3FE019C2046FFF747F9A36913B11A680C
:10E8E0009B885383019B586940F2E93302E0002B77
:10E8F00000F0B4800289013B12F0020F9BB2F6D007
:10E900006A23838140F2E93302E0002B00F0A68005
:10E910000289013B12F0010F9BB2F6D0838940F2CD
:10E92000E93302E0002B00F096800289013B12F0EF
:10E93000020F9BB2F6D01023838140F2E93302E04C
:10E94000002B00F088800289013B12F0010F9BB27E
:10E95000F6D08389019B9B6913B11A689B88138346
:10E960006423434CDFF81491DFF81481414DDFF844
:10E9700014A1414E009314F0FDFD4FF47A774FF04F
:10E98000100C4FF0010ED8F80430C3F30803002B2D
:10E990003ED1EFF31183002B3AD12368A968226896
:10E9A0009342FAD132689142F7D8D9F8002007FB98
:10E9B00002FBABEB0101B1FBF2F107FB03131B1AE6
:10E9C000B3F57A7FDFD3009B013B0093D3D1019B4A
:10E9D0005A69254B9A423CD003F580639A4214BF92
:10E9E00008230023118821F040010904090C11803B
:10E9F000118889B221F038010B431380138801205C
:10EA000043F04003138003B0BDE8F04F14F004BEA0
:10EA1000EFF311818CF31288D5F808B02B68DB0373
:10EA200044BFCAF800E0D5F808B02368DAF800203F
:10EA3000C9B281F31188D9F80010134407FB01F221
:10EA4000A2EB0B02B2FBF1F207FB0323B7E728218D
:10EA50002CE7009BC6E719F039FB7BE719F036FB82
:10EA6000019B58695BE700BF00380040003C004054
:10EA70007C96002010E000E0849600208096002024
:10EA800000ED00E0789600200220FAF767B900BF99
:10EA90000220FEF747BF00BF0120FAF75FB900BFB1
:10EAA0000120FEF73FBF00BF0020FAF757B900BFB3
:10EAB0000020FEF737BF00BF044B187828B1044A86
:10EAC0001268520744BF002018707047B4840020B9
:10EAD0000020014043680B4A23F0407323F4807305
:10EAE00043F48073436083681A4042F002028260FC
:10EAF000C36A0139C9B223F4700343EA0153C36204
:10EB0000704700BFFDF7FFC01149124BD1F88820B4
:10EB100042F4700210B4C1F888201A680E4C00202C
:10EB200042F001021A6098601A6822F0847222F49E
:10EB300080321A605C601A684FF0006422F4802210
:10EB40001A60D8608C605DF8044BFAF7D3BD00BF43
:10EB500000ED00E00038024010300024000000000A
:10EB600030B44FF4167240F2D93340F2C535012467
:10EB70004FF4807102814381002215238581048036
:10EB800041808280837130BC7047054B1B7803F055
:10EB9000070313EAD02314BF01200020704700BFF1
:10EBA00014000020034B93F86930002B0CBF462063
:10EBB00043207047882C0020054B93F869302BB90F
:10EBC0004FF4A4735843642390FBF3F0704700BFE5
:10EBD000882C00200F4B93F88430022B17D00E4A5C
:10EBE0005378127803EB83035B00C01A02EB8202B6
:10EBF000C3EB4203C0EBC00090FBF3F00628A8BFB4
:10EC0000062020EAE070C0F19600C0B2704797205D
:10EC1000704700BF882C0020788F0020034B93F8AA
:10EC20006930002B0CBF0F200C207047882C00206F
:10EC300070B41B4CB4F88630C8B903F00103A3B913
:10EC400094F888508DB1174A02F1F40652F8041B6B
:10EC5000490441BF94F8741104EB8101D1F80C010F
:10EC600046F823000133AB42F0D170BC70475B081B
:10EC7000012B09D90A68A4F8863002F5C332A03204
:10EC800003F001030A60DAE70B6803F5C333A0332E
:10EC900048F20502A4F886200B6070BC704700BFE4
:10ECA000882C0020142D00202DE9F041A8BB2E4A0D
:10ECB00092F8880060B32D4A2D4B92F804C092F967
:10ECC00005E092F90680CCF1FF07ACF17F06FFB2B8
:10ECD000F6B203EB800003F1F402002403E0834268
:10ECE00002F1040214D053F8041B8904F7D5E1B2F1
:10ECF000A1EB0E0181EAE175A5EBE175012D09DDBE
:10ED000008218342D17004F1010402F10402EAD126
:10ED1000BDE8F08179B96146F3E7144B1A79F02A1E
:10ED20000ED802F10F00104A18710B6803F58243E8
:10ED30001A330B60BCE7414514BF39463146E0E762
:10ED4000094A93F9050092F88A5093F906407F2604
:10ED5000A8421E7105DB644264B29C712044587164
:10ED6000E3E70028FADAF6E7882C002014000020F8
:10ED7000142D00202DE9F0412D4EE0B196F800321F
:10ED8000002B52D196F88B20013AD2B2D6F8043239
:10ED9000284C86F8002203EB4303C3EB031384FBE8
:10EDA00003240A682448DB17C3EB6413053390FB84
:10EDB000F3F31A440A6096F8884034B31F49204F91
:10EDC000002301F1F40C1D4602E00133A3421CD0E4
:10EDD00051F8042BC2F303200628F6D13878C00777
:10EDE00015D596F8000296F88B8000EB050E9EFB79
:10EDF000F8F008FB10E00128CCBF0020012058B932
:10EE00000133A34205F10105E2D1BDE8F081E843F9
:10EE100000F001000028F3D0C2F3834206EB820227
:10EE2000D2F80C214CF82320EAE7013BDAB2ADE737
:10EE3000882C00201F85EB5140420F00142D00202C
:10EE4000328F0020F0B54F4C94F80822002858D19A
:10EE5000002A55D04C4BD3ED007AB3EE097AF4EE8C
:10EE6000C77AF1EE10FA7ADCBBEE097AF4EEC77AD3
:10EE7000F1EE10FA4CBF08270027D3ED017AB3EE6C
:10EE8000097AF4EEC77AF1EE10FA6ADD47F001076D
:10EE900094F88850A5B33D48DFF8FCE000F1F40C8D
:10EEA000002218E094F90B62B142ACBF02210021AC
:10EEB00094F90C62B34220DA94F90D62B342D8BFE0
:10EEC00041F008010F421CBFDEF80C304CF8223034
:10EED0000132954214D050F8043BD903F8D594F987
:10EEE0000A6203F00F01B142C3F30313DADC94F9B1
:10EEF0000C62B3424FF00101DEDB41F00401E1E7B7
:10EF0000F0BD94F809320868ABB31F4B204ED3ED27
:10EF1000007A93ED017A1F4DF0EEE77AB0EEC77AF2
:10EF2000F4EEC77AF1EE10FAB8BFF0EE477AFDEED4
:10EF3000E77A82F0010217EE903A193B03EB4303A4
:10EF4000C3EB031386FB0376DB17C3EBE613053332
:10EF500095FBF3F3184484F80822086078E7042747
:10EF60008BE7BBEE097AF4EEC77AF1EE10FA48BFF0
:10EF700047F002078CE700F5433000F5A070086009
:10EF800066E700BF882C0020688F0020142D002029
:10EF9000353AFC4440420F0040C5040870B40B4EA3
:10EFA00096F8884084B106F18C02054606F5C076D5
:10EFB000002352F8040B35EA000004BF086846F845
:10EFC00023000133A342F4D170BC7047882C002089
:10EFD00030B42A4B60B92A48827C42BB93F8753121
:10EFE0002849203301EB83014FF4A06030BCD5E702
:10EFF00093F80E22002A2CD1214893F80F42857CE9
:10F00000A54293BF04240134012283F80F2292BF4A
:10F0100083F80E4283F80F4283F80E220A6802F545
:10F02000C32202F520720A60827C002AD6D0164ADA
:10F0300012689106D2D5154A93F80E1212789207EB
:10F040000CD5A1B993F877310E49203301EB830138
:10F05000CAE7013A83F80E220948DFE70029BDD14B
:10F0600093F876310749203301EB8301BCE793F82D
:10F0700073310449203301EB8301B5E7882C00206C
:10F0800010C40020142D0020AC86002080930020A6
:10F0900010B41C4AA0B91C4C92F810020B6823440F
:10F0A0000B6010B15DF8044B704792F8733117494B
:10F0B0005DF8044B203301EB83014FF440706DE7A2
:10F0C00092F884308BB1012B07D192F81002104CCA
:10F0D00080F0010082F81002E0E792F810020D4C77
:10F0E00080F0010082F81002D8E70B685DF8044B4D
:10F0F00003F5742303F5107301200B6082F81002EE
:10F10000704700BF882C002040420F00142D0020C3
:10F1100020A1070048E801003A4AA0B992F811324C
:10F120006BB192F812128A081341DB070AD501F07D
:10F130000101032A06D8DFE802F04C443C3492F87F
:10F14000143253BB704792F81232013303F00F03AD
:10F1500082F812323BB192F81132086800F5C330E0
:10F16000A0300860DCE7284882F811324079002896
:10F1700040D12648C07818B143F0040382F8113218
:10F1800023480078C0072CD592F813020028E4D059
:10F1900043F0080382F81132DFE71E494FF40030D4
:10F1A000FCE61D4B03F13002002914BF194611463D
:10F1B000F4E71A4BA3F11802002914BF19461146AF
:10F1C000ECE7154B03F10802002914BF194611465C
:10F1D000E4E7114B03F11802002914BF1946114648
:10F1E000DCE70F4800680028CED043F0010382F826
:10F1F0001132C9E792F884000028BAD0022382F8BD
:10F200001132B6E7882C0020788F0020348F002040
:10F21000328F00204CC5040840C5040868C50408A6
:10F220007C93002090F8603043B9426901210720A7
:10F2300082F84430A2F8460082F84810704700BFB8
:10F24000034A0123E021837382F81912184670479C
:10F25000882C00204FF0FF30704700BF4FF0FF3088
:10F26000704700BF704700BF704700BF0020704765
:10F2700000207047F0B5067ADEB1417A134FFF22C5
:10F2800000254FF0200C79B102EB4203C3EBC3031E
:10F29000FC180023072A04D8012BD8B201DD162B55
:10F2A00009DD01338B42F5D101350132B542D2B2CD
:10F2B000E9D10020F0BD023854FA80F090F81BE24A
:10F2C000BEF1200F18BF80F81BC2EAE7882C00208F
:10F2D00010B500248473FFF7CDFF034B012283F8A0
:10F2E0001922204610BD00BF882C0020013AD2B25E
:10F2F00070B402EB42000E4C0239C0EBC000C9B240
:10F30000013B04440DE0072A09D8142904EB010548
:10F3100005D895F81B62864218BF85F81B0201319B
:10F32000C9B213F8010F0028EDD170BC704700BFBF
:10F33000882C0020013AD2B2072A10D80239C9B26B
:10F3400014290CD802EB42020648C2EBC202024466
:10F35000114491F81B229A4218BF81F81B320020F9
:10F36000704700BF882C0020027A407A02FB00F030
:10F37000704700BF027A407A02FB00F0704700BF7E
:10F3800000207047002070474FF0FF30704700BFEB
:10F39000034B93F8ED23027293F8EE3343727047F8
:10F3A000882C002000207047012070470120704702
:10F3B00000207047027A407A02FB00F0704700BFDD
:10F3C000002070470123837318467047012383731D
:10F3D000184670474FF0FF30704700BF704700BFBE
:10F3E000002070470120704700207047027A407A61
:10F3F00002FB00F0704700BF002070474FF0FF3065
:10F40000704700BF00207047012070470020704700
:10F41000027A407A02FB00F0704700BF002070477C
:10F420000020704700207047002070470020704780
:10F4300010B405481E2404FB02110144002081F889
:10F44000F0335DF8044B7047882C0020014B18897D
:10F45000704700BF14000020084B0949D3F8F80595
:10F46000D3F8FC25014022F028020020C3F8F8154B
:10F47000C3F8FC25C3F80006704700BF882C0020A5
:10F480009C2F9FEF00230222027103704370837050
:10F49000C37070477047037913F002031FBF0369FD
:10F4A000D0E9092003F1FF33101A1DBF1840C0B284
:10F4B000181A1846704701717047704703799B0707
:10F4C0000AD5436A8269D154436A01690133B3FBA7
:10F4D000F1F201FB123343627047037913F0010329
:10F4E0001FBFD0E90732C0689B1A00F1FF3014BF7C
:10F4F00018401846704710B5037913F00103014610
:10F500000ED0FFF7EAFF50B10B6A4A69CC68D05CB5
:10F510000133B3FBF4F204FB1233C0B20B6210BD33
:10F520001846FCE790F84B3830B53BB990F84918CD
:10F5300090F84A380124DAB2914200D830BDB0F8D0
:10F54000525804FA03F22A43A0F852280133F2E792
:10F55000D0E90920131A5842584170472DE9F04F5D
:10F56000754C85B094F80436039003F0FF07002B28
:10F5700040F08380B4F80C1602914FF03C09B4F8C7
:10F580000E1694F8082694F8095694F80A36019154
:10F5900004F5C07C49469CF802609CF803E0C6F183
:10F5A000FF06B6B2002E00F0C280C6F1FF060EFBC9
:10F5B00006F6BCF80080B8FBF9FA3612BAF1050F6E
:10F5C0000ED8DFE80AF0035D707F92A1F3B2AEEBD4
:10F5D000060508FB05F5B5FBF1F51D44EDB27246D5
:10F5E000039801280BBF2E02160246EA024646EA9D
:10F5F00005464FF0170E1E4307EB0E0B012000FAD5
:10F600000EFA0198ABEB0E081AEA060F1FFA88F8FB
:10F610008246029804EB880808BF82461EF1FF3E2E
:10F62000C8F810A6EAD21837BFB2B7F5407F0CF180
:10F63000040CB0D1414984F80A362023A1F8C23124
:10F64000012384F8043691F8C431A1F8C07184F81C
:10F65000082684F8095683B1D1F8C83140F22A321D
:10F660005A60D1F8CC2100215162118841F001018A
:10F6700011801A6842F001021A6005B0BDE8F08FEF
:10F68000B8FBF1F201FB12881FFA88F2C2F13C08C4
:10F69000F3B2AEEB060202FB08F2B2FBF1F21A443F
:10F6A000D2B275469CE7B8FBF1F301FB1383F2B2CB
:10F6B0009BB2AEEB06067343B3FBF1F31344DBB22C
:10F6C00075468DE7B8FBF1F501FB15881FFA88F543
:10F6D000C5F13C08F2B2AEEB060505FB08F5B5FB3B
:10F6E000F1F51544EDB273467AE7B8FBF1F201FB90
:10F6F0001282F5B292B2AEEB06067243B2FBF1F2A1
:10F700002A44D2B273466BE7B8FBF1F301FB1388CE
:10F710001FFA88F3C3F13C08F5B2AEEB060303FB16
:10F7200008F3B3FBF1F32B44DBB2724658E77346A0
:10F730007546724654E700BF882C0020803D0020AB
:10F74000034B9A7A0AB901229A720020704700BFCF
:10F7500014000020074BDA7A52B11B7B43B103EB54
:10F76000C203093B044A32F81320044BA3F8D0210A
:10F77000704700BF14000020A4FD0408803D002055
:10F7800008B5174B1B780BB1164AD372164B1B7872
:10F790000BB1144A1373FFF7DDFF144B144A1B78A7
:10F7A000013382F8D231134B1B887BB1192B0FD94F
:10F7B000642B0FD9C82B0FD9B3F5C87F0ED9B3F579
:10F7C000167F03D80423074A01339372002008BD33
:10F7D0000023F8E70123F6E70223F4E70323F2E727
:10F7E000CD85002014000020CE850020C885002093
:10F7F000803D0020CA85002008B5054B1A7B1AB948
:10F8000001221A73002008BDFFF7A4FFFAE700BF2A
:10F810001400002008B5054BDA7A1AB90122DA7211
:10F82000002008BDFFF796FFFAE700BF1400002094
:10F830000A4B93F8D3210A4B5AB10A4A127822B9DB
:10F8400003F11C029A610020704703F1E4029A61FF
:10F85000F9E703F5C2729A61F5E700BF803D002029
:10F86000140000206A910020034BB3F8D421034B0D
:10F870004FF0FF301A807047803D002068910020D3
:10F88000034B1A88034B0020A3F8D421704700BF14
:10F8900068910020803D0020074B93F90030012B38
:10F8A0001FBF064BB3F8D821A3F8D621002008BF0C
:10F8B0004FF0FF30704700BF881F0020803D0020C0
:10F8C00008B5A0F10103B3FA83F302284FEA5313FA
:10F8D00001D0184608BD0F2029F012FB28B9054BAE
:10F8E0001B7803F00103184608BD0F20BDE808404F
:10F8F00029F0B0BB328F002038B50C4C4FF4907219
:10F9000004F5317020213BF0FDFA094B09491B68D1
:10F91000002001252D3384F8EF53C1F8DC31C4F801
:10F92000E403C4F8E80384F8EC0338BD882C002015
:10F930007C960020803D002000228273DCE700BF1F
:10F9400010B50C46A8B9194B194993F8E021236862
:10F950000B44236002B110BD164991F8733101EBDD
:10F96000830101F586714FF48060BDE81040FFF718
:10F9700015BB0FF001FC32280ADD23680B4A03F5A2
:10F98000742303F510730121236082F8E01110BD88
:10F99000064B93F8E021142882F00102C7BF83F8D8
:10F9A000E0210549054983F8E021D0E7803D0020AA
:10F9B00040420F00882C002020A1070048E80100E9
:10F9C0000C4B10B5044600F8011B92FBF3F103FB4E
:10F9D0001123002BB8BF5B420A460749FAF7A8F982
:10F9E000202301300C2802DD0023637310BD235453
:10F9F0000130F7E7809698001D07050810B504460A
:10FA00000846FFF7D9F80146FFF708F90A2203462E
:10FA100091FBF2F220460449FAF78AF923796371DF
:10FA20002E23237110BD00BF2507050810B5044B18
:10FA3000044C1A8804492046FAF77AF9204610BD8A
:10FA400068910020613F00207007050810B5054B44
:10FA50000549B3F8D82103F5F3742046FAF768F99D
:10FA6000204610BD803D002070070508084B93F824
:10FA7000693007EE900A4BB9F8EEE77A9FED057A08
:10FA80009FED050AA7EE870A3BF038BB704700BF21
:10FA9000882C00206766E63F0000004270B50D4CE0
:10FAA000054616460B4602460221D4F8EC0118F032
:10FAB000C3FA2A46084BD4F8EC01142118F0BCFA1A
:10FAC00033462A46D4F8EC011621BDE8704018F000
:10FAD000B3BA00BF803D00205C28050830B424493B
:10FAE000244B91F88120013A9200134430280BBF37
:10FAF00093F8395093F83B5093F8382093F83A2014
:10FB00001D4B31F8100033F9122033F91530B2F5DE
:10FB1000FA6FA8BF4FF4FA62B2F57A7FB8BF4FF41C
:10FB20007A72B3F5FA6F4FF47A71A8BF4FF4FA63A3
:10FB30008B42B8BF0B46C0F34414C2F57A7200F092
:10FB40001F00A3F57A730634C3EBC303C2EBC202F2
:10FB500092FBF1F293FBF1F1014408482244302377
:10FB6000D2B2C9B2D0F8EC0130BC18F05BBA00BF19
:10FB7000882C002040C50408ECC30020803D0020F4
:10FB80002DE9F843174B33F8105005F01F08C5F363
:10FB90004415002605F10309134F0024032E15D147
:10FBA000032C18BF2A1908F10301D7F8EC0107BF8D
:10FBB0002B234A467C23D2B218F034FA0134072CA6
:10FBC000ECD10136072EE7D1BDE8F883032CF5D13F
:10FBD00008EB06012D234A46C9B2D7F8EC0118F00C
:10FBE00021FAEBE7882C0020803D0020012806D078
:10FBF00003D3022807D00020704713F0BBBC044B8E
:10FC0000D3F8F0017047024BD3F8F401704700BFFE
:10FC1000803D002037B504461C4800EB4303B3F891
:10FC20006A5005F00F0039B1611CD8B102288CBFB1
:10FC300020239C2323700C46B2B1C5F30315FFF7B4
:10FC4000D5FF3C23012D1249B0FBF1F191FBF3F2FA
:10FC500003FB12130AD00F49204603B0BDE8304021
:10FC6000FAF766B89B23E5E71546E8E7642542F214
:10FC70001071B0FBF1F0B0FBF5F105FB1100009045
:10FC800005492046FAF754F803B030BD882C00200F
:10FC900040420F002C070508360705082DE9F04FF4
:10FCA000C34C94F818328FB013B90FB0BDE8F08F81
:10FCB000C04E96F80436002BF7D105460C2029F0EB
:10FCC000C9F9E0B196F87B31ABB9BB4C94F8E83197
:10FCD000002BEAD0B94BBA4D1A68002345F823200F
:10FCE0000133202BFAD196F87E01FFF737FC002371
:10FCF00084F8E831D9E796F81432002BE5D0AE4A03
:10FD0000B4F81A02DFF8D8E2DFF8E492DFF8E48210
:10FD10004FF0010C002382F8E8C19A4640FA03F242
:10FD200012F0010F4FEA83010FD15EF82320AA1AC7
:10FD300002EB090747450CFA03FB06D9A14FBA426B
:10FD400088BF41F80E504AEA0B0A0133092BE5D16E
:10FD5000BAF1000FA9D09C4B9C4A1B7813F0010309
:10FD6000039340F04D81039B96F87C0196F8881030
:10FD7000C6F8043232F910300493C4F84032002936
:10FD800000F0D680924B96F87341DFF86CB21A8877
:10FD9000049B904896F8705196F871C1CDF81CA05C
:10FDA00020340BEB8407A3F57A733BF824400D93C2
:10FDB000964600941A46FC7801944FF4B47303FB02
:10FDC00002F3BC78029480FB0374DB17C3EBA4132B
:10FDD00020350CF12002CDE905030BEB85034FEA3A
:10FDE000810908930BEB8203CA4609930BF1F405D2
:10FDF0000024F1465BF80430C3F3032203F4805778
:10FE0000042A1CD8DFE802F02503C7C4B200402151
:10FE1000002219EA010F07D10132042A0FD06E49DE
:10FE200031F822100029F4D1C3F38553002143FA9D
:10FE300001F0C00700F1228101310629F7D1DDE987
:10FE4000003202994FF4B470002F5BD0069F384403
:10FE500058E0C3F3834303F1110000F00F0003F1F6
:10FE60000F0820300BEB800C08F00F0808F1200879
:10FE700020333BF820000A900BEB88010BEB830248
:10FE80009CF802000B909CF8030091F803E091F8B5
:10FE900002C00C9091783BF828803BF82330D27850
:10FEA000002F00F08180049840F2DB57B84200F345
:10FEB000B5800D98059FA1EB0C01A3EB080300FB97
:10FEC00003F300FB01F1A2EB0E020A9300FB02F226
:10FED00087FB0130C91787FB0237C1EB60110A9B12
:10FEE000059880FB03300A9BD217DB17C3EB601326
:10FEF000C2EB6712614472444344C9B2D2B29BB2AE
:10FF00004FF4B4700344354880FB0370C718D8170A
:10FF1000C0EB27204FF4B47707FB10332B5328197D
:10FF20000434A2458170C2707FF464AFDDF81CA078
:10FF30002B4D2C4F2C4B00244FF0010801E057F8BB
:10FF4000043F08FA04F212EA0A0F14BF012000204D
:10FF5000294601349847092C05F10405EFD196F89C
:10FF60007E010FB0BDE8F04FFFF7F8BA0FF004F9CB
:10FF700000B200EB80001D4BC0EB00104000A3FB63
:10FF800000304009002300F5A5701946FF225BE709
:10FF900020F08AFCECE7039B83B3099B9978DA781D
:10FFA0001B884FF4B4704FE74FF4B470AAE700BF5A
:10FFB000803D0020882C00201400002040C504084B
:10FFC000082E00209F860100328F0020ECC3002005
:10FFD000948F0020D34D621088C50408B7600BB61B
:10FFE0009C3F002098C5040831EC00081F85EB51A8
:10FFF0003F4B4C003E4B4C00142D0020089BCDE79E
:020000040801F1
:10000000B2F906002849A0F57A70642303FB00F3D7
:1000100081FB0301DB17C3EBA113A5E60B98471A7D
:100020000C98A0EB020C0A98A0EB03080498A0F22D
:10003000DC5E0EFB08F00A9005980EFB07F70EFB3E
:100040000CFC80FB078EFF1780FB0C08C7EB6E10C3
:100050000B900A9F05984FEAEC7C80FB070EF8177F
:100060000B9FC0EB6E10CCEB681C03443944624418
:10007000C9B2D2B29BB24FF4B47043E70B4B03EB5F
:1000800082024FF4B47092F84A3003EB430306EB5C
:100090004303194491F84C3120330BEB83023BF8B6
:1000A00023309178D278CFE6D34D621040C5040852
:1000B00010B58022044600213AF024FF382204F1D2
:1000C000800000213AF01EFF11482246002350F81C
:1000D0002310C2F8801001330E2B02F10402F6D176
:1000E0001E220C4904F1C0003AF0ACFE0B220A4972
:1000F00004F1E4003AF0A6FE0021032384F8EF1097
:1001000084F8F030102012F0FBFA84F8F10010BDF2
:1001100040C50408BCC50408DCC504082DE9F0434B
:10012000AA4C94F8443285B0A3B1012B03D000202F
:1001300005B0BDE8F08394F8E032082BF7D8DFE88B
:1001400013F0BF00C900D400DD00EF00010122015F
:1001500055016701A0F10A030546222B78D8DFE894
:1001600003F04B77774B7777777777777777777772
:100170007777777777777777777777774377777743
:10018000777712771200924F94F84A3294F84962C6
:100190000020F854002E71D18E4984F84C62384604
:1001A00039F0D2FE002800F04D818B49384639F0F5
:1001B000CBFE002800F046818849384639F0C4FE5D
:1001C000002800F03D828649384639F0BDFE0028FF
:1001D00000F036823846834939F0B6FE002858D1FF
:1001E000032384F84C3254E0002084F8490284F858
:1001F0004A0284F84B029BE794F8B832002B5DD09A
:10020000794901F1140313F8012D5A709942FAD17A
:100210006F4F3B787A78402B85BF373B1B011B0122
:10022000DBB298BF03F0F003402A8CBF373A303A74
:10023000D2B2134494F84B22DBB29A4200F04381CD
:100240003F2384F8BC320020002384F8B8326FE7E3
:1002500094F84A320E2B9EBF5D495A1CC85494F83C
:10026000B83298BF84F84A22002B7FF460AF94F82C
:100270004B02454084F84B52184659E794F84C32EB
:10028000022B00F09081032B00F0E080012B00F0A6
:100290005E832A2D18BF94F84B3206F101064FF009
:1002A00000000CBF01235D4084F8496284F84A02D3
:1002B0000CBF84F8B83284F84B5239E70020C3E70A
:1002C000B5287FF434AF0020012384F8E10284F8DC
:1002D000E0322DE7622815BF0020022384F8E002F7
:1002E00084F8E03208BF002022E7032384F8E2020A
:1002F00084F8E30284F8E032002019E794F8E2324F
:1003000094F8E32284F8E4021844C0B2831804226B
:1003100084F8E20284F8E33284F8E022002007E760
:1003200094F8E23294F8E322A4F8E6021844C0B24A
:100330008318052284F8E20284F8E33284F8E0228C
:100340000020F5E6B4F8E63294F8E22294F8E312DD
:10035000024403EB0020D2B280B25318B0F5AC7F58
:100360004FF0060184F8E22284F8E332A4F8E602B2
:1003700084F8E01240F2A0800123002084F8E132EA
:10038000A4F8E802D4E694F8E222B4F8E83294F84B
:10039000E3120244D2B2B3F5AC7F114484F8E222F6
:1003A00038BFE21803F1010338BF82F8EC02B4F859
:1003B000E62284F8E3129BB29A42A4F8E8323FF6B0
:1003C000B6AE072384F8E0320020B1E6803D00207D
:1003D000B0B800201C0B0508240B05082C0B0508E1
:1003E000340B05083C0B05083C40002094F8E23231
:1003F0000822834284F8E0223FF499AED4F84434D2
:1004000001221344C4F8443484F8E12200208FE62A
:10041000D24B0022A3F1140184F8E02213F8012D3D
:100420005A708B42FAD194F8E332834200F0FC8098
:10043000D4F844343F220133C4F8443484F8BC2255
:10044000002075E6012384F84C3222E7022E00F0EA
:10045000FB80032E05D139F0FBFB94F8496284F848
:100460007102032E7FF615AF331F94F87072C3F339
:10047000870303EB8707FD37FFB2102F3FF609AF65
:10048000F21EA2EB830303F0FF03012B00F01E8298
:10049000042B0BD1002039F0DBFB7B1E2344002210
:1004A00094F8496283F8940283F8A422D4F8B43211
:1004B0000133C4F8B432ECE60023A4F8E832002893
:1004C0003FF47FAF33E6D4F8D43294F84C020133D2
:1004D00021220128C4F8D43284F8BC2200F0BB8069
:1004E00002287FF4EBAE9E4D9E4BB4F860229A81B9
:1004F000D5E90001B4F86422DA81722384F8BC32B1
:1005000050EA01037FF4DAAED4F86C22002A3FF4FB
:10051000D5AED4F8681200293FF4D0AE642301EAC6
:100520000300B2FBF3F703FB172C00EB80000CF584
:10053000FA6C4600ADF804C0B7FBF3F0B1FBF3FC76
:1005400003FB1070BCFBF3F703FB17C78DF8060025
:100550008DF80A7042F21070B2FBF0F2B2FBF3F7C2
:1005600003FB1722B1FBF0F08DF80720B0FBF3F787
:1005700003FB17077C48B1FBF0F101A8B1FBF3F2D4
:1005800003FB12118DF80970ADF80C608DF808109E
:10059000F9F7A0FC754B1B68C61A61F10007C5E9A5
:1005A0000067002050E6731E082B3FF672AE01A2D2
:1005B00052F823F01906010893020108930201087A
:1005C000930201089302010893020108F90501084A
:1005D000E9050108D9050108002039F039FB94F834
:1005E0004962C4F86C0254E6012039F031FB94F8FA
:1005F0004962A4F864024CE6012039F029FB41F27B
:1006000018435B4A94F8496203FB00F3A2FB0323FF
:100610009B09A4F860323CE6022039F019FB94F8FB
:100620004962C4F8680234E6D4F8D43294F8E1227E
:100630000133C4F8D4323AB33E2384F8BC3276E5B1
:10064000022384F84C3224E639F002FB94F8496224
:1006500084F8700205E7474B1B786722990784F8F6
:10066000BC227FF5F1AD3F4BD4F85012D4F85422A0
:1006700094F8585219605A60D4F85C12B4F86222A7
:100680009D7499601A82DFE594F8E4322121023BDF
:1006900084F8BC122E2B3FF64AAD01A151F823F08D
:1006A000950801086D0801082F0101082F010108B4
:1006B000130801082F0101082F0101082F0101086B
:1006C0002F0101082F0101082F0101082F01010846
:1006D0002F0101082F0101082F0101082F01010836
:1006E000D90701082F0101082F0101082F01010876
:1006F0002F0101082F0101082F0101082F01010816
:100700002F0101082F0101082F0101082F01010805
:100710002F0101082F0101082F0101082F010108F5
:100720002F0101082F0101082F0101082F010108E5
:100730002F0101082F0101082F0101082F010108D5
:100740002F0101082F0101082F0101082F010108C5
:100750002F0101082F0101087907010850400020EE
:100760005840002010C4002040420F007C9600201A
:10077000D34D62108093002094F8F02284F8712207
:100780004923102A84F8BC3240F2AD80102284F84C
:1007900071229B4B0021A3F17807A3F16806A3F116
:1007A0004805A3F1580093F808E093F809C007F84A
:1007B00001EB013193F80BE006F801CB914213F8FD
:1007C0000CCF05F801EB00F801CBECD3D4F8B43230
:1007D0000133C4F8B4323EE08A4AD4F80003908171
:1007E00094F86114D4F80433562084F8BC02012034
:1007F00042F2107584F8620493FBF5F3D38100296B
:100800003FF495AC002384F8613484F8623401200D
:100810008EE494F8F7024F2384F8BC32C30703D563
:1008200094F8F632032B69D077490B7823F0020352
:100830000B70764984F86024D1E90023714D94F857
:100840001B73B4F81863AF7413432E8203D100F006
:100850000C000C2854D094F86134002B3FF467ACA2
:1008600094F86234002B3FF462ACCBE794F8F13299
:10087000532284F8BC22DA0703D594F8F032032B14
:1008800038D0614A1378002123F00203137084F8F2
:100890006014E0E75B4BD4F8F0525B4994F86004D5
:1008A0005D60D4F8FC220A2592FBF5F2D4F8F452EC
:1008B0009A6050221D6084F8BC220B78B8B143F0D6
:1008C000020301220B7084F86124C9E707F1FF38A5
:1008D000A044002088F8747239F0BAF994F849629B
:1008E00088F88402E2E5002A7FF453AF6EE703F054
:1008F000FD03E6E7012384F86034ACE7012298E7C2
:100900004348B4F9F462D4F8EC52A6FB0023F7177D
:1009100000FB0733D4F8F0623E4F3F4896FBF7FCEC
:1009200035A7D7E9006712EB050843F10009006815
:1009300018EB0C0249EBEC7312EB060843EB0709CA
:10094000B8EB000269F10003C1E9002383E7B31E9D
:10095000072B3FF69EACDFE803F004433E34292129
:10096000140938F0C7F9C4F8500292E4012039F0B4
:100970006FF900EB80004000C4F85C0294F8496213
:1009800087E4012039F064F900EB800000EB80007F
:100990008300A4F8623294F849627AE4002039F0C6
:1009A00057F994F8496284F8580272E4164A397883
:1009B000137830298CBF43F0020323F00203137035
:1009C00067E43B78572B7FF464ACD4F854325B4235
:1009D000C4F854325DE438F08DF9C4F8540258E498
:1009E0003B78532B7FF455ACD4F850325B42C4F8BB
:1009F00050324EE4AFF30080B0F5F79049000000AC
:100A00006C40002010C4002080930020584000203B
:100A100000840C2440420F007C96002078B310B56F
:100A200082B040F25514AA2200238DF80210ADF8CE
:100A300000408DF803208DF80430694655220DF1F1
:100A400003045340082213F0800F4FEA430318BFFA
:100A500083F03103013ADBB2F5D1A14202D011F8A3
:100A6000012FEEE702688DF80330536AAA228DF851
:100A70000420694605221BB1984702B010BD70479B
:100A800012F088FFF9E700BF2DE9F04190F86030DF
:100A900044699AB07BB94268537884F84430D1787D
:100AA0009378012243EA0123A4F8463084F84820D1
:100AB0001AB0BDE8F081064602E0206812F0B4FFEB
:100AC000206812F0B9FF05460028F6D101466222DF
:100AD0000DF106003AF016FA194A1A49D2F86834AC
:100AE0000968194C92F86424A77803930B44179271
:100AF0000493164A73691648029040F2FF51132F6F
:100B0000ADF80410CDE9052313D894F801806422D0
:100B100002FB084001A908F1010804303AF092F9FB
:100B2000B8F1130FD8BF5FFA88F501377369A77062
:100B300065701868FF211AB0BDE8F0416EE700BF8C
:100B4000803D00207C9600203097002025F2000890
:100B5000F096002090F8603063B910B50278032A4F
:100B60000DD0042A19D0022A1C4C0FD0002384F87F
:100B70006C3410BD194B002283F86C247047174C5D
:100B800084F86D34002384F86C3410BD012384F89C
:100B90006D34002384F86C3410BD4268017E5278B5
:100BA0000E4C0120814202F00F0284F86D0409D03E
:100BB0000229DBD1002AD9D0162084F86E342CF01B
:100BC000D7F8D3E72AB1152084F86E142CF0D0F8AA
:100BD000CCE716202CF0CCF8C8E700BF803D002001
:100BE00008B5044B93F86F3413B901210FF086FE5A
:100BF000002008BD803D002038B50A4839F0AEF924
:100C0000084AC0B20023024420251918CCB2092C8E
:100C100005D9054B0B44002283F8702438BDD55408
:100C20000133F2E7F0410020803D002038B50A484A
:100C300039F094F9084AC0B200230244202519185B
:100C4000CCB2142C05D9054B0B44002283F8702438
:100C500038BDD5540133F2E7F0410020803D00203B
:100C60002DE9F041144C94F8EE5385421BD9064609
:100C700010468846174639F071F904F53173AA1BFE
:100C800005FB086582421D44A8BF02463946284636
:100C900016463AF00FF94444002814BF01230023FC
:100CA00084F8E43301D1BDE8F08132463946284664
:100CB000BDE8F0413AF0C6B8882C002030B583B0CA
:100CC00014460D461A4601A80749F9F731F8074BB3
:100CD00093F8ED33A34204D901AA21462846FFF731
:100CE000BFFF002003B030BD440B0508882C002056
:100CF000074890F8ED03904207D908B50846114619
:100D00001A46FFF7ADFF002008BD0020704700BF66
:100D1000882C0020082A07D808B5084611461A462C
:100D200034F08BFB002008BD00207047F8B5074663
:100D30000026F5B20024E0B220222946013434F026
:100D40007CFB0C2CF7D10136092EF2D11B4D42222F
:100D500001200021441C34F070FB15F8012FE4B28F
:100D60002046002AF5D197F90E302BBB144D1446BE
:100D70004D22E0B2022134F060FB15F8012F01345E
:100D8000002AF6D10F4D2B2202200321441C34F0FF
:100D900054FB15F8012FE4B22046002AF5D10A4D84
:100DA0002B2202200421441C34F047FB15F8012FAC
:100DB000E4B22046002AF5D10020F8BD700B0508EA
:100DC000600B0508540B0508480B050810B50024F6
:100DD0008473FFF7ABFF204610BD00BFF8B508468F
:100DE00017465E1E16F8015F421CD4B239462A46E9
:100DF0002DB1082F01D834F020FB2046F2E7284619
:100E0000F8BD00BF70B50B4C4FF0FF3504F52576EB
:100E10002368DC34184643B193F83430142B04D0E3
:100E200012F006FE854228BF0546A642F0D12846AC
:100E300070BD00BFECA5002010B50B4B0B4993F81B
:100E4000892493F88834097882B00D321E33042443
:100E5000027243728DF8044021B901210DEB0400A8
:100E600036F0C0FB02B010BD803D00207091002024
:100E7000F0B518468BB01C460E46174639F06EF892
:100E80001E2828BF1E2003232146024605460024B3
:100E900002A88DF804308DF805708DF806608DF885
:100EA000074039F0CFFF064B1B7813B120460BB03B
:100EB000F0BD291D01A836F095FB0BB0F0BD00BFB9
:100EC0007091002010B582B000248DF8043001AB81
:100ED0008DF80540FFF7CCFF02B010BD00B5094BFF
:100EE00083B01B7804228DF804201BB1002003B0CE
:100EF0005DF804FB01210DEB020036F073FB03B03B
:100F00005DF804FB7091002000B5094B83B01B789D
:100F100002228DF804201BB1002003B05DF804FB11
:100F2000012101A836F05EFB03B05DF804FB00BFB1
:100F30007091002000B5084B83B01B7801218DF81B
:100F400004101BB1002003B05DF804FB01A836F0CB
:100F500049FB03B05DF804FB7091002000B5074B1E
:100F600083B01B7800208DF804001BB9012101A873
:100F700036F038FB03B05DF804FB00BF7091002031
:100F8000ECE700BF70B50F4C94F88D64054646B988
:100F9000012384F88D34FAF779FCFAF7E3F884F842
:100FA0008D64094B94F8911493F8E92194F89034E6
:100FB00012F0400F14BF10220D220A441E332A7271
:100FC0006B7270BD803D002014000020FAF794BEC3
:100FD00008B5084611461A46FAF7B2FE002008BDC9
:100FE00008B5064B93F88D2412B993F895340BB1DC
:100FF000002008BDFAF79EFD002008BD803D0020BE
:1010000010B5094C94F89204FAF75EFF94F8941422
:1010100094F89304FAF7B2FE4FF4F07220210348DB
:1010200039F070FF002010BD803D00207830002096
:1010300010B50C4658B115F019FE18B10323837191
:101040000023C3712146BDE8104015F08BBF10BDD1
:1010500010B5044601210079FFF7EAFF62792068A4
:101060009108838902228A4023EA0203838110BD0A
:1010700010B5044622210079FFF7DAFF6379226870
:10108000990802238B409BB2D94389B2118291897E
:101090000B43938110BD38B5A0F664040022206C88
:1010A000344D03685A62A1F12903302B31D895F8E9
:1010B00096340133DBB2012B85F896340BD995F8C1
:1010C000973485F89624B4F8522801335208A4F8CE
:1010D000522885F8973495F897240023082AA4F815
:1010E000543815D185F89734B5F8983401339BB24C
:1010F000032BA5F8983408D92379DB0705D5E36AD3
:1011000094F8520853B3216B98470023A4F852383F
:1011100038BD5B396C290ED8B4F8523885F896245E
:101120005B0843F08003A4F8523895F897340133F4
:1011300085F89734CFE794F84D38002BCBD10121B7
:1011400085F89634A5F89834802384F84D18A4F8CF
:10115000523885F8971435F0A5FEBCE7E36962695B
:10116000D054E369E1680133B3FBF1F201FB1233C0
:10117000E361CAE7803D002038B5A0F66404237916
:101180006579DB0722D594F8483803B3D4F84434A2
:101190001A68D36A5B08536294F84C3823B1B4F8E8
:1011A00056380133A4F85638E94301F00101206CA8
:1011B00035F078FE012384F84B38002384F8493851
:1011C00084F84A38A4F8523884F8483838BD94F87E
:1011D0004B38012B04BF94F8493884F84A3820462C
:1011E000FEF7A0F994F84B384BB90123E94384F892
:1011F0004B381940206CBDE8384035F053BE002311
:1012000084F84B3805F00101206CBDE8384035F01A
:1012100049BE73B590F85B38032B05460C462FD1B9
:101220000023204E8DF807309DF8073095F85C2894
:101230009A4201D802B070BD9DF8073006EBC30397
:1012400093F8A0348BB184F0010383B19DF807308B
:1012500006EBC303D3F89C0415F026FF9DF8073076
:101260000133DBB28DF80730DEE72346EDE79DF86A
:10127000073006EBC303D3F89C0415F00FFFEDE72E
:10128000036CC06BDB79DB0748BF81F0010424B13C
:1012900002B0BDE8704015F007BF02B0BDE8704075
:1012A00015F0FCBE803D002070B5A0F5066494F8F2
:1012B0004D3893B1B4F8543801339BB2082BA4F8DD
:1012C00054381CD9002184F84D18A4F85418206C07
:1012D00035F0E8FD94F84D388BB93E4E96F8DC3485
:1012E0001BB901212046FFF794FF94F84C3853BBFB
:1012F000D4E909239A4203D1002386F8DC3470BD77
:1013000096F8DC24022A12D802F1010214BFFF234E
:101310007F2386F8DC24A4F85038082384F84E385C
:10132000012384F84C38206CBDE8704090E65A1CCC
:10133000A169A262CB5C21698A4228BF0022DBB28C
:1013400028BFA262E7E794F94E38C3B394F8501867
:1013500096F8DD5411F0010123D0012D03D80121AD
:101360002046FFF756FFAB1E012B03D80021204675
:10137000FFF74FFF0135EDB2032D86F8DD54BED9DE
:10138000B4F850385B08A4F8503894F84E38013B54
:101390005BB2002284F84E3886F8DD24002BA7D0FB
:1013A000ADE715F0FD0304D101212046FFF731FF21
:1013B000E0E7012BDED12046FFF72BFFDAE7D4E987
:1013C000091291429BD184F84C38206CBDE87040E2
:1013D0004EE600BF803D002010B5A0F5066494F8ED
:1013E0004D381BBB94F84C288ABBD4E909139942A9
:1013F0001CD0591CA069A162C35C2069DBB25B00F0
:1014000043F40073A4F850380A2384F84E380123BB
:1014100084F84C3894F85B38814228BFA262012BD3
:1014200001D0042B02D1206CFFF712FE94F848384B
:10143000002B6FD194F849380133DBB2092B84F8C3
:10144000493827D12046BDE81040FEF76BB894F923
:101450004E387BB1B4F850184B08A4F8503801F05E
:1014600001012046FFF7D5FE94F84E38013B84F881
:101470004E38DBE784F84C38D4E909239A42D5D1B9
:1014800094F85B38012B01D0042BCFD1206CFFF7EF
:10149000EFFDCBE70A2B3DD194F84B382BB9B4F8CC
:1014A000523843F00103A4F852382379D9070AD5FA
:1014B000B4F85208820501D4C30718D4B4F85838D8
:1014C0000133A4F85838012284F8482894F84B28AE
:1014D0000023012A84F849381CD1617984F84B38FB
:1014E000206C01F00101BDE8104035F0DBBCE36A7F
:1014F000C0F3470013B1216B9847E4E7E3696269E1
:10150000D054E369E1680133B3FBF1F201FB12331C
:10151000E361D8E710BD01EB81010D4B70B5A1F17E
:10152000A1051D449C3B06465C1815F8013F7179E6
:1015300096F904004022FCF745FAA542F5D17179ED
:1015400096F9040000234022BDE87040FCF73ABA47
:10155000E7C5040838B505464C1E14F8011F01B94B
:1015600038BD2846FFF7D7FFF7E770B505460C46AC
:101570008E1814F8013B697995F904008022FCF774
:1015800021FA08B1A642F4D170BD07B501EB4103C1
:1015900001EB4101C1F3C301503A10315B008DF8FA
:1015A000042003F00E038DF80610032201A98DF824
:1015B0000530FFF7DAFF03B05DF804FB38B50446E9
:1015C0001D464068FFF7E1FF60682946FFF7A3FF6B
:1015D000002038BD38B504461D464068FFF7D5FFEA
:1015E00060682946FFF7B6FF002038BD0A46002193
:1015F000CBE72DE9F0410F4FDFF84080002407F5DD
:101600008E6638F914300C4922463046F8F790FBC4
:10161000FFF70CFBD7F8E0540134E1B22846FFF79E
:10162000E5FF31462846FFF795FF042CE9D1BDE8D8
:10163000F08100BF803D002045070508649400202C
:101640002DE9F0472D4DDFF8C080D5F8E0442DEDB1
:10165000028B20468CB00121FFF7C8FF20462849A5
:101660009FED288AFFF776FF0024022605F58E6796
:1016700004A9E0B22AF08EFF9DF81830ABB3062C17
:1016800033D0DDED087A099B0B98B8EEE77A41F28A
:10169000883EC8EE077A42F2107C06F101095FFA33
:1016A00089F9FDEEE77A17EE902A00FB02E102FBD2
:1016B00003E2B1FBFCF1B2FBFCF20291CDE90002C6
:1016C000414622463846F8F733FBFFF7AFFAD5F824
:1016D000E0A431465046FFF789FF39465046FFF7F0
:1016E00039FFB9F1080F03D84E4601341A2CBFD187
:1016F0000CB0BDEC028BBDE8F08700BF803D002040
:101700004E07050800247449640705082DE9F341D4
:10171000404C414ED4F8E05401212846FFF766FFC3
:101720003E492846FFF716FF326892076FD53C4DB9
:1017300095ED0B0A39F0E2FC95ED0C0A074639F0FD
:10174000DDFC95ED0D0A804639F0D8FC3B46354A64
:101750003549CDE9008004F58E60F8F7E9FAFFF726
:1017600065FAD4F8E05402212846FFF73FFF2846E7
:1017700004F58E61FFF7EEFE03253368DB0727D5FE
:101780002A4E96ED010A39F0B9FC96ED020A074699
:1017900039F0B4FC96ED030A804639F0AFFC3B46C5
:1017A000234A2149CDE90080A6F17400F8F7C0FA78
:1017B000FFF73CFAD4F8E08429464046FFF716FFCD
:1017C000A6F1740140466F1CFFF7C4FEFFB23D4610
:1017D000184A0A20B2F90030B2F9041091FBF0F176
:1017E0000191B2F9022000920F49134A1348F8F709
:1017F0009FFAFFF71BFAD4F8E04429462046FFF78A
:10180000F5FE0E49204602B0BDE8F041A2E60225F1
:10181000B3E700BF803D0020AC86002074070508B8
:10182000988F00208A0705088E070508644200206B
:101830009D070508D48F0020A1070508F04100206E
:101840007C4B1B6813F0800F2DE9F0417A4C07D1D7
:1018500094F8FC3443F0020384F8FC34BDE8F081D2
:10186000D4F8B422D4F804359A4208D094F8083554
:10187000C4F80425013303F0030384F80835D4F8D1
:10188000E064DFF8F081012200213046FFF77DFEA1
:1018900094F80835694A3046D15CFFF73CFE0122D6
:1018A00002213046FFF771FE0025362718F8051093
:1018B000C1EBC10191FBF7F10629A8BF06216039F0
:1018C000C9B230460135FFF726FE102DEED15C4B34
:1018D0005C4D1B78AA7C5C495C4813F0020F0CBF7E
:1018E0004E235923F8F724FAFFF7A0F9D4F8E0645F
:1018F00002213046FFF77AFE30465449FFF72AFEB0
:1019000029686B68524A514893FBF2F391FBF2F25B
:101910005049F8F70DFAFFF789F9D4F8E06403218C
:101920003046FFF763FE30464849FFF713FEAA89A9
:1019300049494648F8F7FCF9FFF75EF9D4F8E06446
:1019400004213046FFF752FE30464049FFF702FEC1
:10195000EA8942493D48F8F7EBF9FFF74DF9D4F829
:10196000E054042228460A21FFF70FFE2846374993
:10197000FFF7F0FDD4F8D42239493448F8F7D8F904
:10198000FFF73AF9D4F8E05405212846FFF72EFE78
:1019900028462E49FFF7DEFDD4F84834D4F8442415
:1019A00030492A48F8F7C4F9FFF726F9D4F8E0548B
:1019B000052228460A21FFF7E8FD28462349FFF7BC
:1019C000C9FDD4F85034D4F84C2427491F48D21A02
:1019D000F8F7AEF9FFF710F9D4F8E05406212846DD
:1019E000FFF704FE28461949FFF7B4FDD4F8482450
:1019F0001E491648F8F79CF9FFF7FEF8D4F8E044C2
:101A0000062220460A21FFF7C0FD20460F49FFF7B6
:101A1000A1FD1749152201F5DA7039F0B1FAFFF787
:101A2000EBF820460721FFF7E1FD20460749BDE816
:101A3000F0418FE5A8B80020803D0020A5070508EB
:101A40008093002010C40020AA070508F041002060
:101A500080969800BB070508C8070508D007050849
:101A6000D7070508DE070508E7070508EE0705089C
:101A70003C40002014400020F7B5374B374F5C78CE
:101A8000374907F58E6622463046F8F751F9D7F800
:101A9000E05401212846FFF7A9FD31462846FFF70B
:101AA00059FD30493046F8F743F9FFF7BFF8D7F84A
:101AB000E05402212846FFF799FD31462846FFF7FA
:101AC00049FD1A2303FB0474304694F8111594F869
:101AD000103594F80F2500912349F8F729F9FFF7FD
:101AE000A5F8D7F8E05403212846FFF77FFD3146DB
:101AF0002846FFF72FFD94F8171594F8163594F83B
:101B00001525009130461949F8F712F9FFF78EF8BC
:101B1000D7F8E05404212846FFF768FD31462846EF
:101B2000FFF718FD94F8141594F8133594F812255E
:101B3000009130460E49F8F7FBF8FFF777F8D7F831
:101B4000E04405212046FFF751FD3146204603B011
:101B5000BDE8F040FEE400BF90A80020803D0020DA
:101B6000F6070508070805081A0805082D080508DE
:101B7000400805082DE9F3471D4B1E4C1A781E49F5
:101B8000DFF87CA0DFF87C9004F58E60F8F7D0F8E1
:101B9000D4F8E05401212846FFF728FD284604F533
:101BA0008E61FFF7D7FC154B1E68002504F58E6883
:101BB000B27A337A0192727A009249465AF8252015
:101BC0004046F8F7B5F8FFF731F8D4F8E074A91CEF
:101BD000C9B23846FFF70AFD013541463846FFF7DE
:101BE000B9FC032D06F10606E2D102B0BDE8F0878C
:101BF00090A80020803D0020530805088493002011
:101C00008CC804085F08050838B50E4C0E4B0F4A07
:101C10000F4904F58E652846F8F78AF8D4F8E044B1
:101C200001212046FFF7E2FC29462046FFF792FCFF
:101C300020460221FFF7DAFC20460649BDE838407D
:101C400088E400BF803D0020752E05087408050853
:101C50007A0805088308050838B5042208490546AE
:101C6000FFF783FC4FF48064013C00234022697934
:101C700095F90400A4B2FBF7A5FE002CF4D138BD01
:101C800098C8040808B54068FFF7E6FF002008BDC3
:101C900038B5124C124D217BE07A32F02DF8A37A40
:101CA000104A013B32F813300F4A13800F4A128852
:101CB0009A421EBF0E4B02221A7031F06FFBE07A7F
:101CC000217BA37A6970AB70287032F001F8A8808C
:101CD00011F0B8F84FF0FF3038BD00BF14000020FD
:101CE000288F002094FD0408FA900020FC9000202A
:101CF000FE90002008B5084B93F8D21121B90122BB
:101D000083F8D221002008BD4B1E59425941492079
:101D100031F07EFBF6E700BF803D002008B5044BA4
:101D2000B3F8D60140F4004031F098FD002008BD22
:101D3000803D002070B5364B86B01A788DF80C20A7
:101D40005A788DF80D2000269A78CDF80E608DF81F
:101D50000E209A88ADF810201A7ACDF8126003ADE3
:101D60008DF8142095E807006C4603C42280294AA8
:101D70001278022A1C4630D1274B1878274B8DF851
:101D8000000019788DF8011031F0A2FF244BADF856
:101D9000040093F8A835E3B9052031F00BFD214B81
:101DA0000A221E788DF802606946284639F082F8CA
:101DB00058B19DF8003023709DF801306370BDF874
:101DC0000430A670A38011F03DF84FF0FF3006B04C
:101DD00070BD062031F0EEFCE1E7134B1B7863B9D0
:101DE0000D4B18780D4B8DF8000019788DF8011007
:101DF00031F06EFFADF80400D1E7304631F0DAFC87
:101E00000A4B8DF800601B88ADF80430C7E700BFAF
:101E1000288F0020609100206291002063910020B3
:101E2000803D0020669100206A910020689100208A
:101E3000F8B50B4D0B4F06462946F7F78FFF346870
:101E40007460A91E641A402CA8BF40243160224649
:101E500007F2AC5038F0F6FF87F8EC45F8BD00BF4C
:101E600082900020803D0020034B1B6A30EA030370
:101E700014BF012000207047FC86002003885A060A
:101E800006D513F4057F03D00A4A127A072A0ED921
:101E900003F48253B3F5825F01D000207047054BF5
:101EA000187AA0F10700B0FA80F0400970470120CD
:101EB000704700BF54B800202DE9F041B84C94F8A9
:101EC000ED35012B84B000F0EB8094F8F905FDF7B7
:101ED000F7FC94F8FA358342054608D0002870D103
:101EE000B04E30682AF005FD356084F8FA5594F854
:101EF000FB35012B00F08D80D4F8045694F8087659
:101F0000ADB32846FFF7BAFF88B33FB9D4F8F4352C
:101F100023B1A54901220B6084F80826D4F80C5699
:101F200094F81076002D39D02846FFF7A7FFA8B304
:101F30003FB9D4F8F43523B10122C4F8143684F83B
:101F4000102694F81906FDF7BBFC94F81A36834264
:101F5000054609D000286ED1D4F820062AF0C9FC25
:101F6000C4F8205684F81A5604B0BDE8F08194F8FD
:101F70000906FDF7A5FC87420646CFD0002840F0B1
:101F8000A380894D28682AF0B4FC2E60D4F80C5642
:101F900084F8086694F81076002DC5D194F81806D8
:101FA000FDF78EFCB8420646CBD0002840F0B18049
:101FB000D4F814062AF09DFCC4F8146684F8106660
:101FC000BFE77A4B1B68002B91D0794A93F9020046
:101FD0005379002B18BF08254FF0000308BF0025D8
:101FE00003214FF49642CDE90115009208211A46CB
:101FF0002AF094FC6B4B186000283FF478AF33F064
:10200000B7F9012384F8FA3594F8FB35012B7FF4F6
:1020100073AF94F8FC05674DFDF752FC2B6806463C
:10202000002840F09B80002B3FF466AF18462AF052
:1020300060FC2E6060E7604BD4F81C564FF47A7257
:10204000C3F85023002D8FD04FF4805240212846F2
:102050002AF0CAFD0646002886D1554B95F90200A4
:102060001B79002B0CBF0821092103224FF4E13317
:10207000CDE901210093324633464FF480512AF0D6
:102080004DFCC4F8200600283FF46EAF4B494C4A83
:1020900084F8246601230860167084F81A3663E712
:1020A000D4F8F075474D3846FFF7E8FE2E68002853
:1020B00000F08C80002E7FF408AFD4F8F435002BAC
:1020C0003FF403AF2B6000E7002D3FF427AFAB795F
:1020D000002B00F09E803C4A02EB8303D3F85C3374
:1020E000334A95F9020012790093003218BF012299
:1020F00000230221CDE901121A4610212AF00EFC1C
:10210000294B186000283FF409AF012384F80836F2
:1021100004E7002D3FF415AFAB79002B76D02A4AA7
:1021200002EB8303D3F85C33214A95F9020012795C
:102130000093003218BF012202210023CDE90112D1
:102140001A464FF400712AF0E9FBC4F8140600287F
:102150003FF4F7AE012384F81036F2E6002B7FF44B
:10216000CBAED4F80026002A3FF4C6AE104992F94F
:1021700002004A790979002A0CBF002208220029AE
:1021800008BF42F0010203264FF46141CDE901622C
:1021900000911A4620212AF0C1FB2860ACE600BF5E
:1021A000803D00209C93002068930020A093002095
:1021B000FC86002090930020B4220020B8910020DB
:1021C000909100205C8F002040C5040894F8F80529
:1021D000FDF776FB8046F8B1002E7FF476AE002F37
:1021E0003FF473AE114B97F902001B79B3FA83F3F6
:1021F0005B0902214FF41652CDE9011300923346D8
:10220000324604212AF08AFB28605EE64FF46143DF
:102210008AE74FF4964363E7002E3FF456AE30460C
:102220002AF067FBC5F800804FE600BFFC8600205F
:10223000F8B5AF4C94F8ED35002B00F0DD800820A8
:102240002AF0E6FCAB4A1060C0B308212AF0D6FCA5
:102250000026A94984F8F905A848C4F82C6615F0A9
:10226000D1FE41F60A13A548A4F8303607F0E6FE81
:1022700031462A22A24838F045FE48F67C607D258A
:10228000E02331462A22A4F838069E4884F83B36DB
:1022900084F8635638F036FE9B4B84F88F564EF226
:1022A0007B0048F67C21A02283F81A6283F8C3528F
:1022B000A3F81802A4F8641684F8672694F8FB358E
:1022C000002B00F0838010202AF0A2FC1021C4F81B
:1022D00004062AF093FC8D4D8D4B84F8090640F2DC
:1022E0003B113A2019806A7918719F214AF21E40E9
:1022F0009971002198601973002A40F0CC80AB7965
:10230000002B5DD1834F3B68580741BF82490A6863
:1023100042F402720A60990700F1CA801A0748BFA6
:102320007D4A7E4E48BF1368306848BF43F48073CF
:10233000C0F3C01048BF136032F0D6FF002032F067
:10234000B9FF774B18704FF400702AF061FC4FF41E
:102350000071C4F80C062AF051FCD4F8903684F8C9
:102360001806002B14BF0123002384F8943657D19C
:10237000D4F818376B4D00269B1B18BF01234FF470
:10238000805084F81437C4F810672AF041FC4FF4E9
:102390008051C4F81C062AF031FC634B84F81A669D
:1023A000624E634A634984F819069E601D61C5E95F
:1023B0000066D9605A61BDE8F840C2E900117BE5CA
:1023C000554A136843F0040313609BE720202AF06A
:1023D0001FFCC4F8000600283FF475AF20212AF046
:1023E0000DFC554B554A1A6084F8FC0532F0A8FDE7
:1023F000012384F8FB3566E704202AF009FCC4F8C1
:10240000F00500283FF41BAF04212AF0F7FB4C4AEB
:102410004C4984F8F8050123116084F8ED350EE786
:10242000394B49494948092283F8ED23202283F892
:10243000EE23002384F8953684F8963642F2090399
:10244000A4F8A03615F0DEFD404807F0F7FD3A6825
:1024500012F0020234D16B79A3B10120FFF704FD21
:1024600080B1A318022183F8A8160132A31830689E
:10247000042183F8A816030602F1010129D484F887
:10248000AC1675E7AB79002BF0D00620FFF7ECFC1B
:102490000028EBD0E5E7204BA9791A6842F002004A
:1024A000186000293FF42EAF42F036021A6029E787
:1024B00019490A6842F4601242F0C0020A602DE72E
:1024C0004FF46070FFF7D0FC78B1012284F8A826A1
:1024D000C1E74FF45850FFF7C7FC0028CFD063186E
:1024E0000820911C83F8A806C9E70246B3E700BF9D
:1024F000803D0020A0930020DCC80408A8430020F1
:10250000BA430020E6430020882C0020788F00206A
:10251000CCB80020AC86002094930020A8B80020FE
:1025200098930020C0910020E0860020D4910020E4
:102530005493002054920020F88600204F52040843
:1025400020870020511404080CC9040818440020F6
:10255000034A012303FA00F0536F034353677047A4
:10256000882C002008B50146831E00F16202EA2093
:1025700023F8020F9342FBD140F649134B85264BBB
:102580004B60CE230B8100234B670320FFF7E0FF56
:102590000520FFF7DDFF0820FFF7DAFF0920FFF72E
:1025A000D7FF0A20FFF7D4FF0C20FFF7D1FF0D2043
:1025B000FFF7CEFF0220FFF7CBFF0123174A81F878
:1025C0006930B2F86E306FEAD3236FEAC323A2F802
:1025D0006E304FF42063A1F86A3040F60123A1F871
:1025E0006C300F4B4B66142381F86830802381F8E0
:1025F000783042F61403A1F870304FF6FF73A1F85B
:102600007A30A1F87C304623A1F87E3040F20123D5
:10261000A1F8803008BD00BFCD004E00882C0020FE
:102620009808640003280BD8064B074A83F88000FB
:10263000012308B913707047013803FA00F01070D5
:10264000704700BF882C00201400002030B585B0F2
:10265000054601A8F7F71AFC044618B92870204669
:1026600005B030BD044A0123B2F91C2701A9284650
:10267000F7F764FCF3E700BF803D00200F2A03D882
:10268000052803D805290CD900207047062812D048
:102690000728F9D10029F7D10B4B012083F87C21C1
:1026A0007047094B00EB400003EB40000144012060
:1026B00081F84C2170470A29E6D8034B19440120C0
:1026C00081F87021704700BF882C00201B4B2DE93A
:1026D000F04100F120070C4603EB870840F2671633
:1026E00000252046F7F764FF03469E424FF02C0179
:1026F00020461CDB95B1114E06EB87062C2186F88F
:102700008E3038F016FC90B10130F7F751FFFF28FA
:102710000DDC86F88F002846BDE8F081A8F88C30E3
:1027200038F007FC18B1441CFF260125D9E7044BFB
:10273000002043F82700BDE8F08100BF882C00206E
:10274000142D002074492DE9F043002508462E463B
:102750002B460AE0062C03F1010308BF013694045E
:1027600048BF0135202B00F0C38050F8042BC2F382
:102770000324002AEED1694FF6B287F8896087F802
:10278000883087F88A50002B00F0BB8000204FF083
:102790000F0EF04605460446894659F8042BC2F34D
:1027A000031C654502F00F02B8BF6546E045A8BFAF
:1027B000E046904204F10104B8BF10469645A8BF18
:1027C00096469C42E9DB4545C1BF45446C10013447
:1027D00005F1FF35C7BF64B245F34702062207245F
:1027E0007045C8BF704487F80C42C2BF4410013422
:1027F00000F1FF3087F80D22C7BF64B240F34702F3
:1028000006220724464887F80A22A0FB06029208FF
:1028100002EB4202A6EB420212F0FF0F87F80B42D6
:1028200064D0062E324608D9F00706D401E0D50759
:1028300002D45210062AFADCD6B287F88B60002B3D
:1028400066D0D7F88C50C5F305356C074CD40C1FF7
:1028500004EB83040A4603E052F8040F400443D417
:102860009442F9D10126AC070CD40C1F04EB83046D
:102870000A4603E052F8040F870403D49442F9D1C6
:1028800046F002066A090CD10C1F04EB83040A46C9
:1028900003E052F8040F800303D49442F9D146F4C4
:1028A000807628070CD40C1F04EB83040A4603E04F
:1028B00052F8040F070403D4A242F9D146F01006DF
:1028C000EA060BD40A1F02EB830303E051F8042F3E
:1028D000D50303D49942F9D146F00806B6B2114B9C
:1028E000A3F81A62BDE8F0830026BCE70626A4E739
:1028F0000A4FF6B287F8896087F8883087F88A50DF
:1029000044E70622072487F80D2287F80C4279E76E
:1029100040F21B16E3E700BF142D0020882C002096
:10292000ABAAAAAA803D00202DE9F04F714ADFF83A
:10293000D0B1002389B042F820300C4602909A466C
:10294000019319461E4699461F464FF02C0E4FF034
:10295000010823785FFA8AF5A3B173457ED0601C25
:102960000DF1140C00220CF8013B044610F8013B59
:10297000013243B1734572D00A2AF4D1002009B064
:10298000BDE8F08F1A4608AB1A44002302F80C3C4D
:10299000BEF1000FF2D16B1E0134032B03D8DFE828
:1029A00003F05439106405A8F7F702FE0135EDB2C3
:1029B000042D014660D85D440AF1010A95F8FCE354
:1029C000C7E79DF81420002A45D00DF1140E8C465F
:1029D0004320824248494FF0000306D00133072BC1
:1029E00004D011F8010B8242F8D19946542A64D0E0
:1029F0004F2A67D0422A6CD0562A73D0492A57D022
:102A0000572A08BF052354D01EF8012F002ADFD112
:102A1000614620E09DF81430EBB105AA0EE0452B8D
:102A200055D0532B5AD0572B5AD0552B5FD0442B0F
:102A300008BF052305D012F8013F63B14E2BEED13C
:102A4000002308FA03F31F43F5E705A80391F7F7FE
:102A5000AFFD039901900135EDB2ACE7002208AB60
:102A60001A44002302F80C3C95E705A80391F7F7F8
:102A70009FFD0F28039919DD0022019B03F00F032E
:102A800043EA8753134343EA09231C4A43EA0636C1
:102A9000029B0901C9B202EB83090E43C9F88C609D
:102AA000FFF750FE012009B0BDE8F08F8204E4E793
:102AB000042308FA03F31E43A6E7002308FA03F3EE
:102AC0001E43A1E7012308FA03F31E439CE70123F9
:102AD000B7E7022308FA03F31E4395E70223B0E7A2
:102AE0000323AEE7032308FA03F31E438CE7042312
:102AF000A7E700BF142D002061010508882C0020E5
:102B000040C504082DE9F041B84DB94C94B0FFF729
:102B100019FE95F87D71012305F5C26040F6A842C3
:102B2000002184F8183238F0EDF987B9B14B002054
:102B300003F18001FF2218809A70DA700433994201
:102B4000F9D10120FCF70AFD14B0BDE8F081384648
:102B50000FF0FAFDC3680268C4F8CC210646002BCA
:102B6000E4D0384614F082F8C4F8200718B12922BE
:102B700000238271C371327ADFF8A0822A2114F017
:102B80003DF9D4F8CC010FF077FD32F021FDD4F8F7
:102B9000CC3199491A8809689848DFF870C222F048
:102BA000010281424FEA02424FEA124288BF944F2B
:102BB0001A8081BF01F1B77202F55852B2FBF7F7E4
:102BC00007F1FF378CBFBFB2002718887A1C4FF07F
:102BD000030EB1FBF2F26345B2FBF8F291B2B1FB26
:102BE000FEF1A5F80C164FEA410180B2A5F80E16C9
:102BF00011D084498B420ED0B3F1804F0BD0A1F598
:102C000080318B4207D001F580618B4203D001F502
:102C100080618B4202D120F0700080B27A498B42F1
:102C200000F0C48001F580618B4200F0BF8020F489
:102C30004071764889B283421980DA621F8540F07C
:102C4000EF8000221A860022CDE90222012104929F
:102C50009982F379ADF8042098074FF06002009252
:102C600040F19880DB0003F008030422ADF80E3039
:102C7000ADF80420002302937179D4F8CC016A46A0
:102C80000EF084FF7179D4F8CC310C2910D8DFE82C
:102C900001F0070F0F0FA30F0F0F9A0F0F0F9100E7
:102CA0001A8B22F008021204120C42F008021A8356
:102CB000B3F8442042F40042A3F844201A8842F0BA
:102CC00080021A80F27992074CBF042201228A40C6
:102CD000198C92B221EA02011984198C0A431A84D0
:102CE0001A8842F001021A80307D00222921F9F76A
:102CF00079FC60224649307D0023F9F7DBFBF06860
:102D0000C4F8C8012FF0B6FDD4F8C801036823F059
:102D1000010303602FF0AEFD05A82FF06FFDD4F87E
:102D2000CC3172793169059134331A444FF48060A3
:102D300040F22A3306920993364A0B9040234FF40F
:102D40008050002505A9079208934FF480424FF464
:102D500040330C90D4F8C8010D920F930A950E954C
:102D60002FF05DFD7379D4F8CC110C2B98BF2A4A53
:102D7000888998BF32F81330D4F8C82188BF2B4611
:102D800003438B811368012143F01003136084F81F
:102D9000C411CBE65B0003F002034FF48072ADF880
:102DA0000C30ADF80210ADF8102063E71880DA623D
:102DB0001F8548E79A8B22F400621204120C42F439
:102DC00000629A8374E79A8B22F008021204120CB4
:102DD00042F008029A836BE71A8B22F40062120415
:102DE000120C42F400621A8362E700BF882C0020B4
:102DF000803D0020082E00209CAB0020FF6BDC02F1
:102E0000006CDC02000401400010004000000140A2
:102E1000118D0008983200205C00050800350C0078
:102E2000024A93423FF40DAF0DE700BF000401409A
:102E30000E499FED0F0A0A68496807EE902AF8EEDE
:102E4000E77A08B5F0EEE77A0A4B27EE800AC3F876
:102E50002817C3F82427F6F70BFE074A074913780B
:102E600081ED000A43F00103137008BD10C4002077
:102E700050E0EF30803D002080930020FC270020B0
:102E80002DE9F04F804F3B789A0785B040F187805D
:102E90007E4DAA7C042A40F2828013F0010300F0E8
:102EA0008180D5E900CA7A4A7A4E7B4C019294F827
:102EB00044277A487A4F9FED7B7A0132A0FB0210BB
:102EC000800800EB8000101A4FEAEC7E87FB0C12A2
:102ED000754984F84407CEEBA25E01FB0ECC326844
:102EE000D4F8801704EB800B521A00F1050804EBAC
:102EF0008808DBF85007D4F84817CBF850C707EE1E
:102F0000902A87FB0A294FEAEA72D8F85077C2EB79
:102F1000A959081AD4F84C276349F8EE677A01FBDF
:102F200009AAD21B67EE877A6049C8F850A76044A7
:102F30005244B7EE007A81FB007B4FEAE07ADFF87B
:102F40008481C4F84807F4EEC77A81FB0201D717E1
:102F5000C7EB6107CAEB6B0AF1EE10FA5448D6F8DA
:102F600000C0C4F84C2708FB0EA108FB097788BFF6
:102F7000F0EE477AC4F87817C4F87C77C0ED007A91
:102F8000C4F880C7002B40D14A4AA4F88837138080
:102F9000019B1B78DB0710D4012384F88A3705B026
:102FA000BDE8F08F3A4B01931B7813F0010343D136
:102FB000D5E900CA374E384C79E7AB8936680F2B14
:102FC00054D8B4F93C37AA68D4F84017A4F83C2781
:102FD000D21A4FF47A7303FB02F3711A93FBF1F3E5
:102FE00040F2DC511BB28B42334AC4F84067A8BFA1
:102FF0000B469342B8BF1346D5E90021A4F83037F9
:10300000C4F83817C4F83427C6E7A0F15C0103AB55
:1030100002AA603836F05AFE2849039B029A2548D6
:10302000A1FB027281FB0371DB175209C3EB611331
:103030000280A4F88837ABE7164E174CFFF7F8FE6E
:10304000D5E901A132683B78C4F84027D5F800C023
:10305000A4F83C17002203F00103C4F82C27A4F8BD
:103060003027C4F838A7C4F834C720E7144903ABA5
:1030700002AA081F36F02AFED4F82C37029A13440D
:10308000C4F82C379DE700BF8093002010C40020B7
:10309000328F00207C960020803D0020CDCCCCCC0F
:1030A0006BCA5F6B6F12833A806967FF67666666FB
:1030B000044500208C93002024FAFFFF1F85EB516C
:1030C000B84400208096980030B40B4B0B4893F81E
:1030D0008B170B4C0268D3F84C542468C3F8505437
:1030E00081F0010183F88B1742F02002C3F84C44B1
:1030F00030BC0260C4E600BF803D0020AC860020EA
:103100007C9600202DE9F843C74CD4F88C3705464F
:103110004BB944E1D4F88C0710F086FCFCF7FEFFB5
:1031200098B9D4F88C37184610F086FC0028F1D1F5
:1031300094F85C24531E052B52D8DFE813F00900E5
:1031400051000900090055016600FFF7BDFFE8E7DF
:1031500094F84462002E00F08981012E40D1D4F809
:103160008C0710F05DFCD8B394F85C34032B00F0AE
:103170007383042B00F03083012B31D1AB4AD4F898
:1031800058341168CB1AC72B2AD9D4F85434042BDD
:1031900000F2D483A64AD4F88C07C4F8581403EB81
:1031A000430302EB8303D0F808E093F805140023EF
:1031B00002F557771E4604E0102B00F0C68357F83F
:1031C000046FB6455FFA83FC03F10103F4D1614556
:1031D00000F0E68302EB8102D2F85C130DF030FEC2
:1031E000944B1B6803F02003002B3FD1924D2B78AA
:1031F000DA075FBF914A137823F00103137025F0BB
:10320000A5FE002845D1BDE8F883D4F8483494F8E9
:1032100047220133C4F8483462B194F85D34884AD7
:103220000133DBB2A2FB0312920802EB82029B1A6B
:1032300084F85D3481487F4B02787C491B68814E5D
:1032400022F0020202700A680968C4F84C24C4F82B
:1032500058140022012103F02003B274C4F854244E
:1032600084F85E2484F85C14002BBFD0D4F8903727
:10327000EB1A002BBADB734B9B7C042BB6D905F5FC
:10328000123505F5F8750120C4F8905713F092FB3C
:10329000ACE76D4B1B8813F4006300F0A28094F838
:1032A0009437002B00F0608194F85C346749684AD9
:1032B000C978126884F8CC17A3F10503B3FA83F335
:1032C0005B0984F8BC37C4F89C2710F053F994F8D4
:1032D0008A37002B54D05F4AD4F8D41792ED0B7A7A
:1032E000D2ED0D4AD2ED0C5AD4F89C37C4F8D4373D
:1032F00027EE077A5B1AA4EEA47A574907EE903AB4
:10330000A5EEA57AD4F8D037C4F8D007C01AB1EE2C
:10331000C76A4C4B09889E7CA4F8A0179989B4F819
:10332000883784F8A867A4F8A617A4F8A437DFEDB7
:103330004B2A92ED003ADFED4A6A4A4A9FED4A5A1B
:10334000D2ED093A92ED074AF8EEE77A07EE100A55
:1033500067EEA27AB8EE477A26EE036AC7EE875A7E
:1033600066EE267A65EEA66AE3EE857AE4EE056AF5
:1033700082ED086AC2ED097AC2ED065AC2ED076A0B
:1033800094F89437072B00F2A280DFE813F0700165
:10339000AC00C4004A011101F50097009D0094F8AB
:1033A0008B67B1077FF5C4AE224FDFF880803A68A3
:1033B000D8F80010C4F8543442F0200284F85E3487
:1033C000D8F800903A60052326F00206C4F8581495
:1033D000C4F84C9484F85C34FFF752FD84F88B6792
:1033E00007E084F894375FE7D4F84C94DFF83C802A
:1033F000104FD8F800203B68A2EB090240F6C41138
:103400008A427FF6EFAE23F02003D8F800103B602D
:1034100006220023C4F8581484F85C24C4F85434F9
:1034200084F85E34E2E600BF803D00207C960020F8
:1034300040C50408AC860020328F00208093002015
:10344000CDCCCCCC10C40020948F0020348F002031
:1034500074930020988F00208C93002000247449DE
:10346000CDCC4C3E14450020CDCC4C3F012A00F081
:103470007281032A7FF4B4AECF4AD4F8583411686D
:10348000CB1AB3F57A7FFFF4ABAED4F85434C4F85A
:103490005814002B00F01082012B40F22582C74BFC
:1034A00012681B68C4F858240522C4F8546484F8D0
:1034B0005E6403F0200384F85C2495E64FF48010EA
:1034C0002BF026F816F0C8FB002384F8943725F07B
:1034D00033FA94F894370BB125F0CAFA002384F834
:1034E0008A37BDE8F883B4F814381BB9B4F82C381F
:1034F000A4F81438B4F8A027B4F836389A4207D2A2
:1035000094F8CC37062284F89527002B40F0BD8133
:10351000022384F89437D4F8C037D4F89C27B4F841
:103520001A189B1A002BB8BF5B42B3F57A7FB8BF5D
:103530000323D4F89827B8BF84F89437642303FB97
:1035400001F302F2DC529342B8BF13464FF4FA7013
:10355000012140F60A72C4F8C037C4F8C40784F8E1
:10356000CA17A4F8C827B2E7012384F8943725F0D6
:103570007FFA25F0E1F997E6914BD3ED097A93EDC7
:10358000087AF7EE086A67EEA67AB4EEE77AF1EE0B
:1035900010FA00F30681002301214FF4706284F8D1
:1035A000CA17C4F8C037C4F8C437A4F8C8278EE7D0
:1035B000B4F8A037092B07D8D4F89C27B2F57A7F46
:1035C000DCBF052284F89427B4F81A28B4F81E58F2
:1035D000B4F81C08D4F8C067642101FB02F203FBB5
:1035E00002F292FBF0F2632A03FB05F393FBF0F384
:1035F00040F3D580B242A8BF3246632BC4F8C0273F
:10360000D4F8C42740F3C9809342A8BF13460121D0
:1036100041F20A42C4F8C43784F8CA17A4F8C8278C
:1036200055E7B4F81C38B4F8A027B4F81A189A4231
:103630003CBF042384F89437D4F89827B4F81E3894
:10364000C4F8C437642303FB01F302F2DC52934253
:10365000B8BF134601200F21B4F81828C4F8C037AA
:1036600084F8CA0784F8C81784F8C9272FE72B788D
:10367000DB077FF52CAF94F8D837002B3FF427AF4A
:10368000504BD4F89807D3ED037A4F4AD4F89C37BF
:10369000B4F8A257B4F8A017D2ED086AFCEEE77AA6
:1036A0009842B8BF184617EE903AF6EE007AA94253
:1036B000F4EEE76A38BF29469BB20025F1EE10FA16
:1036C000A4F8E437C4F89807A4F8A217C4F8E057A0
:1036D000C4F8DC577FF7FBAEDFED3C7AF4EEE76A27
:1036E000F1EE10FA7FF5F3AED4F80C18DFED387A6E
:1036F00007EE101AB8EE477AB4EEE77AF1EE10FA58
:103700007FF5E5AE40F22E4083427FF6E0AEA3F5B2
:103710007A7307EE903AB8EEE77ADFED2E7AE7EEAD
:10372000267A4D1CFCEEE77A17EE903A9BB207EE34
:10373000903A002940F04881F8EE677A02F12803B8
:10374000B0EE670AC3ED007A37F0D8FCC4F80C5825
:10375000A4F81408BBE6184AD4F858341168CB1AF8
:10376000B3F57A7FFFF43CADD4F85434C4F8581460
:10377000002B00F09180012B40F2B0800F4B1268BB
:103780001B68C4F858240322C4F8546484F85E64A7
:1037900003F0200384F85C2426E5642337E70A4617
:1037A0002BE74FF480102AF0B3FE16F055FA0723EA
:1037B00084F89437EFE600BF7C960020AC860020AA
:1037C00014450020688F0020684500208FC2753F97
:1037D0000024744900007A4494F84622002A00F03C
:1037E0009D8094F85E24002A40F0828084F85E6414
:1037F000D4F85424B22A40F2C38000230222C4F831
:10380000543484F85E24794AD4F88C07134493F82E
:10381000F41410F015F9D4F8543494F85E240133FC
:10382000C4F85434032A00F09380714F3B68032A94
:1038300003F020037FF6D8AC6E4A3B681268C4F8E8
:1038400058240521002203F0200384F85C14C4F8F6
:10385000542484F85E24C7E494F85D34634AD4F8B1
:103860008C0703EB430302EB830393F8053402EB6D
:103870008302D2F85C130DF0E3FA5E4A5C4B1268E7
:103880001B68C4F858240421DCE74FF480102AF0A8
:103890003FFE16F0E1F93BE64FF49651D4F88C0761
:1038A0000DF0CEFA524BD4F854241B68013203F0C9
:1038B0002003C4F8542497E494F85D344B4AD4F8B8
:1038C0008C0703EB430302EB830393F8053402EB0D
:1038D0008302D2F85C130DF0B3FAE3E74649D4F85B
:1038E0008C0713F057F8DDE74449D4F88C07F8E764
:1038F000012A3FF47DAF022A94D1D4F85434092B25
:1039000081D90F2B54D994F8482200230321C4F8FD
:10391000543484F85E141ABB354F8DE7344B354967
:103920001B680868C4F85424052184F85E2403F059
:103930002003C4F8580484F85C1455E42C4B126836
:103940001B68C4F8582403217CE74FF0000C3EE4C8
:1039500094F84832002BDFD0D4F85434432BDBD812
:10396000224AD4F88C07134493F8241510F068F811
:10397000D4F8543494F85E240133C4F8543454E732
:103980001A4BD4F88C07134493F8401410F058F8ED
:10399000D4F8543494F85E240133C4F85434AAE7BC
:1039A00094F85D340C2101FB0322D2F8081498E747
:1039B00094F845120D4AD4F88C07C1EBC1010A44B2
:1039C000134493F8F71424E792ED0A6A07EE105AAD
:1039D000F8EEE77AF8EE476A77EEC67A134687EE96
:1039E000A67A283377EE067AAAE600BF40C5040817
:1039F000AC8600207C9600207C0B05089C0B0508FB
:103A0000F0B5364C364D94F844122B68C4F858344F
:103A10002868C4F84C040023022985B0C4F8C032D9
:103A2000C4F8C432C4F8C832C4F8CC3284F8D032F6
:103A300084F85D34C4F84434C4F84834C4F8BC3263
:103A400084F85C34C4F8543484F85E343CD00220EA
:103A500029F0DEF8B0B3077994F85D34214E02E026
:103A6000CBB2042B36D803EB430206EB8202591C7F
:103A700092F80524BA42F3D184F85D3494F85D34A9
:103A800090F902000C2202FB0363002793F805342F
:103A9000029706EB83060321D6F85C33009301916D
:103AA0003B463A46022128F039FFC4F88C0748B15A
:103AB0002B68C4F858340123C4F8547484F85E7435
:103AC00084F85C3405B0F0BD2B68C4F8583484F831
:103AD0005C14F7E7002384F85D34CFE7803D0020D5
:103AE0007C96002040C5040870B50446CC2582B001
:103AF00044306171A11D2571CDE90010251D9AB1D9
:103B00006E46114630461A46F7F78AF8304629467F
:103B1000F6F724F9009A019220680095521B294675
:103B20000FF05AFF02B070BD6E46EFE72DE9F04F7F
:103B3000DFF8E082B04F98F8023089B03D68002B82
:103B40003CD098F80040642303FB048214461369B8
:103B50000434002B60D09D425ED9D36D002B00F35E
:103B60008D80022620E098F80040621C132AC4BF12
:103B700000210A464FF0640403F1FF33D8BFD1B2ED
:103B800004FB02F4DBB208EB040288F802300434D0
:103B900088F8001093B113694444002B3CD0AB4229
:103BA0003AD2D36D002B69DC236984F8606020462B
:103BB00003B1984798F80230002BD4D18F4CDFF82E
:103BC0004082D4F83C78DFF83C9204F6880604F68C
:103BD0003C0A00255FFA85FB0BF11803DBB218469F
:103BE000059325F037FA00285BD0725D059B002A0B
:103BF00040F0C780192BB4F8822800F0D8801A2B27
:103C000074D1530700F1E9801FB1B4F882381A0764
:103C10007DD409B0BDE8F08F636918680FF00CFF20
:103C20000028CBD0636918680FF0FEFEA3785BB95B
:103C300094F85720012A05D032B9552804D098F8B5
:103C400002307BE7CC28FAD16268D054A37862783E
:103C50000133DBB29A42A370F1D194F85730012BB3
:103C600000F094800BB984F8603023690BB12046D2
:103C7000984798F80230F3B93B689FE794F85730BB
:103C8000012B27D023B9636921781868FCF7C6FE99
:103C9000A268A36D1544013B0022E560A365A270F4
:103CA0008CE70BF1190B70555FFA8BFBBBF11B0F07
:103CB000AAD001358EE798F800200132132A03F1CB
:103CC000FF33D4BFD2B20022DBB288F8023088F8CA
:103CD000002033E760690368002BD9D094F8563090
:103CE000217804F11802FFF7FFFED1E70BF1190B61
:103CF00090075FFA8BFBD9D598F80030D907D5D457
:103D0000D9F8003013F02003D0D1194655E094F8CB
:103D10008B38002B7FF47DAF394B1B78DB073FF5E9
:103D200078AF384B1B6813F020037FF472AF94F820
:103D30006D24002A7BD0344A9188A1F24751B1F515
:103D4000957F3FF666AF5188A1F24751B1F5957F57
:103D50003FF65FAF1288A2F24752B2F5957F3FF669
:103D600058AF2A4A029202214FF4C872CDE90021CD
:103D700027481A46032132F085FF012384F86C346A
:103D800047E70BF1190B5FFA8BFB8FE762B16568B0
:103D9000013DAE18002015F8011FF6F71BF8B542DB
:103DA000F9D1021C18BF012284F860205DE7D20718
:103DB0007FF57FAF4FF01A0B012194F880388DF812
:103DC0001E10012B28D02BB938460131FCF726FEF6
:103DD000D4F83C780123735568E798F80030D80789
:103DE0003FF512AFD9F8003099063FF50DAF4FF00F
:103DF0001B0B0221E1E700BF7C960020803D0020E4
:103E0000328F00207C930020ECC30020550B01086A
:103E1000BC45002030970020002FDBD019460DF163
:103E20001E025046FFF760FED4F83C78D2E794F8C3
:103E30006C34002B7FF4EDAE4A4B94F86E24D88896
:103E4000A0F2475080B2B0F5957F28D81988A1F22A
:103E50004751B1F5957F22D85988A1F24751B1F564
:103E6000957F59D8B3F90410B1F5876F54DA002A59
:103E70003FF4CFAE08AA022302F8013D3A4901936C
:103E80004FF4C8730291009304210123374832F0A4
:103E9000F9FE012384F86D3484F86C34B9E6002A05
:103EA0003FF4B7AEB3F90010B1F5876F32DBB3F969
:103EB0000220B2F5F06F52DCB1F5F06F4DDCB2F5D7
:103EC000876F48DBB0F5957F3FF6A3AEA1F247516F
:103ED00089B2B1F5957F3FF69CAEA2F2475292B2FD
:103EE000B2F5957F3FF695AEB3F90430B3F5F06FB8
:103EF0007FF78FAE012308AA1B4802F8013D02217B
:103F00004FF4C873CDE9011000931848012332F033
:103F1000B9FEBEE70223EEE7002AC3D15A88A2F217
:103F20004752B2F5957F3FF674AEB3F90430B3F55E
:103F3000F06F7FF76EAE08AA01230B4902F8013D2E
:103F4000022002914FF4C871CDE900100421074806
:103F500032F098FE9DE70523CDE70323CBE704234A
:103F6000C9E700BFECC30020550B0108BC45002089
:103F700030B5194C85B000254FF4804084F8845842
:103F800028F046FEF8B14FF4E133032290F9020025
:103F90000295CDE900324FF480412B462A4628F0A5
:103FA000BDFCC4F83C0870B10C4994F86424D4F802
:103FB00068340093CDE901212B462A46294604F6B0
:103FC0003C0032F05FFE012384F8883884F8893899
:103FD00084F88A3805B030BD803D0020890A010888
:103FE00010B50A4C94F88B3803B110BD04F5D360BA
:103FF00006F00DF80028F8D005F0EEFA044B1B6827
:1040000003F5C873C4F8DC3110BD00BF803D00204B
:104010007C9600200A4B30B5D3F8F814094C0022E6
:10402000155D854208BFA1181032A02AF8D193F877
:10403000FC24C3F8F81442F0020283F8FC2430BDDB
:10404000803D0020A8CA0408144C08B50646D4F8E0
:104050008C0728F043FC304628F040FCD4F88C57FD
:1040600029798A0711D50E4B1B689B0308D50820B8
:10407000FFF7D0FF94F8FC3423F0010384F8FC34FC
:1040800031462846074A35F04BF8284641F00201F0
:104090000FF0C2FCD4F88C57E5E700BF803D00204C
:1040A000A8B80020114B0108024B0146D3F8E004E8
:1040B000FDF731BA803D002070B5104E002496F80F
:1040C0008C38A34201DD0E2C00D170BD611001318E
:1040D000C9B2D6F8E004E5B2FDF788FA284635F013
:1040E00091FD96F88C38A34206DD2020FFF7DCFF17
:1040F000681CC0B235F086FD0234E0E7803D002048
:10410000642928BF6421F8B511FB00F56424064634
:1041100095FBF4F40027E4B2FBB29C4212D8A6420D
:104120000BD9142095FBF0F0C4EB84156638C4EB72
:1041300085052844C0B2FFF7B7FF0134E4B2B442AA
:1041400005D3F8BD9F20FFF7AFFF0137E4E79A20C2
:10415000FFF7AAFFF1E7F7B52F4F7A79002A57D07A
:104160002E4B2F4D19880A23B1FBF3F203FB1213D8
:104170002C49097800919BB22B4905F58E60F5F723
:10418000D7FDFCF753FDD5F8E04401212046FDF7AB
:104190002DFA05F58E612046FDF7DCF91CF084FB55
:1041A000022105462046FDF721FA29461520FFF792
:1041B000A7FF0326BB796BB31C49194D08688968B2
:1041C000009164230A2190FBF3F203FB120305F52F
:1041D0008E6093FBF1F31649F5F7AAFDFCF726FD77
:1041E000D5F8E04431462046FDF700FA05F58E612A
:1041F0002046FDF7AFF91CF057FB711C0546204621
:10420000FDF7F4F92946152003B0BDE8F04077E743
:104210000126CFE703B0F0BD788F0020608F00202B
:10422000803D0020668F002091080508888F0020BF
:10423000A908050803685B6A184703681B6A1847E2
:104240000368DB69184700BF2DE9F041764B1D6814
:1042500082B0002D3ED0FF230C468DF803308DF840
:104260000230002839D1714A92F8A438002B6DD061
:104270006F4B93F888506DB392F8AA186D4A0029D5
:104280004FF0000192F8EAE192F8EB8103F18C0023
:1042900014BF4FF00F0C8C460A460F4603F5C0734F
:1042A00050F8044B24040ED5002A4CD0964503D375
:1042B000B8F1000F00F08780002426460132D2B208
:1042C0001E809F70DC700131A94203D0062A03F1E1
:1042D0000403E5D102B0BDE8F081564E0DF10202B3
:1042E0000DF103012846FFF7ABFF06F5F5712846EF
:1042F000FFF7A3FF284606F2EB11FFF79BFF9DF89F
:1043000003309DF8020096F8EA5196F8EB111A0175
:1043100002EB450200EBC303093B1144464D434AFF
:1043200001EB002135F8130092F8A438A2F8A60892
:1043300089B2002B4AD1B2F8A8388B425FD0A2F8DC
:10434000A8180F2344E064467826B7E7394EB2F840
:10435000A63841F228618B421AD80123344996F8D5
:10436000EB0101EB8303D3F80C310193002840D01B
:1043700092F8AA38002B0CBF00230F2301A94FF499
:1043800000408DF80730FAF709FE02B0BDE8F08171
:1043900041F24F618B422ED941F276618B422CD98A
:1043A00041F29D618B4239D941F2C5618B4237D9C7
:1043B00041F2EB618B4235D941F212718B428CBFD5
:1043C0000D230B23CAE764461E2677E7A2F8A81838
:1043D000216892F8AA08013B01F54331DBB201F5EF
:1043E000A07180F0010082F8A438216082F8AA0848
:1043F0003CE7FF23C2E70223B0E70323AEE72168CF
:1044000092F8AA08A2F8A83801F5433303F5A0737F
:1044100080F00101236082F8AA1898E704239DE741
:1044200006239BE70A2399E764900020803D002043
:10443000882C002014000020A4FD040803685B6998
:10444000184710B103685B681847FF2070472DE9D3
:10445000F04F0C46002185B007460846164612F07C
:1044600031FE0021012012F02DFE19F0ABFB022ECF
:1044700000F09281042E44F6C01818BF4FF49648FD
:10448000C04800232425024602E001330A2B06D04F
:1044900005FB0301897911F00401F6D0D9B221445A
:1044A000C9B2092913D8032E00F07C8101EBC103A6
:1044B000B54802EB83030364242303FB0121CB797A
:1044C000990740F16F81B14B0022C3F8AC2805B0C9
:1044D000BDE8F08F012E08D1D4F84404414634F0F1
:1044E000CDFD206C34F0A6FDCAE1022E08D1206C6F
:1044F000FCF7AEFD4146D4F8440434F0BFFDBFE103
:10450000032E40F082804FF0000984F85C9840222E
:1045100049469F48DFF87CB236F0F4FC994B8DF8A1
:104520000E909DF80E20072A09D901219648FCF724
:1045300070FE4146D4F8440434F0A0FDA0E19DF89B
:104540000E2002EB42020BEBC202527C002A4ED03C
:104550009DF80E2002EB42020BEBC2025269002AC8
:1045600045D000228DF80F204FF0240A9DF80F202F
:10457000092A2CD89DF80E909DF80F2001930AFB74
:1045800002325FFA89F909EB490910790BEBC90985
:1045900012F06CFBD9F81420019B82422ED19DF8B9
:1045A0000F0000EBC00003EB8000FCF751FD9DF80D
:1045B0000F20019B0AFB023A9AF80720D20706D582
:1045C00094F85C2805EBC202012182F8A0149DF842
:1045D0000E2094F85C1802EB42020BEBC20205EBD2
:1045E000C1005269C0F89C24013184F85C189DF820
:1045F0000E200132D2B28DF80E2092E79DF80F20E6
:104600000132D2B28DF80F20B0E7042E40F038818D
:10461000206CFCF71DFD5FE7D5F8AC080FF004FA3D
:10462000014638460FF00CFA39E138460FF0FCF934
:1046300095F8BF2803469AB9242803D14FF0010208
:1046400085F8BF28012E05D11946384601930FF091
:10465000F7F9019BD5F8AC0819460FF0F1F934E1F0
:10466000012A06D14D2814BF0022022285F8BF2856
:10467000E8E7022A06D13C2814BF0022032285F86D
:10468000BF28DFE7032A10D10A2802D985F8BF889E
:10469000D8E7042285F8B20885F8B18885F8B4888F
:1046A00085F8B30885F8BF28CCE7042A09D195F826
:1046B000B32885F8C008424085F8B32885F8BFB80C
:1046C000C0E7052ABED195F8B11895F8B29895F8CB
:1046D000B308494509D24A1C2944584085F8B30813
:1046E00085F8B12881F8B538ACE79842CED195F875
:1046F000C01885F8BFA8F429A4D1B9F1000FA1D141
:104700002421384685F8BF980FF09AF94D21384694
:104710000FF096F93E2138460FF092F94946384697
:104720000FF08EF9F42138460FF08AF9F42138465B
:104730000FF086F9032E17D0206C437901689D088D
:104740000223AB40DB439BB20B828D892B408B81D4
:1047500000792021FCF76CFC206C494632F006FB06
:10476000236C18682EF0A4F9D4F84404002132F028
:10477000FDFAD4F84434186805B0BDE8F04F2EF0C7
:1047800097B900BF88FE040864B90020803D00206E
:104790001C420020DCAA0020FF2C4FF416487FF4B6
:1047A0006FAE0326514C524D84F85B6895F8B00803
:1047B0000DF0CAFF4F4B236004F1440103234FF473
:1047C000806223716161002304F589614FF0010962
:1047D000032EC4F84404C4F808806371E362E26005
:1047E000C4E90733A1612261C4E9093384F84C3874
:1047F000A4F84898C4F85438A4F8583884F85A38BB
:104800000DD0D4F840A09AF8040012F02FFAE0631B
:104810005046FCF72DFC49462046FCF7FAFC3220B6
:104820000EF058FF002E7FF455AED4F84484D8F82B
:1048300000002EF03DF940462F4A22210DF05AFE8D
:104840002E4BC4F8603832462D4940460DF0BCFD71
:10485000D4F84080D8F800002EF02AF9264A4FF606
:10486000FF7140460DF046FE3146404632F01AFBDD
:10487000244BC4F864383246234940460DF0A4FD69
:10488000C5F8AC484FF0060A022E12D0D5F8AC0895
:104890000FF0D2F868B10121002012F013FCD5F816
:1048A000AC080FF0C9F8014600287FF4B5AE12F04D
:1048B00009FC38460FF0C0F888B10121084612F013
:1048C00001FC4FF0050B4FF0000838460FF0B4F82C
:1048D000014600287FF4A9AE012012F0F3FB042E5C
:1048E000D4D005200EF0F6FECEE700BF64B900205C
:1048F000803D002048CB040840420F00A912010867
:10490000C4C1002097100108C8C1002038B5417902
:104910000446AE23802290F90400F9F753F80546C7
:1049200088B1162209492046FCF71FFE04220849D7
:104930002046FCF71AFE2046FDF78EF903220549B2
:104940002046FCF712FE284638BD00BF78CB04088D
:104950008ECB040892CB040870B5654CD4F8C438EB
:10496000064623B193F90E30002B00F3C080D4F833
:10497000C838F31A002BC0F2BA8006F5433303F5AA
:10498000A073C4F8C8385B4B1D7894F8CC3805F098
:10499000010584F8CC5875B3012B00F0A8800120E4
:1049A000FFF738FB012384F8F43494F8F434002B37
:1049B00059D094F8FC3423F0020384F8FC344E4BB5
:1049C0003344D4F8E064C4F800353046FFF79EFF66
:1049D00084F8CD08002800F08A803046FDF73CF9C5
:1049E00030460021FCF702FED4F8F834304659680E
:1049F000FCF7B0FD37E02BB194F8FC3443F0020330
:104A000084F8FC3494F8FC3413F002011DD0012228
:104A100084F8F424D907C8D594F8FD3437480A211E
:104A20000133DBB2B3FBF1F201FB1233DBB200EB7B
:104A3000031292F87425D207F2D4314A84F8FD3477
:104A400002EB0313C4F8F834AFE7D4F80025B21A28
:104A5000002A02DA84F8F414A7E703F0010284F8CC
:104A6000F424002AD6D194F8CD38002B3FD0D4F8C6
:104A7000F8349B689847002D39D1224BD4F8E06474
:104A800093F82020062A9BBF1C4B9B183F2593F8C8
:104A90005556002212213046FCF777FD2946304654
:104AA000FCF739FD132100223046FCF76EFD164B52
:104AB00093F80932002B94F8CE3814BF72212121CB
:104AC000002B18BF52213046FCF725FD002214218F
:104AD0003046FCF75AFD94F8CF580C4B595D013520
:104AE000304605F00305FCF716FD84F8CF5870BD7D
:104AF000803D0020328F0020404B4C0040C5040810
:104B0000A8CA0408348F0020882C0020A5070508B7
:104B100008B5FBF703FB48B9064B1B689B0300D4A1
:104B200008BD0EF027FDBDE8084015E7FEF7CCFAFA
:104B3000F2E700BFA8B80020064B1A78064B1B7896
:104B400003EBC203093B054A32F81320044B1A80D9
:104B5000704700BF6291002063910020A4FD04080B
:104B6000649100202DE9F04FAF4A32F810B093B0B5
:104B700006465846FAF709F803901446002800F054
:104B80006483730902EB830206F01F000123D2F84D
:104B9000F8258340134205D0A44B93F8EC31002B49
:104BA00040F0388700211C220BA80BF01F050A914A
:104BB000CBF3441B36F0A6F92F2E00F22B87DFE84B
:104BC00016F08100A100AB02F5024803A201A20188
:104BD000E9016A0281028E02BB00CC00DE00D40033
:104BE0009C0186039303A003AD03BB03C503C0056B
:104BF0000001F900DB05EC05EC053D06790607012F
:104C000059018F06A8068301C606DC06A901F40631
:104C1000F9061007250273033502140730008F00D0
:104C2000760194F81332002B48D08149B1F9003055
:104C3000B1F9021009294FF00A0293FBF2F3A3F134
:104C4000B00221DD032A03D903F1B302032A0BD8F2
:104C500060238DF8283077480AAB5A462946D0F8A9
:104C6000EC0113F0E9F9F0E29BB25A1EAD2A03D829
:104C700066238DF82830EEE7AE339BB2AD2BEAD831
:104C80006E238DF82830E6E7032A03D903F1B30237
:104C9000032A03D868238DF82830DCE79BB25A1E1C
:104CA000AD2A03D86A238DF82830D4E7AE339BB2FF
:104CB000AD2BD0D862238DF82830CCE720238DF897
:104CC0002830C8E70AF08EFA642343439B12632B13
:104CD000A8BF6323012258490AA8F5F729F8BAE7C3
:104CE000544B564993F8D02802EB8202FF2352001E
:104CF00092FBF3F20A2A08BF0922D2B20AA8F5F7FA
:104D000017F8A8E74E4B1C884E4B0A2101FB04F014
:104D10001B7890FBF3F0F9F75DFFB4FBF1F201FBB8
:104D2000124306218DF8280000919BB246490DF1EF
:104D30002900F4F7FDFF8EE7444B1B68002BB8BF3A
:104D40005B4264219A2093FBF1F2009001FB123345
:104D50000AA83F49F4F7ECFF7DE73C4A3D499268D9
:104D600007230AA8F4F7E4FF75E73B4B3B499B7C1C
:104D700000931E221F230AA8F4F7DAFF6BE7364BD5
:104D800094F869209B8952B942F210725A4334490F
:104D9000344B92FBF3F20AA8F4F7CAFF5BE7242234
:104DA0005A4331494FF47A730AA892FBF3F2F4F7AD
:104DB000BFFF50E7284B68211A680AA8FAF700FEDF
:104DC00049E7254B64215A680AA8FAF7F9FD42E73A
:104DD000264B1B7803F00303032B20D1244B1B88A5
:104DE000CBB1144B124AB3F98837B2F904200A2127
:104DF00092FBF1F29B1A1B0103F5B95314334FF4E4
:104E0000B472B3FBF2F3C3F1080303F00F03603392
:104E10008DF828301FE705238DF828301BE72D2358
:104E20008DF8283017E700BF882C002014000020E0
:104E3000D48F0020803D0020D908050836090508D8
:104E4000608F0020668F0020BC080508888F002036
:104E5000C6080508D108050810C40020D7080508B1
:104E6000DF08050840D20600E4080508809300200A
:104E70008C930020AC4B1B7803F00303032B0CD165
:104E8000AA4B1888F9F798FE0246F9F7C7FEA84919
:104E900003460AA8F4F74CFFDDE62D238DF82830F1
:104EA0004FF02033CDF82930ADF82D30D3E69E4BAE
:104EB0001B7803F00303032BEFD19E4BD3F82C0791
:104EC0006423B0FBF3F0DDE79B4B0A22B3F9043017
:104ED00093FBF2F31B0103F5B9534FF4B47214338F
:104EE000B3FBF2F3954A03F00F0313440AAA1868C0
:104EF00059681B7A03C21370ADE6914B0AA8196872
:104F0000FAF77CFDA7E60122731F11460AA8FAF7FB
:104F100081FEA0E68B4B9FED8C7A9A68B4F86430E2
:104F200007EE902AF8EEE76A07EE903AF8EEE77A95
:104F300067EE877AF4EEE76AF1EE10FA04D8834957
:104F40000AA8F4F7F5FE86E6934204DA80490AA837
:104F5000F4F7EEFE7FE69B1A07EE903A754B7D4A1A
:104F6000B8EEE77AD3ED7C7AF8EE677A3C2167EE0B
:104F7000277A0AA887EEA67AFDEEC77A17EE903A4E
:104F8000B3FBF2F393FBF1F201FB12337249F4F736
:104F9000CFFE60E6714B1B885A0504D570490AA8FC
:104FA00035F0D4FF57E61F0504D56E490AA835F041
:104FB000CDFF50E65E0604D56B490AA835F0C6FF62
:104FC00049E6DC0704D569490AA835F0BFFF42E687
:104FD000980704D566490AA835F0B8FF3BE62520B6
:104FE00024F038F820B163490AA835F0AFFF32E663
:104FF000504B93F8D13823B15F490AA835F0A6FF8A
:1050000029E65E490AA835F0A1FF24E65C4B93ED42
:105010007C7AD3ED7D7AB4EEE77AF1EE10FA7FF781
:105020001AAE58490AA835F091FF14E623F007FCA0
:10503000554E564B1C783346F3EC017AFDEEE77A79
:10504000002217EE90CAD3ED007AFDEEE77A08361B
:1050500017EE901A0AAFA1EB0C01944205DC12ABDB
:105060001C44002304F8203CF5E590B106EB8203D4
:10507000D3ED007AFDEEE77A17EE903AA3EB0C033E
:10508000DB0093FBF1F3C3F18803DBB2D3550132AC
:10509000E3E78823FAE7274E96F8FC280AAF22B9FF
:1050A0003B49384635F052FFD5E5002406F6FC06AC
:1050B000A05D0028D3D0F5F7EDF938550134102C58
:1050C000F6D1CCE740F20453ADF8283014F056FD89
:1050D000304902460DF12A00F4F72AFEBBE52E49BD
:1050E0002E4A0B78D45C2E4B4A7853F822608B788A
:1050F0008DF81C302B4B186820B10B7A13B107A91F
:10510000FFF79BF89DF81C30009322463346264952
:105110000AA8F4F70DFE9EE547F62663ADF82830A1
:1051200027238DF82A3096E5809300208C93002069
:10513000E9080508803D0020D48F00209CCB04089E
:1051400074930020888F0020CDCCCC3DEE0805085C
:10515000F408050840420F002C070508948F002032
:10516000FA080508FF0805080409050809090508E3
:105170000E09050813090508180905081D09050881
:10518000140000202209050854460020058600204E
:10519000250905083F0A0508288F0020F4FD0408AA
:1051A000FCFD0408649000203009050894F87F1085
:1051B00094F87120BC4894F87030B0F90040002990
:1051C00002EB82020CBF01214FF0FF3152004C4331
:1051D000574203EB8303BC424FEA430303DB944291
:1051E000A8BF14462746B0F902205C424A43A242B7
:1051F00003DB9A42A8BF1A4614461BB11922544336
:1052000094FBF3F4293C4FEA87086FF003064FF054
:1052100040094FF0090A98FBF9F31B1B512B0FD8DB
:1052200093FBFAF202EBC2015B1AA048803B5A449E
:10523000A919DBB2D2B2C9B2D0F8EC0112F0F2FE79
:105240000136052EA8EB0708E5D1039813B0BDE899
:10525000F08FA5F10708954C6FF002065FFA88F809
:105260000BEB0607FFB213233A464146D4F8EC0194
:1052700012F0D8FE013613233A46E91DD4F8EC01AA
:1052800012F0D0FE042EEBD1A91F5A460323C9B257
:10529000D4F8EC0112F0C6FE02235A46A91DD4F838
:1052A000EC0112F0BFFED0E7814B93ED000AF2EE65
:1052B000047A20EE270A35F021FF0A237D4990FB6E
:1052C000F3F203FB12030AA8F4F732FDC3E47A4BAE
:1052D0001A68917A137A0191527A00927749784A42
:1052E0000AA8F4F725FDB6E4734B1A68117C937B8A
:1052F0000191D27B00927149724A0AA8F4F718FD15
:10530000A9E46D4B1A68917D137D0191527D009245
:105310006A496D4A0AA8F4F70BFD9CE46B4B6C4993
:105320001A886C4B1B680AA853434FF47A7293FB9C
:10533000F2F2F4F7FDFC8EE4674A6849537812787C
:10534000013301320AA8F4F7F3FC84E494F88430C2
:1053500005930EF00FF9D4F8F835B4F86E70534E8B
:1053600023F4001317F0010F8046C4F8F83545D038
:10537000002023F06FFE00283DD0594B1A68002A08
:1053800039D0D10204D5B2F5801F18BFA2F5801222
:10539000D6F814099FED537AA8EB000307EE903A74
:1053A000F8EE677AF4EEC77AF1EE10FA05DCD6F87B
:1053B000181901238B40134212D110B91423C6F8D7
:1053C0001839D6F81839C6F8148901200133152B7D
:1053D00028BF002300FA03F11142F7D0C6F81839AC
:1053E000D6F81829404B03EB82030AA8D3F87416A9
:1053F00034F0B2FC2FE40023C6F81439D6F81C3977
:10540000A3B33A4B1B78DA0730D4D6F820099FEDC6
:10541000387A00F5921000F57860A0EB080307EEEB
:10542000903AF8EE677A67EE877AFDEEE77AB8EEA3
:10543000E77A17EE903AF1EE0C7AB4EEE77AF1EEF5
:1054400010FA04DB2B490AA834F086FC03E40A2195
:1054500007A893FBF1F201FB12332749F4F768FC2C
:1054600007A90AA834F078FCFFF7F5BBBB050ED5F9
:10547000224BDB785BB122490AA834F06DFCD4F8EA
:10548000F83543F40013C4F8F835FFF7E4BB3807E8
:1054900004D5059B022B01D11A49EDE71A4B1B8855
:1054A000590635D51949E7E7D48F0020803D002003
:1054B000904600203A090508849300204909050810
:1054C00045090508580905085C090508608F002092
:1054D00060090508888F002090A80020650905084C
:1054E0007C9300200024F44840C50408328F00203B
:1054F000ACC527376B09050876090508348F0020ED
:10550000830905088D090508948F0020970905086F
:105510003A0611D5B6F9240994F87E3098420BDB8F
:10552000FAF7A4FA0246F9F73DFBAA49034607A891
:10553000F4F7FEFB07A99FE7A74B1B681B0179D572
:105540007F0677D5A54B1E78C6F10806760800239E
:1055500007AA20219E4225D19319A14904931846F8
:1055600035F0F4FC4FF00009DFF89C8203364F461B
:105570009A4B1B78BB4201D90A2E16D912AB1E4496
:10558000002306F82C3CB9F1000F53D007A90AA854
:1055900034F0E2FBD8F8F83543F40013C8F8F835D6
:1055A000FFF759BBD1540133D4E75FFA87FA50466D
:1055B0002EF0ACFD8B4B0AF1310293F800A01AF0EB
:1055C000010AD2B234D0B8F97AE0BEF1FF3F2FD051
:1055D0008189642311FB03F1834B93F816C04FEAD2
:1055E0005C0C91FBFCF39E45B4BF1346522398F923
:1055F00078C004991CF1800F06F10106394404D0EB
:1056000090F901E0E64580F20882BAF1000F08D077
:10561000B8F97CC0BCF1FF3F03D040686045A8BF2B
:1056200043239342CB7001D009F1010901379FE771
:105630001346DCE7B4F86E309E0608D594F81322C2
:105640002AB16A490AA834F087FBFFF704BB13F4B8
:10565000806F674A28D092F82619012924D1654B1A
:105660001B689C071AD5644BB2F93629B3F902308E
:1056700062499B1A0A2293FBF2F35A2B6FF05902EC
:10568000A8BF5A239A42B8BF1A4607A8F4F750FB9E
:1056900007A90AA834F060FBFFF7DDBA58490AA849
:1056A00034F05AFBFFF7D7BA58070FD505990129EF
:1056B0000CD154490AA834F04FFB534AD2F8F835BC
:1056C00043F40013C2F8F835FFF7C5BAD9050DD574
:1056D00044490978CF0709D54C4991F8251001298B
:1056E00004D14B49097809B94A49E3E79E0717D520
:1056F0003C4909788C0713D4434991F8841079B94F
:1057000045484649047846480988807B91FBF4F176
:10571000884205D943490AA834F01EFBFFF79BBA1B
:10572000D80608D592F838392BB13F490AA834F089
:1057300013FBFFF790BA00210AA834F00DFBFFF726
:105740008ABA364B1B880A215943334B1B7891FB8D
:10575000F3F10846F9F73EFA64238DF82800062095
:1057600091FBF3F2009003FB12130DF129002F4976
:10577000F4F7DEFAFFF76FBA2D49B1F90600B1F977
:105780000230B1F900200190B1F9041000910AA88B
:105790002849F4F7CDFAFFF75EBA174B1A2E0CBF63
:1057A000B3F90200B3F900000A21002890FBF1F3DD
:1057B00001FB1301ACBF20222D220029B8BF4942B2
:1057C000002B0091B8BF5B421B490AA8F4F7B0FA5E
:1057D000FFF741BAA0090508A8B8002005860020F7
:1057E00000090508328F0020A0AB0020AC09050895
:1057F000803D0020AC860020D48F0020B70905082A
:10580000C1090508C8090508882C002054B80020E3
:1058100024C20020D4090508668F0020608F002074
:10582000788F0020E0090508EC090508372B0508EA
:1058300064940020F60905080A0A05087A4B1A89BB
:105840007A4B9B68D31A9342A8BF134623EAE373AB
:1058500007EE903A0B23B2FBF3F300EE103AF8EEAA
:10586000E77AB8EEC00A87EE800A35F001FC12A98B
:105870008A2201F8202D0122FCEEC07ACDED047AB7
:105880009DF810309342B4BF8D208B2050540132CC
:105890000C2AF7D18F228DF834205A1E092A9FBF77
:1058A00012AA9B188E2203F81F2C00238DF8353086
:1058B000FFF7D1B95E4B1B78D90705D45D490AA81B
:1058C000F4F736FAFFF7C7B95B4B93F83939002B79
:1058D0007FF4C1A959490AA8F4F72AFAFFF7BBB91E
:1058E000574B0A22B3F9043093FBF2F31A0102F585
:1058F000B9524FF4B4711432B2FBF1F2C2F10802A2
:1059000002F00F0260324F490AA8F4F711FAFFF7CC
:10591000A2B94D4BB3F90000F9F74EF964210A2200
:1059200090FBF1F301FB130191FBF2F10029B8BFE9
:105930004942002B0091B8BF5B4244490028ACBFEC
:10594000682260220AA8F4F7F3F9FFF784B9404B04
:105950001B681A017FF57FA9374BD3F83C3993F9BF
:105960000100FAF783F80246F9F71CF939490346B2
:105970000AA8F4F7DDF9FFF76EB9354B1B681B0178
:105980007FF569A92C4BD3F83C2942B19289642355
:1059900012FB03F2304B9B7D5B0892FBF3F22F4925
:1059A0000AA8F4F7C5F9FFF756B90AA8FCF74EFEA6
:1059B000FFF751B9204BD3F84029002A7FF74BA9B4
:1059C000274B03EB8203D3F8C426002A3FF443A9F4
:1059D000244B2549D3F8F8310AA8F4F7A9F9FFF7C1
:1059E0003AB9154BB3F92409BBE7134B93F8462991
:1059F000032A02D1D3F84C392BB91C490AA8F4F771
:105A000097F9FFF728B9002219490AA8F4F790F985
:105A1000FFF721B90023039317E45423BAF1000FD1
:105A20007FF4F6ADCB70FFE5788F0020888F0020E3
:105A3000328F0020160A0508803D00201F0A050845
:105A4000D48F0020280A0508DA8F00202F0A0508C5
:105A5000A8B80020A6090508A0AB00204A07050841
:105A600040C50408140000203B0A0508430A050845
:105A7000460A05082DE9F04FB14DB24C95F81432A5
:105A80008BB0814613B1012384F83839D4F85039EA
:105A90000527B3FBF7F707EB8707DF1B40F0088507
:105AA000A94A94F85419137803F0010399429046D7
:105AB00035D0002B00F0FC804FF0FA730022C4F8C0
:105AC000F831D4F8EC01C4F80822632384F8FE31DD
:105AD00084F8143284F8557984F85679C4F8007241
:105AE000A4F80472C4F8F471A4F8FC71A4F80C7260
:105AF000C4F8107212F0C4FA944BD4F8EC010722E7
:105B00000C2112F099FA09F5F42303F59073C5F806
:105B1000003698F8003003F0010384F8543998F8FF
:105B2000003013F0010300F0EA80894B9A8995F860
:105B30006930002B40F0DB8042F210735343854AFA
:105B400093FBF2F31BB2B4F9F8219A42B8BFA4F860
:105B5000F831814BB4F9FA21B3F900309A42C8BF49
:105B6000A4F8FA317D4B64221B6893FBF2F3B4F97D
:105B7000FC211BB29A42B8BFA4F8FC3109F0FCFA30
:105B800094F8FE31D4F8002294ED827A8342744B6B
:105B900088BF84F8FE011B689A42B8BFC4F800327F
:105BA000704BD3ED007A94F8D038642213FB02F3E3
:105BB000B4EEE77AFF2293FBF2F394F81422DBB2FF
:105BC000F1EE10FA48BFC4ED827A9A4288BF84F899
:105BD0001432654B1B7803F00303032B07D1634B8F
:105BE000B4F904221B889A42B8BFA4F80432604B6F
:105BF0001B681E0119D5D4F83C39B4F90C1293F97D
:105C000001209B899142B8BFA4F80C22642213FBA7
:105C100002F3584A927D520893FBF2F3D4F8102213
:105C20001BB29A42B8BFC4F81032D4F85C39D4F829
:105C3000F021A9EB03031A44C4F8F021D4F8F421AD
:105C40001344C4F8F431D5F80036C4F85C99002B3D
:105C500000F0CB82A9EB0303002BD4F8EC0180F217
:105C6000BB82454AB2F9061040F2D663994203DC82
:105C7000B2F902209A4201DDC5F8009612F0CEF981
:105C8000002384F83839D4F850390133C4F8503936
:105C9000D4F8EC3123B193F90E30002B00F30F84CC
:105CA000364A136823F4804313600BB0BDE8F08FCD
:105CB0006B6F002B3FF42DAF94F85739002B7FF416
:105CC00028AF2E4B1B689B0605D5688DF8F75DFF46
:105CD00000287FF41EAF012384F85539284B4B442C
:105CE000C5F800361C4B1B88A4F8583911E724234B
:105CF00053434FF47A7293FBF2F31BB223E794F809
:105D00005529002A9FD0D4F8EC6156B196F90E209F
:105D1000002A06DD84F85539C5F80036C4F8F43198
:105D200091E70E2023F096F994F8563950B3002BE2
:105D300089D00023304684F8563912F0A1F982E761
:105D4000882C0020803D0020328F0020190A050891
:105D500010C4002040D20600608F0020888F0020F1
:105D60007493002090460020809300208C930020A4
:105D7000A8B80020A0AB0020ECC300207C9300203A
:105D80000087930323B9012284F85629C4F86039A7
:105D9000D4F860399945FFF456AF09F5742303F53B
:105DA00010733046C4F86039B4F858A912F068F995
:105DB0000222B94BD4F8EC01114612F03DF96B6F99
:105DC000D80740F1078202A8FCF740FC18B9B34994
:105DD00002A8F3F7ADFF02AB03220221D4F8EC01D5
:105DE00012F02AF904266B6F99071CD5B5F86A20C2
:105DF000002312F00F0218BF0122194602A8F9F77A
:105E000009FFB5F86A3003F00F02A54B03EB8203DC
:105E1000304602AAD3F84C1706F1010BF9F73EFE03
:105E20005FFA8BFB5E466B6F5A071CD5B5F86C208A
:105E3000012312F00F0218BF1A46002102A8F9F739
:105E4000E9FEB5F86C3003F00F02954B03EB8203CB
:105E5000304602AAD3F84C1706F1010BF9F71EFEE3
:105E60005FFA8BFB5E466B6F1B0712D58D4B1B6871
:105E700018060ED502A9B4F9F80132F0B1FF304688
:105E800002AA894906F1010BF9F708FE5FFA8BFBBC
:105E90005E466B6FD90619D5824B1B681A0615D55D
:105EA000B4F90402F8F788FE0246F8F7B7FE7F4916
:105EB000034602A8F3F73CFF304602AA7C4906F1EC
:105EC000010BF9F7EBFD5FFA8BFB5E466B6F9B06F0
:105ED00017D5B4F9FA110A2391FBF3F203FB12135D
:105EE000062100911BB2734902A8F3F721FF304647
:105EF00002AA714906F1010BF9F7D0FD5FFA8BFB9D
:105F00005E466B6F580615D50A230621BAFBF3F2DD
:105F100003FB12A300919BB2664902A8F3F708FFA6
:105F2000304602AA654906F1010AF9F7B7FD5FFAA2
:105F30008AFA56466B6F190617D5614B19880A23E2
:105F4000B1FBF3F203FB1213062100919BB25949F6
:105F500002A8F3F7EDFE304602AA5A4906F1010AFB
:105F6000F9F79CFD5FFA8AFA56466B6FDA0512D58F
:105F700002A994F8FE0132F033FF534902A834F02D
:105F8000C9FF304602AA514906F1010AF9F786FD18
:105F90005FFA8AFA56464E4B9B794BB36B6F9B0563
:105FA00012D502A9B4F9FC0132F01AFF494902A83E
:105FB00034F0B0FF304602AA474906F1010AF9F76A
:105FC0006DFD5FFA8AFA56466B6F580510D5434A45
:105FD00036499268072302A8F3F7AAFE304602AAC0
:105FE0003F4906F1010AF9F759FD5FFA8AFA564668
:105FF0006B6F19050ED5D4F8001202A8F9F7FEFC54
:10600000304602AA374906F1010AF9F747FD5FFA5F
:106010008AFA56466B6FDA0412D594F846397BB18A
:10602000032B0DD0304902A8F3F782FE304602AAB6
:106030002E4906F1010AF9F731FD5FFA8AFA564650
:106040006B6F9B0412D594F846397BB1032B0DD0AE
:1060500002A9002032F0C4FE304602AA244906F10B
:10606000010AF9F71BFD5FFA8AFA56466B6F58046E
:1060700051D5204B1B6899074DD594ED820AF2EE5D
:10608000047A20EE270A35F039F80A231A4990FBE2
:10609000F3F203FB120331E04A0A05085A0A050825
:1060A00040C50408A8B80020610A0508E9080508E9
:1060B0006B0A0508780A0508810A05088D0A050893
:1060C000608F0020910A05084B2A0508990A0508E7
:1060D000788F0020FA2A0508A20A0508888F002078
:1060E000AE0A0508B70A0508C40A0508CA0A050861
:1060F000D30A0508AC8600203A09050802A8F3F780
:1061000017FE304602AA7F4906F1010AF9F7C6FCDC
:106110005FFA8AFA56466B6F1A0415D5B4F90C0269
:10612000F9F7A4FC0246F8F73DFD7749034602A8BB
:10613000F3F7FEFD304602AA744906F1010AF9F7A9
:10614000ADFC5FFA8AFA56466B6FDB030ED502A9E7
:10615000D4F8100232F044FE304602AA6C4906F12F
:10616000010AF9F79BFC5FFA8AFA56466B6F9803AF
:1061700012D502A994F8140232F032FE654902A841
:1061800034F0C8FE304602AA634906F1010AF9F765
:1061900085FC5FFA8AFA56466B6F59037FF553AD5B
:1061A0005E4B1B681A067FF54EAD6423D4F82C07AE
:1061B000B0FBF3F0F8F700FD0246F8F72FFD584961
:1061C000034602A8F3F7B4FD02AA56493046F9F790
:1061D00065FC38E5032606E611F052FF0023C5F8FA
:1061E000003684F85539C4F8F4314F4BB9FBF3F954
:1061F0004E4B09F0010983F8EC91484B1A6812F0F4
:10620000006F994604D0FF202DF080FFC4F83C09B0
:10621000D4F8ECA1BAF1000F04D09AF90E30002B9B
:1062200000F33981424B1868F8F7C6FC834608F042
:10623000A3FF95F86830D5F8F865834295F8843067
:106240008CBF46F0010626F00106002B44D126F44F
:10625000800626F00206374BC5F8F8651B789B07C9
:106260000BD5354B9B7C042B07D994F834289A42E4
:1062700045D922F06BFE002841D046F48046C5F88F
:10628000F865B5F86A6006F00F00F9F7AFFC2B4B24
:10629000360A5E4325D1D5F8F83523F02003B5F84A
:1062A0006C60C5F8F83506F00F00F9F79FFC234B3A
:1062B000360A5E431CD1D5F8F83523F04003204957
:1062C000B5F864008968D5F8FC2588423ADD23F0EA
:1062D000102322F0200239E046F4800646F0020640
:1062E000B9E7B042D5F8F835D5D343F02003D6E767
:1062F000B042D5F8F835DED343F04003DFE726F4AB
:106300008046BCE7DE0A0508A6090508EA0A050872
:10631000F70A05084B2A0508030B0508A8B8002052
:10632000E90805080C0B0508400D030014000020C7
:10633000749300208093002010C4002000879303F2
:10634000888F002043F0102342F0200264219BFB41
:10635000F1FBB5F86610C5F8FC258B45ACBF43F4DE
:10636000004323F40043C5F8F835D9F8003018018C
:1063700010D595F9783013F1800F00F09480D4F89F
:106380003C1991F901109942C0F28D8042F0080247
:10639000C5F8FC25504611F073FE0E2022F05AFE7F
:1063A000002874D1494B4A4E00221A60326812F01C
:1063B000020F1A4623D0B5F85400F8F7E6FB10B9DF
:1063C0006B6F590415D5434BD3ED017AD3ED006AB9
:1063D00093ED027A404B67EEA77AE6EEA67AE7EEF7
:1063E000077AB1EEE77AD3ED007A67EE877AC2EDED
:1063F000007A0320FEF7B6FB2A20FEF7B3FBDFF896
:10640000DCA01AF807000137FEF7ACFB242FF8D107
:1064100033689A0614D50E20FEF7A4FB0D20FEF774
:10642000A1FB1820FEF79EFB1720FEF79BFB1F2009
:10643000FEF798FB1E20FEF795FB2F20FEF792FB40
:10644000D9F800301B0105D52320FEF78BFB242053
:10645000FEF788FB132022F0FDFD10B12C20FEF783
:1064600081FBB5F86000F8F790FB28B13020F9F710
:1064700087FB3020F9F732FBB5F86200F8F785FBAF
:1064800028B13120F9F77CFB3120F9F727FBD4F84C
:10649000EC0111F0C3FD98F8003003F0010384F81B
:1064A0003939FFF7EDBB22F00802C5F8FC2571E78A
:1064B000D4F8EC010368DB689847FFF7E4BB4FF4BE
:1064C000804028F025F8FFF7F0BB00BF9046002081
:1064D000AC860020E4460020988F002098CC040869
:1064E000064B93F90020064B12B91A700020704732
:1064F0001A78002AFAD10122F7E700BF881F00208E
:1065000066910020094B0A4A1978517159789171A6
:1065100099781170DA791A719A891A81DA895A810F
:106520009A8A1A82DA8A5A8200207047A04900208B
:10653000788F0020094A0A4B5179197091791278A5
:106540009A701A79DA711A899A815A89DA811A8AC3
:106550009A825A8A5970DA8200207047788F002018
:10656000A0490020044A054B117E9970517E927E0D
:10657000D9701A7100207047A049002010420020F5
:10658000044A054B91781976D178127959769A7622
:106590000020704710420020A04900200E4A0F48FA
:1065A000D37E517F03F00F0343EA0123D17F09011A
:1065B000C9B20B43A0F86A30917F137F92F8202074
:1065C00003F00F03120143EA0123D2B21343A0F8F0
:1065D0006C300020704700BFA0490020882C0020AC
:1065E0000C490D4BB1F86A2002F00F00D876C2F3C7
:1065F0000310120A5A77B1F86C20D87702F00F0115
:106600001977C2F30311120A83F820109A77002039
:10661000704700BF882C0020A0490020064A074B85
:1066200092F8211083F86810518C928CA3F86410B2
:10663000A3F8662000207047A0490020882C002085
:10664000064A074B92F8681083F82110B2F86410DC
:10665000B2F8662059849A8400207047882C002064
:10666000A049002008B564220249034834F0EAFB3F
:10667000002008BDC6490020882C002008B56422EF
:106680000249034834F0DEFB002008BD882C0020BE
:10669000C6490020084A0949B2F88A300B8292F8AC
:1066A0008C3092F88D2003EB83035B00CB81044B8D
:1066B00000209A70704700BFA0490020A0AB0020C6
:1066C00090A80020084A094B118AA3F88A10D289A1
:1066D0000A21B2FBF1F283F88C20054A927883F804
:1066E0008D200020704700BFA0AB0020A0490020F3
:1066F00090A8002030B1007910F1FF3018BF4FF0A2
:10670000FF3070474FF0FF307047074B93F88E20F3
:1067100042B9064A528802F0010283F88F20012212
:1067200083F88E2000207047A0490020A8B80020E0
:10673000034B002083F8900083F89100704700BF5E
:10674000A04900200A4B0B4A1B68B2F892105980EE
:10675000B2F89410A3F84C10B2F896109980B2F8E1
:106760009810B2F89A20D9801A800020704700BF94
:1067700084930020A04900200D4B93F89C206E21AB
:1067800001FB02320020B2F8A210A3F89210B2F876
:10679000EC10A3F89410B2F8A410A3F89610B2F875
:1067A000A610B2F8A020A3F89810A3F89A2070477A
:1067B000A04900200D4BB3F81422A3F8F421B3F83C
:1067C0001622A3F8F621B3F81822A3F8F821B3F89B
:1067D0001A22A3F8FA21B3F81C22A3F8FC21B3F87B
:1067E0001E22A3F8FE210020704700BFA049002010
:1067F0000D4BB3F8F421A3F81422B3F8F621A3F853
:106800001622B3F8F821A3F81822B3F8FA21A3F856
:106810001A22B3F8FC21A3F81C22B3F8FE21A3F836
:106820001E220020704700BFA0490020144B1549CC
:1068300093F8202230324A7093F89C206E2101FB9D
:106840000232002092F8E71083F8211292F8BA1071
:1068500083F8221292F8BB1083F8231292F8BC102E
:1068600083F82412B2F8D410A3F82612B2F8D2108A
:1068700092F8EF20A3F8281283F82A22704700BF6D
:10688000A04900200C0600200D4A92F89C306E2191
:1068900001FB032392F82B1283F8061192F82C12B5
:1068A00083F80A1192F82D1283F8071192F82E122C
:1068B00092F82F2283F8081183F8092100207047ED
:1068C000A04900200D4B93F89C206E2101FB023261
:1068D000002092F8061183F82B1292F80A1183F81F
:1068E0002C1292F8071183F82D1292F8081192F8E1
:1068F000092183F82E1283F82F227047A049002027
:106900000E4B0F4993F8202230320A7193F830224F
:1069100030328A7193F84C220A491A2000FB021285
:1069200003F2322302F1180152F8040B43F8040B6E
:106930008A42F9D112881A8000207047A0490020AD
:106940000C0600208C42002010B50A4A0A4892F832
:106950004C321A2402F2322104FB030302F24A22CF
:1069600051F8040B43F8040B9142F9D10A881A80BC
:10697000002010BDA04900208C42002010B5124A12
:10698000124992F8203292F89C0030334B7002F199
:10699000A0016E2300FB031302F24D21002002F23E
:1069A00056221C7A0C705C7A4C709C7A8C709C8994
:1069B00022F810400130032803F1060301F103011E
:1069C000EFD1002010BD00BFA04900200C06002020
:1069D0000749084B0A7883F89C20013283F820226B
:1069E0004A7883F84C22013283F830220020704725
:1069F00090A80020A0490020064A002302F5177045
:106A0000194619540133072BFBD182F86312002079
:106A1000704700BFA0490020084B93F86422012A68
:106A2000074A05D893F86512032918BF032191700E
:106A3000B3F8663213800020704700BFA0490020E1
:106A4000C446002010B5044623790E2B00D110BD9A
:106A5000032B03D1E3689868FFF7F4FF1434F3E7DE
:106A60000B49D1F868329A68134618790E280CD170
:106A70009B1A9A10074B5343013B91F8712293FBE9
:106A8000F2F3013381F8703270471433EDE700BF41
:106A9000A0490020CDCCCCCC084BD3F8740210B563
:106AA00058B1074CA168013191FBF0F200FB1210C4
:106AB00003EB8003A060D3F8780210BDA04900204A
:106AC0000C06002030B44FF4983240F29E730D4D06
:106AD000026043834FF4E17203230B4C0B49C56101
:106AE00002840825962280F82230002380F8235063
:106AF0004462C0F81610826043608382C360036101
:106B000030BC70477D0096007800960002010001BD
:106B100000230122C270837003800371437183716B
:106B2000C37103724372704700230A2203604360FB
:106B3000C381C0F80630C0F80A30028070472DE9E2
:106B4000F843794C94F88F2294F890329A4200F0EE
:106B5000888094F88F2294F88F32C2EBC20204EB43
:106B60008202C3EBC30304EB830392F8B31293F8DE
:106B700098628B1E9E422FD06C4AB4F8EC32127889
:106B8000D4F8941201339BB21C2AA4F8EC326CD0D6
:106B9000002594F88F32664A0133A2FB03025208A3
:106BA00002EB42029B1ADBB284F88F3200293DD0FF
:106BB0000CF0E0FCD4F82033C01AB0F5FA7F04DB07
:106BC000002345F0040584F81E33D4F81833002B55
:106BD00034D12846BDE8F88394F88F3204F526773F
:106BE000C3EBC30307EB830361B11944002213F81D
